:020000040800F2
:1040000000500020C1F800082DCA000831CA00087D
:1040100035CA000839CA00083DCA0008000000007F
:1040200000000000000000000000000045CA000879
:1040300041CA00080000000049CA00083998000879
:104040004DCA000851CA000855CA000859CA0008DC
:104050005DCA000861CA000865CA000869CA00088C
:104060006DCA000871CA000875CA00080000000087
:104070000000000000000000000000000000000040
:10408000000000000000000095CA000899CA00085E
:10409000A9CA0008B9CA0008C9CA0008B14900087D
:1040A000DDCA0008E1CA0008E5CA0008E9CA00083C
:1040B000EDCA0008F1CA0008F5CA0008F9CA0008EC
:1040C000FDCA000801CB000805CB000809CB000899
:1040D0000DCB000811CB0008218D0008E58D0008EC
:1040E0001DCB000821CB000825CB000800000000F4
:1040F00000000000000000000000000000000000C0
:0C41000000000000000000005FF800005C
:1041100030BF704720BF704740BF7047BFF36F8FFD
:104120007047BFF34F8F7047BFF35F8F704701DF5A
:104130007047EFF31480704780F31488BFF36F8FDC
:104140007047EFF30980704780F309887047EFF3F9
:104150000880704780F30888704772B6704762B66F
:10416000704771B6704761B6704780F31188704729
:10417000EFF31280704740BA704700BA70470000F2
:1041800010B500F03FFC0B4C0B490C4A0C4B48B1EE
:104190004FF0010C0B4884F800C00B4C1860146001
:1041A000086006E020700948086009491160094A62
:1041B0001A6010BD700B0020980B00207C0C0020B2
:1041C0000C0C0020B1910008E19F00084592000806
:1041D00081970008C996000837B50AF043F86B4B81
:1041E00000254FF480301D700AF05CF80AF0C0F929
:1041F0000128044627D1102009F01EFB28460AF0AA
:10420000A1F828460AF0B2F84FF480600AF0A4F84A
:104210004FF440304FF4E0110AF070F820460AF0F5
:1042200079F839200AF08EF90028FAD0022009F036
:10423000EBFA02200AF074F80AF07CF80828FBD1A7
:10424000524B01221A70042001210AF031F9032394
:104250008DF80630153301A94D488DF807304FF41D
:104260008073ADF8043009F01BFD06200AF064F9F4
:10427000012001460AF01CF9464C4FF480414FF0F2
:10428000006009F011FF4FF4407009F06FFE00F07C
:1042900001FC00F0A9FDFFF773FF00F0F3F805F053
:1042A0000FFC05F06BFB04F015FC00F079F82078AA
:1042B00004F0AAFEE07804F09BFC207804F0EAFD0C
:1042C000E07804F0BDFC344B1B7823B92269607997
:1042D000A16805F051F8304B1B780BB105F030FFA9
:1042E00006F0B8FC00F016FA08F072F900F066F972
:1042F00001F094FE05F040FF06F0F2FC274B4FF46E
:1043000000521A6105F034FB044603F099FC06F0F4
:10431000F5FC05F06BFF05F02BFB001B0028B8BF78
:104320004042B0F57A7F24DD1B4D2B782C4683B1BB
:1043300000F068FB68B9287005F0C2FE05F0A0FD2A
:10434000FFF71EFF134B1A695879996805F014F8A6
:104350000CE0237853B900F055FB38B104F0D0FFDE
:1043600001232370FFF70CFF05F0EAFE05F000FBC8
:10437000044600F05FF900F051F90028C5D006F0BE
:1043800069FC01F04BFE06F0ABFCBEE76C0C0020B4
:104390000008014008000020700B002000100140C0
:1043A000114B82B01B78E3B1104B08225A610422F2
:1043B0001A61002301E0019B01330193019A0C4B28
:1043C0009A42F8D9094B08221A6104225A61002343
:1043D00001E0019B01330193019A054B9A42E3D816
:1043E000F7E702B0704700BFAC0B0020001001409F
:1043F0003F0D030010B1012805D101E0402200E08B
:104400008022014B5A617047000C014010B1012815
:1044100005D101E0402200E08022014B1A61704783
:10442000000C014038B50546002455FA04F2E3B209
:1044300012F0010F184602D0FFF7E8FF01E0FFF786
:10444000D9FF0134082CF0D138BD00BF18B10128C4
:1044500006D0002008E0054BD868C0F3801003E0C8
:10446000024BD868C0F3C010704700BF000C014079
:1044700008B1002003E0024B9868C0F38000704749
:10448000000C014062B6704772B6704718B9024B13
:104490004FF400521A6170470010014018B9024BE6
:1044A0004FF400525A6170470010014010F0010FA4
:1044B00003D00E4B08221A6102E00C4B08225A610D
:1044C00010F0020F03D0094B10221A6102E0074BD3
:1044D00010225A6110F0040F03D0044B20221A61FD
:1044E00002E0024B20225A61704700BF000C0140DD
:1044F00008B1002005E0034BD3E90023100A40EA8D
:1045000003607047B00B0020F8B50D460446B8B9FB
:10451000FFF7BAFF0B492A464FEAE273C1E90023CD
:10452000D1E900673B0243EA16633202C1E9002386
:10453000054B1C60054B1C60054B9C84FFF7A2FFDC
:10454000F8BD00BFB00B0020B80C0020900B00207D
:104550000004004010B9024B09011960704700BF08
:10456000B80B002020BB11F0040F10D011F0100F79
:1045700004D0104B9A6842F480720CE00D4B9A689C
:1045800022F480729A60DA6842F4807207E0094B84
:104590009A6822F480729A60DA6822F4807211F0CC
:1045A0000801DA60044B02D001221A7000E0197091
:1045B000704700BF0004014030020020084B4FF458
:1045C00000721A60074B10B50024204610211C60B1
:1045D000FFF7C0FF20462146FFF7C4FF10BD00BF14
:1045E000A00B00209C0B002010B9024B09011960A0
:1045F000704700BF0400002008B9014B5970704794
:1046000030020020044B98780138C0B201288CBFDA
:1046100000200120704700BF30020020044B987832
:10462000012801D0002001E002229A70704700BFEB
:1046300030020020082008B505F0B6F9592804D941
:10464000064B9A784AB9013206E0082005F0ACF929
:10465000542802D8014B00229A7008BD3002002075
:10466000012808B505D003D30A280AD000200CE0A1
:10467000002005F099F9B0F5006F94BF00200120EB
:1046800003E0024B9868C0F3402008BD00100140D1
:1046900038B500242546E0B2FFF7E2FF20B1012340
:1046A000A34043EA0505EDB20134082CF3D12846B6
:1046B00038BD00BF10B5FF210022032000F01AFB17
:1046C000FF210122032000F015FBFF21002203201F
:1046D00000F010FBFF2104460122032000F00AFB3A
:1046E000034B40EA04205B6803EA9000181A10BDEF
:1046F0003002002008B5FFF7DDFF052801D80120B2
:1047000007E0FFF7D7FF40F2F933984294BF00204B
:10471000012008BD38B51E4C002021694909FFF76A
:1047200063FF2169002001F01F01FFF765FFFE21F3
:104730000022032000F0DEFA40210122032000F0D5
:10474000D9FA00210A46032000F0D4FA00210446D9
:104750000122032000F0CEFA082C0E4B05D14FF4B5
:1047600000629A6040F6FF7204E04FF400729A60B3
:1047700040F2FF325A60FFF79DFF064B04022446C9
:104780004FEAE475C3E90645C3E90445D86038BD7E
:10479000100C0020300200202DE9F84305F0E8F865
:1047A000624C2062FFF786FFE368606298423EDD5C
:1047B000A268C11A91420BDA5D4BA56A1A684D19BD
:1047C0005143D4E90667721847EBE173A5622BE009
:1047D00094F801C0564A1CF0040F12D063681668A2
:1047E000C31A5E432CF0040C36464FEAE677A36208
:1047F00000220023C4E9066784F801C0C4E9042349
:104800004EE0656816685A190132121A7243D4E9EB
:104810000667A36AED43ED18B6EB020867EBE27991
:1048200042464B466918A162C4E9062338E037DAEC
:10483000A1681A1A8A420EDA3D4DA16A2D68C91A7A
:104840006A43D4E90667B6EB020867EBE2794246B1
:104850004B460918E7E76178354A11F0040F0FD08D
:10486000126821F00401424312464FEAE273C4E9A0
:104870000623002200236170C4E90423A0620FE034
:10488000616812680131CB1A1B185A43D4E90667D4
:10489000B61847EBE277A26AC4E906679B18A362E1
:1048A000224B9D6ADA6A196BAA1A82EAE27CACEBA7
:1048B000E27C8C452CD942F210714A431E6A5C6B33
:1048C0003C21341B92FBF4F251434FF4807C91FB6A
:1048D000FCF181EAE172A2EBE172D96340F6B831F2
:1048E0008A425E63DD629C6301DDC82219E0B2F595
:1048F0007A7F01DD642214E0322A01DD0A2210E011
:104900000A2A01DD05220CE0012A0BDD012208E064
:10491000196A5A6B8A1AB2F5FA6F03D90022DA6360
:1049200001321A63014BD860BDE8F88330020020E1
:104930000400002038B50D4618BB124CFFF72CFFC1
:10494000D4E90601002901DB626803E062684042A5
:1049500061EB4101120212464FEAE2730DF0D0FD05
:10496000C4E9042328464FEAE071064C0B02020218
:1049700043EA1063D4E90401801841EB0301C4E960
:10498000060138BD3002002008B508B100200CE057
:10499000FFF702FF054BD3E90401D3E90623121AFE
:1049A00063EB0103100A40EA036008BD30020020F7
:1049B00008B54FF4807008F021FF0C4A0023136003
:1049C0000B4A002013600B4A0021C2E900010A4A89
:1049D00093840A4B1B7843B9094B9A6822F480727E
:1049E0009A60DA6822F48072DA6008BDB80C0020A0
:1049F000900B0020B00B002000040040300200208B
:104A00000004014008B5084B587E10F0010005D0A5
:104A1000002007F0EFF980F0080001E007F0EAF964
:104A2000C0F3C00008BD00BF0800002010B5044658
:104A3000C0B1002007F040FC0221002007F0C4FABA
:104A4000421E0020014607F071FB0020024601468D
:104A500007F094FA6821002007F0B6FA40F0080247
:104A6000002005E0682107F0AFFA20F00802204698
:104A7000682107F05BFB10BD08B510B109F01EFB03
:104A800001E009F023FB08BD08B5C90805F04CFD9D
:104A900008BD00BF2DE9F04501218BB0DFF8488249
:104AA0008B4809AC09F08CF904200121032709F097
:104AB000FFFC10254046214642F21303ADF8243096
:104AC0008DF826708DF8275009F0EAF840F203239C
:104AD0000426C8F810504046DFF814A22146C8F852
:104AE00014304CF20063ADF824308DF826708DF848
:104AF000276009F0D5F80820012109F0D9FC2146EA
:104B000041F2F8035046ADF824308DF826708DF848
:104B1000275009F0C5F841F2380321465046CAF83B
:104B200010304FF0070308F50068ADF824308DF819
:104B300026708DF8276009F0B3F82846012109F0A6
:104B4000B7FC404621464EF20C038DF82750ADF8D5
:104B500024308DF8267009F0A3F84CF20C03C8F845
:104B6000103042F2300340462146C8F814304FF46A
:104B7000FE53ADF824308DF826708DF8276009F0CB
:104B80008FF82020012109F093FC214651488DF82F
:104B90002670ADF824608DF8276009F081F80220B6
:104BA00001214D4C09F084FC01214C4809F008F921
:104BB0000121022009F08AFC03AD20460AF058FCCE
:104BC00028460AF04BF8294620464FF000054FF0E2
:104BD000FF33ADF81030ADF80C50ADF81250ADF811
:104BE0000E5009F0E3FE00221346394620460AF033
:104BF000EBF868460AF046F84FF008082046694688
:104C0000ADF808800AF0D0FB20466946ADF8006098
:104C10000AF0CAFB204641F65F610AF01BFB204602
:104C20000121A5840AF042F80821022009F0F6F8D3
:104C300001244FF4807306A806938DF81D808DF82B
:104C40001C508DF81E4008F073FD254B08A89A688B
:104C50008DF8234022F480729A60DA686F4622F45D
:104C60008072DA6017238DF820308DF822508DF88D
:104C7000215009F085F921461A4809F0A1F80023CE
:104C800019461A46184C4FF4005565612046A46831
:104C9000013114F4804F4FF400540461806808BF60
:104CA000013310F4804F18BF01320A29EAD10A2BD0
:104CB00003D10A2A01D1012200E000220B4B044853
:104CC0001A70012109F07CF80BB0BDE8F08500BF37
:104CD000000230000014014000040040000C1A00E3
:104CE000000401400004300000080140AC0B00202B
:104CF000000C014070B504460D461646032867D8DF
:104D0000DFE800F00206090E4FF48052314B11E04B
:104D10001022314B02E0314B4FF480425A611BE0CC
:104D20002F4A138823F002031B041B0C13802B4B08
:104D30004FF400425A612A48022109F01BFD002865
:104D4000F9D02946264809F0B9FC2548012109F087
:104D500011FD0028F9D00FE02248022109F00AFDD8
:104D60000028F9D029461F4809F0A8FC1D48012158
:104D700009F000FD0028F9D0EEB1032C28D8DFE8B7
:104D800004F002070A0F134B4FF480521A611AE025
:104D90001022114B02E0114B4FF480421A6110E0D7
:104DA0000E4A0F4B4FF4004111611A8892B242F043
:104DB00002021A8007E0032C0AD8DFE804F004029C
:104DC0000204084800E0064809F07AFCC0B200E09E
:104DD000002070BD000C014000080140001001409F
:104DE00000380040003001402DE9F04F01218BB028
:104DF0004FF4804009F06AFB494C012009AF01469D
:104E000009F056FB03264FF0180B204639464AF2AC
:104E10000003DFF81491ADF824304FF0040A8DF848
:104E200026608DF827B008F03BFF204639464FF446
:104E300080430DF11008ADF824308DF826608DF810
:104E400027A008F02DFF4FF48273002402224FF4B4
:104E5000007C012548464146ADF812304FF008036A
:104E6000ADF81620ADF81AC00392CDF808C0ADF821
:104E70001C30ADF81040ADF81440ADF81850ADF846
:104E80001E40ADF8204009F0A5FB4846294609F030
:104E9000DDFB29464FF4805009F00AFB09F5504923
:104EA0002846214608F08CFF484639464FF0A003BB
:104EB000ADF824308DF827B08DF8266008F0F0FEAC
:104EC000484639464FF04003ADF824308DF826604F
:104ED0008DF827A008F0E4FE039ADDF808C04FF42F
:104EE00082734146ADF812300E484FF02803ADF8FA
:104EF0001620ADF81AC0ADF82040ADF81040ADF85E
:104F00001440ADF81850ADF81C30ADF81E4009F053
:104F100061FB0448294609F099FB0BB0BDE8F08F0E
:104F2000000C01400030014000380040014B18786F
:104F3000704700BF700200202DE9F8450546144671
:104F40000E4600294BD0002849D0814247D04FEA75
:104F500042185FFA88F848F006073946002007F043
:104F600033F848F00C018246002007F02DF8804607
:104F700028460DF087F8054630460DF083F80146C7
:104F800028460DF08BF9064650460DF07BF8314669
:104F90000DF084F90DF094FA054640460DF072F8D4
:104FA00031460DF07BF90DF08BFA0E49002814BF45
:104FB00080464FF001083046002D08BF01250DF056
:104FC00057FA18B14146204607F078FA39462A4682
:104FD000002007F0ABF8044BE41801232371BDE86F
:104FE000F88500BF0000A0417002002070B50D4D93
:104FF000044645192B799BB1C6B20B4B710141F0A8
:10500000060153F8202001F0E601002007F022F904
:10501000064B304653F8241007F050FA00232B714A
:1050200070BD00BF70020020680B002064070020E4
:1050300013B5A14CA078002840F031836378A62BEB
:1050400000F06C825FD8852B00F0F08027D8072B0A
:1050500000F024810FD8032B00F0E88005D8012B45
:1050600000F0BC8000F2C480B2E0052B00F0F680B6
:1050700000F20981E0E0812B00F0B08009D80D2B0F
:1050800000F03A81802B00F0A3800C2B40F00583C8
:1050900020E1832B00F0D08000F2AA803EE1952B26
:1050A00000F0708115D88C2B00F05D8108D8872B1B
:1050B00000F03E81C0F0D2808A2B40F0EE823DE1CC
:1050C000932B00F0198100F205818D2B40F0E582D1
:1050D00052E1A12B00F0F48109D89A2B00F08281D3
:1050E000A02B00F0E781992B40F0D78265E1A32B3C
:1050F00000F0F081C0F0E881A42B00F0F181A52B35
:1051000040F0CB82FBE1B82B00F0818229D8AE2B96
:1051100000F0448211D8AA2B00F01D8206D8A82BDB
:1051200000F00E82644B00F2118204E2AC2B00F01E
:105130002482614B00F22D821AE2B22B00F04382EE
:1051400006D8B02B00F034825B4B00F237822AE2A3
:10515000B62B00F0448200F25582B52B40F09D82C0
:1051600035E2D12B00F0578216D8C32B00F05F81B7
:1051700008D8C12B00F04F8100F25281C02B40F0C3
:105180008C828BE0C82B00F05981CC2B00F066811B
:10519000C72B40F0828276E0D62B00F0748108D8CD
:1051A000D42B00F0638100F26981D22B40F075822C
:1051B00038E2D92B00F0548203D8D82B40F06D820E
:1051C00045E2DA2B00F06182FE2B40F0668261E15D
:1051D000394B00205A680146DB7804E0364B00204A
:1051E0005A68DB78022143EA022206F09FFF59E267
:1051F000314C0020E3786268082143EA022207F07C
:1052000029F8E378A1786268490143EA0222002A7A
:1052100041F00601B8BF524201F0E601002007F05C
:1052200019F8264AA378D3180122EEE1224B002078
:105230005A680A21DB7876E01F4C0020E378626828
:10524000062143EA022207F005F8E2786068A378B5
:1052500042EA0020194A1A499A180FE0164C002019
:10526000E378616843EA012107F028F9E278606891
:10527000A37842EA0020114A12499A1841F8230003
:10528000002313710EE20C4B0F4AD9780F4B01200B
:105290001B7810700E4A022B5172D9E0064B012286
:1052A000D9780A4B1878084B1A70094B9972002864
:1052B00040F0F881CFE000BFE0060020700200203F
:1052C000680B002064070020740C0020780C00207C
:1052D000100C00201421002001AA06F0C7FEA04AED
:1052E0009DF805305168D27852EA012114BF43F08D
:1052F000020323F0020354E01421002001AA06F067
:10530000B5FE974A9DF805305168D27852EA0121DE
:1053100014BF43F0010323F0010342E0904B00204F
:105320005A68DB78042143EA022206F093FFB9E1D0
:105330008B4B00205A680E21DB78F4E701AC224643
:105340001421002006F092FE854B22469978DB78E6
:10535000490141F0140101F0F40100208DF80630FC
:1053600007F020F89EE1E3787E4AC3F10801C9B254
:10537000D37205F0F3FB95E1794B00205A681A21AE
:10538000DB78D0E7142101AA06F070FE6168E278AC
:105390009DF8053052EA012114BF43F0040323F0C5
:1053A00004038DF805306E4B0020997801AA49015D
:1053B00041F0140101F0F401D2E701AC22461821BA
:1053C000002006F053FE664A9DF805309178D278A9
:1053D000490102F00F0223F00F0341F0180142EAE5
:1053E000030311E001AC22461821002006F03EFE26
:1053F0005B4A9DF805309178D278490103F00F039C
:1054000041F0180143EA021301F0F801224600209E
:105410008DF80530A4E7524BDA78524B1A7241E10D
:105420004F4B5A68DB7843EA02224E4B33E1E37874
:10543000626843EA02224B4B5A6033E1484B4A4AC6
:10544000D9784A4B01201B781070464A032BD1773C
:1054500040F028810138FFF717FB23E1404B5A68E1
:10546000DB7843EA02223F4BDA811BE13C4B5A686E
:10547000DB7843EA02223B4B5A6113E1384BDA787E
:10548000384B9A770EE1E378626843EA0222354BA3
:105490009A8307E1324B334A5968DB7843EA0121AA
:1054A000052904D818461373FFF7C0FAFAE0002361
:1054B0001373F7E02A4B0020D97805F041FBF1E0A7
:1054C000E17805F033FBEDE0254B0020D97805F0BD
:1054D0000DFAE7E0224B0020D97805F0FBF9E1E076
:1054E000002004F0B9FE1E4B20B9D978987805F059
:1054F000D9F9D7E0D978987805F0A4F9D2E000205E
:1055000004F0AAFE164B20B9D978987805F0BEF9B8
:10551000C8E0D978987805F07DF9C3E004F09CFEE6
:10552000E178A37818B9184605F0A4F9BAE018464E
:1055300005F07CF9B6E0D978002005F08FF9B1E0EC
:10554000074B0020D97805F093F8ABE0D97800201C
:1055500005F082F8A6E0E17805F072F8A2E000BF5D
:10556000E0060020100C0020740C0020780C0020B5
:10557000D978002005F058F894E04B4C0020E178F1
:1055800005F046F8A178494BE27803EBC1035A7164
:1055900088E0D978002004F0DFFF83E094F903105D
:1055A00004F0CEFF7EE0D978002005F063FA79E0C0
:1055B0003D4B0020D97805F051FA73E0D9780020EE
:1055C00005F040FA6EE0E17805F030FA6AE0364B1B
:1055D0005A68DB7843EA0222354B9A6162E0324A2C
:1055E000324B5068D27842EA0020186010B95979DD
:1055F00005F00EF82C4B2F4A9878125C012A51D1F5
:10560000D97828E7284BDA78284B1A714AE0E178F4
:1056100005F054F946E06168E37843EA0121FFF7B9
:1056200089F93FE0204C0020E378626803F01F0115
:1056300043EA02221E4B1A61FEF7DEFFE37861683F
:10564000A07843EA01214911FEF7CEFF2AE0164B6C
:1056500000205968DB7843EA0121FEF755FF21E07D
:10566000114C0020E378626803F01F0143EA022234
:10567000114B1A60FEF776FFE3786168A07843EA81
:1056800001214911FEF766FF0CE0074B5A68DB78F1
:1056900043EA0222094B1A6004E0032200E00422DC
:1056A000074B1A701CBD00BFE0060020800B0020D5
:1056B000100C0020780C0020A00B00209C0B002078
:1056C0005807002013B5AD4CA078002840F0728236
:1056D0006378A62B00F00782A94C7DD8852B00F0BB
:1056E0000B813AD8092B00F032811CD8042B00F032
:1056F00006810CD8012B00F0F680002B00F0F08022
:10570000022B00F0F680032B40F05182F4E0062BD0
:1057100000F0FA80C0F0F580072B00F0F880082B2D
:1057200040F04582F6E0802B00F0DA8009D80B2BA0
:1057300000F01281C0F02E810C2B00F0F4800D2BB4
:1057400024E0822B00F03381C0F0CD80832B00F069
:10575000D680842B40F02B82CBE09A2B00F0558131
:105760001ED88D2B00F039810BD8872B00F02481B7
:10577000C0F0C7808A2B00F022818C2B40F017826A
:1057800025E1942B00F0CF8003D8932B40F00F82BB
:10579000D3E0952B00F02581992B40F008822AE177
:1057A000A12B00F077810BD89C2B00F0F380C0F088
:1057B000D3809D2B00F0AE80A02B40F0F88165E1F6
:1057C000A32B00F06E81C0F06881A42B00F06F81E4
:1057D000A52B40F0EC8178E1C12B00F01E813BD875
:1057E000B02B00F0B0811BD8AB2B00F099810BD807
:1057F000A82B00F08981C0F08381A92B00F088815B
:10580000AA2B40F0D48187E1AD2B00F08F81C0F04E
:105810008A81AE2B00F08E81AF2B40F0C8818EE1E3
:10582000B52B00F0A2810BD8B22B00F09381C0F011
:105830008D81B32B00F09281B42B40F0B88191E1BF
:10584000B72B00F09881C0F09481B82B00F09681BE
:10585000C02B40F0AC815AE0D02B00F008811DD85D
:10586000C72B51D00BD8C32B00F0DC80C0F0D88000
:10587000C42B00F0DA80C52B40F09981D7E0CC2B07
:1058800000F0DA8003D8C82B40F09181D1E0CE2B14
:1058900000F0D580CF2B40F08A81D2E0D62B00F0EB
:1058A000EF800BD8D22B00F07181C0F06B81D42B2C
:1058B00000F0E080D52B40F07A81DEE0D92B00F0BB
:1058C0006F8106D8D72B00F06481D82B40F06F8110
:1058D00062E1DA2B00F06681FE2B40F06881D2E0B5
:1058E0000020014601E00020022106F06DFB60600F
:1058F00063E10020082171E000200A2159E0214BDA
:1059000000E0214B1B6832E1204B5B7A2FE11F4BFB
:105910009B7A2CE1002006F06DFA184B9B785B0017
:1059200050FA03F310E00020142101AA06F09EFBB8
:105930009DF80530C3F3400319E10020142101AAAA
:1059400006F094FB9DF8053003F001030FE1104BC6
:105950009B68C3F3C0330AE17C21002001AA06F052
:1059600085FB064B02219A789DF80630520011FA09
:1059700002F21A420CBF00230123F8E0E0060020E7
:1059800058070020680B002064070020100C00203E
:105990000008014001AA00207C2106F067FB904B23
:1059A0009DF806209B785B0052FA03F3CCE70020B9
:1059B000042106F043FB77E000200E21F9E701AA5D
:1059C0000020142106F052FB9DF80620ECE0002098
:1059D00004F022FCC0F1080066E01A2106F02EFB5C
:1059E00085E701AA0020142106F040FB9DF8052060
:1059F000C2F38002D8E001AA0020182106F036FB8D
:105A00009DF8052002F00F02CEE0182101AA06F051
:105A10002DFB9DF805301B09A9E0724B1B7AA6E00F
:105A2000704BC0E06F4B5A68BEE06F4BBBE06F4BF2
:105A3000B9E06C4BDA7FB7E06A4BDA89B4E06C4BC3
:105A4000B1E06C4A6C4B1278002159600AB1012216
:105A50005A606A4B674A1B780021117023B1664B6C
:105A60005A6842F002025A600022644BA4E0644B80
:105A70001B787CE05B4B5A6996E05A4B9A7F93E027
:105A8000584B9B8B73E0574B1A7B8DE0002004F042
:105A9000CBFB09E004F0D0FB29E7002004F0D4FBA5
:105AA00002E0002004F0D8FB534B586085E0002052
:105AB00004F0D2FB504C4A4B18B9987804F0DCFB48
:105AC00015E7987804F0F8FB11E7002004F0C4FB18
:105AD000494C434B18B9987804F0D6FB07E79878FF
:105AE00004F0FAFB03E704F0B7FBA378424C18B9C3
:105AF000184604F0D1FBFAE6184604F0E5FBF6E69A
:105B0000002004F0D1FBCFE7002004F0EDFBCBE751
:105B1000002004F0F1FBC7E7002004F0F5FBC3E729
:105B200004F0FAFBE3E6374B5A793DE0002004F03D
:105B300003FCB9E7002004F007FC40B2B4E7002002
:105B400004F014FCB0E704F019FCD0E6002004F0E7
:105B50001DFCA9E7002004F021FCA5E7002004F0CB
:105B60002DFCA1E7284B1A781EE01E4B9B69636051
:105B700023E0244B17E0234B1A7915E0002004F0B2
:105B800073FB91E70020FEF7FFFE8DE7154B1A69C6
:105B90000AE0FEF78FFD87E70020FEF7A9FC83E708
:105BA0001A4B00E01A4B1A68134B5A6005E00323A6
:105BB000237002E0104B04221A70164B1B786BB155
:105BC0000D4B15495A68154B0A601AB91A6842F00C
:105BD000080202E01A6822F008021A601CBD00BF29
:105BE000E0060020100C0020740B0020340C002074
:105BF000A80B0020040C0020580700208C0B00206C
:105C0000080C0020800B00207C0B0020A00B002043
:105C10009C0B00205207002040070020E8060020CF
:105C200010B51B4A5378142B2DD8917871B954684C
:105C3000D078184A1849927E40EA042041F823009F
:105C400022B31BB303F5C270013013E0FF2918D152
:105C500063B94FF4C364114920460919042204347E
:105C600002F070FDB4F5CD6FF5D10FE003F5C27011
:105C70000949013001EB83018000042202F062FD3A
:105C800004E0042200E00322054B1A7010BD00BF9F
:105C9000E006002008000020EC060020D8000020CC
:105CA0005807002038B51F4C6578142D36D8A078D9
:105CB00010F0800F18D010F0010F06D00020022144
:105CC00006F082F9184B43F82500184B9B7E43B32E
:105CD000144B5B782BB303F5C2701349013001EB11
:105CE00083018000042214E0B0B9022106F06CF9AF
:105CF0000E4A0D4B927E43F8250092B1617881B136
:105D0000A0780422091801F5C270013003EB81016B
:105D1000800002F017FD04E0042200E00322044B9F
:105D20001A7038BDE0060020EC06002008000020B4
:105D30005807002038B56E4CA07808B10422D3E093
:105D400063789A2B22D8992B80F09B80822B00F0CD
:105D500081800BD8062B6ED003D8042B38D0052BAE
:105D60000AE0072B6DD00C3B012B0CE08C2B75D07F
:105D700005D8832B2CD0862B40F0B5803FE08D2BAF
:105D80007DD0933B022B00F2AE8060E0C72B52D057
:105D90000ED8C12B7AD005D8B52B74D0C02B40F0CB
:105DA000A2804EE0C22B77D0C32B40F09C8076E0DF
:105DB000D42B7DD005D8C82B74D0CC2B40F0938049
:105DC00073E0D62B7CD077D3FE2B40F08C807DE027
:105DD000474D0020062106F04FFBAC780020610102
:105DE00041F0060101F0E60106F028F9414AAB78DE
:105DF000D318414A42F8240000221A7176E03C4D43
:105E000000200C2106F038FBAC780020610141F045
:105E10000C0101F0EC0106F011F9AB78374A354975
:105E200042F8240018465B1852F8201000221A711C
:105E300006F044FB5AE0492002F06CFC304B5872EB
:105E400054E04A2002F066FC2D4B98724EE0002090
:105E5000142100E0042106F00FFB47E04B20012253
:105E6000284902F033FCA378254A184602EB431375
:105E7000D97AC1F10801C9B204F070FE36E01A21E6
:105E8000E9E71821E7E758201F4913E0482002F00E
:105E900041FC1B4B187229E0402019490AE04420BC
:105EA0001A4907E05F201A4908E04E20194909E025
:105EB00019495420042206E018495E20012202E01C
:105EC00017495C20022202F001FC0FE04C20012265
:105ED000144902F0FBFBA278094B03EB4213187B39
:105EE000FEF7A4FD02E003220F4B1A7038BD00BF7D
:105EF000E006002070020020680B002064070020EC
:105F0000100C00201B0C0020280C0020140C00207A
:105F10002F0C00201E0C0020240C00202E0C002032
:105F20002C0C00201C0C00205807002010B51E4A25
:105F30005378142B34D89278AAB91C4A1C4952F8C9
:105F400023201C4B4A601B78002B2CD01A491B4B7A
:105F50000A601AB91A6842F0080202E01A6822F0D0
:105F600008021A601FE0FF2A18D163B94FF4C36416
:105F70001349204609190422043402F0A7FBB4F5A2
:105F8000CD6FF5D10FE003F5C2700849013001EB88
:105F900083018000042202F099FB04E0042200E067
:105FA0000322034B1A7010BDE0060020EC0600200F
:105FB000580700205207002040070020E806002074
:105FC000D800002037B5134C657815B1012D1DD1CF
:105FD00012E0042240F2FB7001A902F077FBE378A3
:105FE000626843EA0222019B9A420B4B02D10122D2
:105FF0005A600EE05D600CE0A3782A2B06D1E11C0C
:1060000040F2FB70042202F09DFB02E0024B0322EF
:106010001A703EBDE006002058070020374938B509
:1060200000230B603649374A0B60374993740B6085
:106030009360D36013745374344A4FF0FF3142F8C5
:106040002310334A0024D45401332F2BF4D10731C9
:10605000204605F0B9FF2F4B0C211860204605F0B3
:10606000B3FF2D4D2D4BE97A1860C1F10801204690
:10607000C9B204F073FD287BFEF7D8FC284B002240
:10608000E2500434B4F5806FF8D1264B9B7E5BB1AF
:1060900004F506742449204609190422043402F048
:1060A00015FBB4F5CD6FF5D11E4BDB7E5BB94FF41C
:1060B000A7641E49204609190422043402F006FB95
:1060C000B4F5C36FF5D1174B1B79012B03D0112BFE
:1060D00001D0212B01D1012200E00022094B83F8DD
:1060E000D020104B5B7D23B1FEF78CFA08B1012262
:1060F00000E00022034B83F8D12038BD4007002088
:106100006007002070020020E806002084020020C2
:10611000880C0020680B0020100C00206407002071
:106120006807002008000020D8000020300200206E
:1061300008B50B4B5A7892B9997881B95A68DB78CF
:1061400043EA022240F2D2439A4208D140F2FF7061
:1061500002F076FB02F038FC0120FEF78DFC08BD52
:10616000E006002010B59A4B9A78022A00F05A8176
:10617000032A00F06081002A40F0F0815A784D2A0D
:1061800000F0BD8023D8452A70D00ED8422A56D0C0
:1061900005D8402A45D0412A40F0DE8146E0432A16
:1061A00053D0442A40F0D88156E0482A7CD005D804
:1061B000462A61D0472A40F0CF816AE04B2A00F09E
:1061C000858000F29580492A40F0C68172E0542A09
:1061D00000F0E48011D8512A00F0B18006D84F2A8F
:1061E00000F09380502A40F0B781A1E0522A00F0DD
:1061F000B880532A40F0B081BDE0832A00F0F580DA
:1062000006D8552A00F0D780572A40F0A581E5E04E
:10621000852A00F0FA80C0F0F080FF2A40F09C81CF
:10622000FCE06B4B40F2FF70D97805E0684B694A9F
:10623000DB7800201946137002F002FB91E1DB7855
:10624000644A194601205370F6E7614B614ADB78D6
:10625000042019461371EFE75D4B5E495A68DB78FD
:106260001C2043EA022341F81C3F0EE0DB78594A28
:10627000194605205371DFE7554B56495A68DB78BC
:106280000C2043EA022341F80C3F042202F05AFAA0
:1062900067E14F4B4F4C5A68DB78214643EA0223B3
:1062A00041F8083F082070E0DB784A49262001F8D1
:1062B000263F7EE0464A474BD27812B1464901223A
:1062C0004A60DA75434B1720D97DB5E7404B414C06
:1062D000DB7803201946E37002F0B2FAE07802F0AE
:1062E00087FCE07802F084FCE07802F0A9FC38E159
:1062F000374B384ADB780220194693709CE7DB78ED
:10630000344A19461520537596E7314B314CDB78EA
:1063100019201946637602F093FA607E10F00100AE
:1063200002D00020012100E0014605F081FF18E1C4
:10633000274B284ADB781620194693757CE7254AB7
:10634000127D12F0010F05D0DB7813F0010F01D19F
:1063500002F03AFB1E4B1F4ADB78142019461375D6
:106360006AE71B4B1B495A68DB78202043EA02236B
:1063700041F8203F89E7164B164C5A68DB782146D6
:1063800043EA022341F8103F1020042202F0DAF918
:1063900022696079A16802F0EFFFE2E05A68DB78D9
:1063A00043EA0222012A00F2D9800A491A2001F8A0
:1063B0001A3F01226AE7064B5A68DB7843EA022259
:1063C000012A00F2CB8003491B2001F81B3FF0E7B4
:1063D000E00600200800002058070020614B6249B9
:1063E000DB78272001F8273FE3E75A68DB7843EAA8
:1063F00002225E4BC3F8D420B3E05A4B5A68DB78D4
:1064000043EA02225A4B1A60ABE0564B5A68DB78DB
:1064100043EA0222554BC3F8D820A2E0514BDA7868
:10642000544B9DE05868D9785A78534B41EA002183
:1064300043F8221095E05A78272A59D00ED8022A1C
:1064400033D004D8CAB1012A40F0868021E01B2A4B
:106450003ED01C2A44D0092A7ED132E02B2A5FD0BC
:1064600005D8292A50D0D978444A54D847E02D2A53
:1064700064D05CD32E2A6FD167E05A68DB7843EA98
:1064800002223E4B1A6003F073FA384BC3F8DC006B
:1064900067E05A68DB7843EA0222384B5A6003F01F
:1064A00067FA324BC3F8E0005BE05A68DB7843EAF6
:1064B0000222324B9A6003F05BFA2C4BC3F8E400E3
:1064C0004FE05A68DB7843EA02222C4BDA6048E05E
:1064D0005968DB78002043EA012105F0A3FF40E082
:1064E0005968DB78002043EA012105F06FFF38E0AE
:1064F0005A68DB7843EA0222204B1A6131E05B687C
:1065000041EA032151612CE05A68DB7843EA022218
:106510001A4B9A6125E05B6841EA0321D16120E0D2
:106520005A68DB7843EA0222144B1A6219E05A686F
:10653000DB7843EA0222114B5A6212E05A68DB7898
:1065400043EA02220D4B9A620BE05A68DB7843EA79
:1065500002220A4BDA6204E0032200E00422084B24
:106560001A7010BDE0060020080000207002002014
:10657000540700205107002068070020380C002035
:106580005807002008B5824B9A78022A00F0B9809B
:10659000032A00F0BB80002A40F01E815B78502B5C
:1065A0006ED022D8462B54D00ED8422B47D005D8D7
:1065B000402B3DD0412B40F00D813EE0442B43D099
:1065C000744B754A43D83DE04B2B4DD006D8482B31
:1065D00043D040D3492B40F0FD8042E04D2B49D0C1
:1065E00045D34F2B40F0F68047E0812B5FD010D889
:1065F000542B4ED005D8522B47D0664B664A46D80E
:1066000041E0572B4BD0802B4DD0552B40F0E280F2
:1066100042E0852B5DD004D8832B53D05D4B55D8F9
:106620004DE0FE2B64D066D8F02B40F0D3805FE0C5
:1066300040F2FF7002F06EF89CE0574B59E0564B69
:106640005A78C4E01279C3E0534BDA69BFE052795B
:10665000BEE0514B85E0504B80E04F4B93F8262035
:10666000B5E04D4BDA7D48E04B4BDA78AFE04A4B72
:106670009A78ACE0484B5A7DA9E0474B5A7EA6E099
:10668000454B9A7DA3E0127DA2E0434B95E0126951
:106690009EE0414B9A7E9AE03F4BDA7E97E03E4B7C
:1066A00093F8272093E03D4B93F8D1208FE03B4BAC
:1066B00093F8D120042A14BF0022012287E0374A30
:1066C000926885E0354BD3F8D42080E0344A1268D4
:1066D0007EE0324A334BD2F8D8104B4303F5405397
:1066E00039332C4923F000404860C2F8D83076E0B6
:1066F0002D4B1A786BE02D4B1A78003A18BF012207
:1067000065E05A782A4B53F8222060E05B78272B0B
:1067100033D00DD8022B20D003D8C3B1012B59D1CF
:1067200018E01B2B1FD01C2B21D0092B52D117E0B6
:106730002B2B41D005D8292B24D0164B1D4A24D809
:106740001EE02D2B3ED03AD32E2B43D13DE0194BEA
:106750001A683CE0174B5A6839E0164B9A6836E0E5
:10676000144BDA6833E0002005F0AAFC02E00020B8
:1067700005F092FC074B586031E00E4B1A6926E099
:10678000526925E00B4B9A6921E0D26920E000BFF5
:10679000E0060020580700200800002070020020BA
:1067A000540700206D4EC6416C0C0020510700209C
:1067B00068070020380C0020124B1A6A07E0114BC2
:1067C0005A6A04E00F4B9A6A01E00E4BDA6A0E4BEC
:1067D0005A6004E0032200E004220B4B1A700B4BBA
:1067E0001B786BB1084B0A495A680A4B0A601AB900
:1067F0001A6842F0080202E01A6822F008021A60E1
:1068000008BD00BF380C00205807002052070020A8
:1068100040070020E806002010B5154CA07818BBF2
:106820006378012B16D003D3022B124C19D114E03C
:1068300004F076FFA17839B10F4A937FBBB102EB28
:106840004112927F9A4212D10C4B01221A71013AE5
:106850000B4B0BE004F06CFF09E004F071FF60608B
:1068600005E00323237002E0024B04221A7010BDDE
:10687000E006002058070020100C002070020020C5
:106880008C0B002037B5504B1A7CA2B94F49486891
:10689000CA7842EA0022B2F1FF3F04BF4C4A1268B4
:1068A0000A214A43C3F8E82003F062F8464B01226C
:1068B0001A74C3F8EC00454B5B78042B00F282801D
:1068C000DFE803F003353F4F130003F051F83E4B70
:1068D000D3F8EC10D3F8E820411A0029B8BF494298
:1068E00091426CD900221A746CE0384B364C98787F
:1068F00004F026FF30B9374A2074136823F01003E0
:1069000013605FE0D4F8E830002B57D003F030F884
:10691000D4F8EC20D4F8E830821A002AB8BF5242EA
:106920009A424BD92B4B00211A68217442E0002077
:1069300005F060FA254B244C9D786D0050FA05F562
:106940001CE000207C2101AA05F090FB1F4B0222D5
:106950009D789DF806306D0012FA05F51A4C1D4021
:106960000EE001AA00207C2105F080FB174A9DF86B
:1069700006309578144C6D0053FA05F515F00105B5
:1069800006D0144B00211A68217422F0100213E083
:10699000D4F8E83093B102F0EBFFD4F8EC20D4F84F
:1069A000E830821A002AB8BF52429A4206D9094BEF
:1069B00025741A6842F010021A6003E0024B9A68CC
:1069C000013A9A603EBD00BF70020020E006002040
:1069D00040070020E806002008B5184B9A7812B14D
:1069E000022A26D106E05868DB7843EA0020FDF74A
:1069F0005DFD21E0587807280AD85A68DB7853EA09
:106A0000022202D1FDF7F6FC16E0FDF7FFFC13E0D1
:106A1000FF280CD15868DB7843EA0020B0F1FF3F33
:106A20000ABF074BC0B21878FDF7FCFC04E0032254
:106A300000E00422034B1A7008BD00BFE0060020EE
:106A4000400700205807002010B5254B9A78012AEE
:106A500028D003D3022A234C2DD127E058780828C8
:106A600002D8FDF7FDFD1AE00A2804D11E4B9A68F2
:106A7000C2F340220CE00B2802D1FDF73BFE0EE0F2
:106A80000C2808D1184B9A6882F48052C2F3003265
:106A9000144B5A6011E0FF280FD1FDF7F9FD114B9F
:106AA00058600AE0587802F07FFFF8E75878FDF761
:106AB000CDFC606001E0042323700C4B1B786BB1AC
:106AC000084B0B495A680B4B0A601AB91A6842F016
:106AD000080202E01A6822F008021A6010BD00BF26
:106AE000E006002058070020001001405207002057
:106AF00040070020E806002010B5204B5A78812A74
:106B00003AD19A78922A37D19A79A32A34D15A79EC
:106B1000B42A31D11A79C52A2ED1DB78D62B2BD1C4
:106B2000174B4FF400525A6103F0CAFA02F020FFEB
:106B3000044602F01DFF001B0028B8BF4042B0F51C
:106B40007A7FF6DBFDF7A0FC07F0DEF9002007F006
:106B50000BFF00210B4806F08DFD0A4806F0EAFC09
:106B6000094806F0A5F906F0D5FD4FF0804008F081
:106B70007FFC0020FDF780FF10BD00BFE006002075
:106B80000010014008000240002401402DE9F347B5
:106B90009D4A9E4DD0785168137840EA01204FF00D
:106BA000640C222B85F800C06B70686000F0838550
:106BB00054D80F2B00F03E8324D8072B00F00A8214
:106BC00010D8032B00F0F88006D8012B00F0A68027
:106BD000022B40F0B187C8E0052B00F0F38100F2F2
:106BE000F58101E10B2B00F0E88205D8092B00F0BC
:106BF000DC8200F2DE82D4E20D2B00F0138300F27F
:106C00001583F3E2192B00F0BD8412D8152B00F088
:106C1000C98306D8132B00F01183142B40F08C8706
:106C200074E3172B00F08E84794B00F29E8400F001
:106C300082BC1E2B00F0D08409D81B2B00F0C4842A
:106C4000C0F0B0841C2B40F0778700F0C0BC202B34
:106C500000F0C88400F2C98400F0C1BC812B00F0B0
:106C6000D8852ED8412B00F0BA8515D8252B00F0F9
:106C7000688507D8232B00F02A85242B40F05C87F9
:106C800000F031BD272B00F09385C0F06585402BC7
:106C900040F0528700F0A0BD452B00F0AC8506D82F
:106CA000432B00F0A28500F2A38500F09BBD472B8B
:106CB00000F0A785C0F0A285802B40F03D8700F052
:106CC000A3BD882B00F0478612D8842B00F0EC85FA
:106CD00007D8822B00F0B585832B40F02D8700F07C
:106CE000B5BD862B00F0FA8500F2558600F0F1BDA7
:106CF0008C2B00F09A8606D88A2B00F07D8600F255
:106D00008F8600F076BEF22B00F0E786FF2B00F0B6
:106D100005878D2B40F0108700F08ABE9378FBB971
:106D20003B4B4FF0010C83F804C03A4B00241C701D
:106D3000394B21461C702046022205F01FF92046DF
:106D4000062140F2FF7205F085FA2F4B20465A6863
:106D5000DB78082143EA022205F07CFA00F0EFBE5E
:106D60002A4B04221A7000F0EABE274DAC78F4B921
:106D7000274B4FF0010C83F804C0264B21461C70B2
:106D8000254B20461C70022205F0F8F8204606210B
:106D900040F2FF7205F05EFA6A68EB78204643EA3B
:106DA00002225242082105F055FA00F0C8BE174BE6
:106DB00004221A7000F0C3BE94788CB9154B20469B
:106DC0001C70154B1C7004F0B3FC204621460222B7
:106DD00005F0D4F82046082105F050FA00F0AFBEC7
:106DE00004232B7000F0ABBE074B9A78002A40F0CA
:106DF000E4805B78032B00F2DB80DFE813F00F0008
:106E000049009400BA0000BFE006002058070020A7
:106E100070020020040C00208C0B0020A64D0020E6
:106E2000FEF7E4F8A54EAB7800246868EA78F454DD
:106E3000A34E590142EA0022F45401F0E001204639
:106E400005F074F9A9782246204605F097F8A9784C
:106E50009C4A02EB41139B7F002B00F070860029B7
:106E600000F06D86927F9A4240F069862046FEF7D8
:106E7000BDF86A68EB78204643EA0222214605F015
:106E800055F920462146224605F078F800F057BE15
:106E9000894D0020FEF7AAF8AB78884A00245901F2
:106EA000D454874A41F00201D45401F0E201204653
:106EB00005F08AF8EB786E68A97843EA0626861909
:106EC000490101F0E0013246204605F02FF9204645
:106ED000A978224605F052F8A8787A4A7A4902EB56
:106EE00040139B7F4E60002B00F02986002800F0A5
:106EF0002686927F9A4240F02286FEF777F802219A
:106F0000204605F061F86A68EB78214643EA0222E0
:106F10008218204605F00AF920462146224605F04F
:106F20002DF800F00CBE644CE378626843EA02235B
:106F3000142B19DC654A002052F82360FEF756F83E
:106F4000A37832465D4E0025F5545D4E5901284622
:106F500001F0E001F55405F0E9F82846A1782A4649
:106F600005F00CF800F0EBBD574B04221A7000F04E
:106F7000E6BD514C0020E3786268002543EA022216
:106F8000524B53F82260FEF731F8A37832464B4E4D
:106F90005901F5544A4E284601F0E001F55405F038
:106FA000C5F82846A1782A4604F0E8FF00F0C7BDDE
:106FB000454B03221A7000F0C2BD434B04221A70E5
:106FC00000F0BDBDFEF734F800F0B9BDFEF77AFB66
:106FD00000F0B5BD907818B104232B7000F0AFBD60
:106FE00053789A2B21D8992B80F08480822B6FD0F4
:106FF0000BD8062B4BD003D8042B3CD0052B0AE032
:10700000072B4BD00C3B012B0CE08C2B65D005D80B
:10701000832B30D0862B40F0BF8032E08D2B63D0A5
:10702000933B022B00F2B8803FE0C82B00F0838036
:107030000FD8C12B6AD005D8B52B60D0C02B40F03B
:10704000AB802BE0C32B6FD067D3C72B40F0A4805D
:107050001DE0D42B00F0848005D8CC2B72D0D22B2D
:1070600040F09A8075E0D62B00F088807FD3FE2B0D
:1070700040F0928089E00020062105F035F800F00C
:107080005EBD00200C2105F02FF800F058BD0D4B1F
:107090004920597A01F0D4FB00F051BD094B4A2038
:1070A000997A01F0CDFB00F04ABD0020142105F0D3
:1070B0001BF800F044BD00BFE00600208C0B002050
:1070C000040C0020100C002058070020EC060020C3
:1070D000042105F009F800F032BD4B20A14901223E
:1070E00001F030FB00F02BBD00201A2104F0FCFF62
:1070F00000F025BD182104F0F7FF00F020BD582056
:107100009949042201F01EFB00F019BD974B48205D
:10711000197A01F095FB00F012BD4020934904223A
:1071200001F010FB00F00BBD44209149042201F056
:1071300009FB00F004BD5F208E49012201F002FB33
:1071400000F0FDBC4E208C49022201F0FBFA00F059
:10715000F6BC50208949042201F0F4FA00F0EFBC9B
:1071600054208749042201F0EDFA00F0E8BC5E20CB
:107170008449012201F0E6FA00F0E1BC5C2082497A
:10718000022201F0DFFA00F0DABC4C207F49012234
:1071900001F0D8FA00F0D3BC7D4B03221A7000F046
:1071A000CEBCFEF7C7FD00F0CABCFEF7DBFF00F067
:1071B000C6BCFFF7E7F900F0C2BC9378022B11D1EF
:1071C0005378372B0AD8734903F5A77001EB830175
:1071D0008000042201F0B6FA00F0B1BC03232B704A
:1071E00000F0ADBC04232B7000F0A9BC6A4B9A7868
:1071F000022A12D15B78372B0AD8664903F5A770AB
:1072000001EB83018000023201F060FA00F097BCCC
:107210005F4B03221A7000F092BC5D4B04221A707F
:1072200000F08DBCFFF7F8FA00F089BCFFF7D4FB43
:1072300000F085BCFFF708FC00F081BC5278574B8A
:10724000092A53D8DFE802F0050D151D2631394112
:10725000494C514A19685068D27842EA00225218C3
:1072600043E04D4A19685068D27842EA00228A1AEF
:107270003BE0494A19685068D27842EA00224A4302
:1072800033E0454A19685068D27842EA002291FBFF
:10729000F2F22AE0404819684468C27842EA0422BF
:1072A00091FBF2F002FB10121FE03B4A1968506894
:1072B000D27842EA00220A4017E0374A196850683B
:1072C000D27842EA00220A430FE0334A1968506834
:1072D000D27842EA00224A4007E01A68D24304E02A
:1072E0002D4A5168D27842EA01221A602B4A2C4B6F
:1072F00012682AB91A6842F008021A6000F01FBC2E
:107300001A6822F008021A6000F019BC224B234AC6
:107310005968DB78126843EA01239A4206DD204B64
:107320001A6842F0040222F003020CE01C4B05D163
:107330001A6822F0060242F0010204E01A6822F004
:10734000070242F002021A60144A154B126822B971
:107350001A6842F008021A60F1E31A6822F0080283
:107360001A60ECE31B0C0020280C0020100C0020FD
:10737000140C00202F0C00201E0C0020200C0020DC
:10738000240C00202E0C00202C0C00201C0C0020B3
:107390005807002068070020E00600204007002072
:1073A000E806002053780C2B00F2C983DFE813F0C5
:1073B0000D001B00290037004500530061006F00DD
:1073C0007D008B009900A700B500944B1B6813F05B
:1073D000080F00F0B483924B5A68DB7843EA02222C
:1073E000904B9A60ABE38D4B1B6813F0080F40F095
:1073F000A6838B4B5A68DB7843EA0222894B9A605A
:107400009DE3864B1B6813F0010F00F09883844BBB
:107410005A68DB7843EA0222824B9A608FE37F4B03
:107420001B6813F0010F40F08A837D4B5A68DB78AC
:1074300043EA02227B4B9A6081E3784B1B6813F08E
:10744000040F00F07C83764B5A68DB7843EA022213
:10745000744B9A6073E3714B1B6813F0050F00F0D7
:107460006E836F4B5A68DB7843EA02226D4B9A6059
:1074700065E36A4B1B6813F0020F00F06083684BF2
:107480005A68DB7843EA0222664B9A6057E3634B03
:107490001B6813F0030F00F05283614B5A68DB78CE
:1074A00043EA02225F4B9A6049E35C4B1B6813F08E
:1074B000100F00F044835A4B5A68DB7843EA0222EB
:1074C000584B9A603BE3554B1B6813F0200F00F0BC
:1074D0003683534B5A68DB7843EA0222514B9A6059
:1074E0002DE34E4B1B6813F0400F00F028834C4BEC
:1074F0005A68DB7843EA02224A4B9A601FE3474B03
:107500001B6813F0800F00F01A83454B5A68DB7834
:1075100043EA0222434B9A6011E3404B1B6813F489
:10752000807F00F00C833E4B5A68DB7843EA0222EE
:107530003C4B9A6003E33A4A5168D27842EA01220E
:107540009A60FCE2374BDA68072A00F2F882344985
:107550009C684868C97841EA0020511C03EB82020C
:10756000C2F8F0409860D960E9E2DA682D4B002A51
:1075700000F0E582013A03EB8201D1F8F010DA6005
:107580009960DCE253782E2B03D8274A0121D1548D
:10759000D5E2FF2B03D1234B01225A74CFE2032300
:1075A0002B70CCE21E4B5B782E2B03D81E4A002199
:1075B000D154C4E2FF2B03D11A4B00225A74BEE20D
:1075C0001A4B03221A70BAE2FFF75CF9B7E2154BC7
:1075D000002283F8D120B2E2FEF722FBAFE2FEF7F1
:1075E000A5FCACE2FEF75EFBA9E20D4A104B527817
:1075F0000A2A52D8DFE802F0060B20252B33393F48
:1076000045494C000B491A6809688A1803E0094A81
:10761000196812688A1A1A603FE000BFE806002065
:10762000E006002070020020880C0020580700208F
:107630004007002060070020934A196812684A43F7
:10764000E9E7914A1968126891FBF2F2E3E78E4A82
:107650001968126891FBF2F002FB1012DBE78A490D
:107660001A68096801EA0202D5E787491A680968B9
:1076700041EA0202CFE784491A68096881EA0202F6
:10768000C9E7814B1A68D243C5E71A687E4BC2E747
:107690007D4A18681168106019607C4A7C4B12683A
:1076A00022B91A6842F008021A6048E21A6822F009
:1076B00008021A6043E2754B01F07F4118681B789D
:1076C00041EA10215160D370FDF7B2FC37E26F4BF5
:1076D00001F07F4118681B7841EA10215160D37096
:1076E000FEF740FD2BE26B4B5B78052B00F2278207
:1076F000DFE803F003090F151B21654B1A6802F040
:107700000F021A601BE2624B1A6822F010021A6024
:1077100015E25F4B1A6822F020021A600FE25C4B00
:107720001A6822F040021A6009E2594B1A6822F0E6
:1077300080021A6003E2564B1A6822F480721A60C3
:10774000FDE153782E2B04D8534A02EB8303586192
:10775000F5E103232B70F2E14F4BDFF830C1D3F892
:1077600010914E4993F82C21D3F814A1CCF8009035
:10777000DFF814C1D3F81871D3F81C81D3F8206155
:10778000D3F82451D3F82841CCF800A0885CDFF866
:1077900000C19F60CCF800801E74C3F8EC50C3F8A1
:1077A000E84008B101238B543B4B00229A74C6E198
:1077B00093786BB9374B5B78142B05D8334A116833
:1077C000374A42F82310BAE1364B03221A70B6E169
:1077D000344B04221A70B2E102F0D0FCAFE102F0A7
:1077E000CFFCACE102F0CEFCA9E102F0CDFCA6E1B9
:1077F00002F0CCFCA3E102F0CBFCA0E102F0CAFC59
:107800009DE102F0C9FC9AE1234B002283F8D120CC
:1078100095E1537813B1012B10D104E01E4B0122E6
:1078200083F8D1208BE1B0F5006F04D21A4A906042
:1078300082F8D13083E104232B7080E103232B7085
:107840007DE1154B022283F8D12078E1124B002113
:1078500099745974104A4FF0FF3402F1140040F843
:1078600021400E480023435401312F29F2D1084909
:1078700013740B60054982F8D1300B6002499360A4
:107880000B60D3605BE100BF600700204007002071
:10789000E8060020E006002070020020880C00208E
:1078A000EC060020580700208D4B1B7D13F0020FC3
:1078B0000CD1B0F5006F06D28A4B0422C3F8300118
:1078C00083F8D1203BE104232B7038E108232B708F
:1078D00035E1844B002283F8D12030E1804B012137
:1078E0009A78814BB0F5006F1970804B1A7028D2CE
:1078F0007B4B1C7D0C4024D1694601F0A9F87B4BE1
:107900009DF800709DF801609DF802509DF806C03A
:107910009DF805009DF804109DF803201C725F700F
:107920009E70DD7083F804C058719971DA7101237B
:107930006E4A985C117A01334118082B1172F7D105
:10794000FDE00123694A002199540133082BF9D144
:1079500013781372F3E053788BB9614A0120917860
:10796000634A1468604A1070604A11700133E2186B
:1079700012F8011C5D4A082B9954F7D1DFE0012B66
:1079800040F0DD8018222A710422EA716FF077023C
:10799000AA716B71D3E0574B5B78032B00F2CF8059
:1079A000DFE803F002101D224E4A534BD2F830118B
:1079B00092F8D1C0107C0A0A197183F807C0987137
:1079C0005A71BCE0474A4C4B916892F8D1C0107C88
:1079D0000A0A197183F807C098715A71AFE0474BD2
:1079E0001A68454B5A60AAE0454B1A68424B5A60E8
:1079F000A5E0FEF79DFBA2E05278424B02B10122C6
:107A00001A703C4B404AD878364B107093F83411BA
:107A10003E4A002311703E4A13703E4A13708EE0B6
:107A2000304B012283F8352189E0FEF7CBFA86E05E
:107A3000304B5B78032B4CD8DFE803F00C023C475B
:107A40002C4B28495A68DB78D1F8381143EA022CCC
:107A500000232BE0234BD3F83821092A0CD82549E1
:107A6000501C4C68C97803EB820241EA0421C2F839
:107A70003C11C3F8380162E01F4B09221A705EE026
:107A800052F82340581C64450FD102EB80020139A3
:107A900004E052F8040C013342F8080C04328B4223
:107AA000F7D3104BC3F8381149E003468B421A4A0A
:107AB000E6D344E00B4A0023C2F83831164A0021CD
:107AC000D1500433282BF9D139E00B4B0A225A60EC
:107AD00035E0094B03221A7031E0FFF70DF82EE074
:107AE0000800002070020020440700204807002002
:107AF00000000020E006002058070020400700207A
:107B000060070020780B0020A40B0020760C0020DA
:107B1000BC0C0020940B0020AC030020094B5A68D9
:107B2000DB7843EA022240F2D2439A4207D1064B65
:107B3000012283F8642102E0044B02221A70BDE89E
:107B4000FC8700BFE00600207002002058070020DC
:107B500073B5204B024640781F4D18709078002670
:107B60005870D078EC46987010790C46987150791E
:107B7000587192F806E095E8030083F804E0D279A2
:107B80008CE80300DA70154B1E70FEF7FFFF144BF4
:107B90001B7873B9637023702B78A3706B78E370D4
:107BA000EB792371AB7963716B79A3712B79E371F5
:107BB00008E0012B06D10B4B9B195B78A3550136CE
:107BC000082EF8D1044B6A4692E8030083E80300CC
:107BD0007CBD00BFE00600205807002052070020AF
:107BE0004407002048070020F7B5114D114C6F687D
:107BF0004FF0000C07F07F4747EA13276F600E4FE6
:107C00006E4687F800C028706970AA7094E8030077
:107C1000EB7086E80300FEF7B9FF96E8030063689F
:107C2000227884E80300054918460A70FEBD00BFAB
:107C3000E0060020580700205207002070020020B4
:107C40002DE9F04F834B9BB01B781BB9824B93F807
:107C500065316BB1814B1B78062B09D00A2B07D0FD
:107C60000F2B05D01F2B03D07B4B002283F8342130
:107C7000794A92F83431591EC9B2012946D892F88E
:107C800066017749774ACC681278012B0CBF4FF018
:107C9000070C4FF0080C00230E948DF834C08DF8BB
:107CA00035008DF83630CAB96F4B8E681D7819795A
:107CB0005C7893F807C098795B798DF83C608DF813
:107CC0003D508DF83E408DF83FC08DF840008DF856
:107CD00041308DF842108DF843200AE0012A08D186
:107CE000624A0133995C1AA8C218082B02F82D1CAD
:107CF000F6D15F4B1B78002B40F024810DA801F0DA
:107D000059FA002840F01E8100F0DDBC032B25D17C
:107D100092F8D040002C40F0E880524B1B7893B989
:107D20004F4D514CA8786E78227863788619B61832
:107D3000E279F618A379B6186279F6182379B6189D
:107D4000F618F6B219E0012B40F0FC80474BE05CDE
:107D5000013400F0B9FF092CF8D1F3E0042B27D14E
:107D60003F4D414CAB786E7818469E190136002382
:107D7000012222706360F6B2637000F0A5FF68789C
:107D800000F0A2FF207800F09FFF607800F09CFFD9
:107D9000E07900F099FFA07900F096FF607900F09B
:107DA00093FF207900F090FF304600F08DFFC9E08E
:107DB000052B25D192F8D040002C40F09680294B1D
:107DC0001B7893B9264D284CA8786E782278637872
:107DD0008619B618E279F618A379B6186279F618FA
:107DE0002379B618F618F6B219E0012B40F0AA80F4
:107DF0001E4BE05C013400F04BFF092CF8D1A1E0F0
:107E0000062B37D1164D184CAB786E7818469E1954
:107E100001360023012222706360F6B2637000F025
:107E200037FF687800F034FF207800F031FF607889
:107E300000F02EFFE07900F02BFFA07900F028FF82
:107E4000607900F025FF207900F022FF304600F035
:107E50001FFF77E05107002070020020E00600209D
:107E60000800002044070020580700204807002091
:107E7000700B0020072B3CD192F8D030002B34D16E
:107E8000A74A127822BBA74AA74B557896781C7848
:107E900093F801C0AF19D879E719997967445A79ED
:107EA000C7191B79CF19D719DF198DF858708DF8BC
:107EB00050608DF851508DF852408DF853C08DF8B8
:107EC00054008DF855108DF856208DF8573008E085
:107ED000012A06D1954A995C14AAD1540133092B81
:107EE000F8D1934B1B786BB328E08F4804F000FC6B
:107EF00028E0082B26D18B4B0022597898788C4BA0
:107F000045181C78884B4FF0010C01355A608DF8EC
:107F100052C08DF8532016468DF854208DF8552008
:107F20008DF856208DF857208DF858505A7083F8E8
:107F300000C08DF850008DF851101CB114A8092113
:107F400001F08CFF7B4B1B78002B00F081807A4A7C
:107F5000774B1278794C013A062A74D8DFE802F0A0
:107F600004042A7373734E006E4A94F800C0D068FC
:107F7000926819788DF82C206FF07F028DF82D20F3
:107F80000A3200238DF82E207D328DF832C08DF814
:107F900024208DF826300A908DF82F308DF830305F
:107FA0008DF831308DF8253000294CD109A801F029
:107FB00001F948E05B4D2278AB786E7818469E193F
:107FC0000A36B61800F080FE687800F07DFE80204A
:107FD00000F07AFE8A2000F077FE002000F074FEA8
:107FE000002000F071FE002000F06EFEF6B2207856
:107FF00000F06AFE304600F067FE24E0494822782F
:10800000417880786FF07F0500EB010C1C780CF153
:108010000A0C002394448DF846500A358DF84750D9
:108020008DF84A308DF84CC08DF844008DF845101D
:108030008DF848308DF849308DF84B201CB111A8CF
:10804000092101F00BFF3B4A002313703B4A1370D8
:108050003B4B334893F864110022027083F865218A
:1080600083F8342111B10120FCF706FD344B93F85D
:10807000352152B193F8D0200021D2F1010238BF4E
:10808000002283F8351183F8D020294B1B78002B70
:108090005ED10DA801F06CF8002859D09DF834305D
:1080A000062B55D9274B1F4A9DF83C709DF83D6023
:1080B0009DF83E509DF83F409DF840E09DF841C03E
:1080C0009DF84280116983F803801F705E709D7077
:1080D0009C7183F805E083F804C00E9B184A9DF854
:1080E00035008B4282F8660102D1012382F86531A6
:1080F00001F03EFC9DF834304FF00002072B124B8C
:108100000F4C1860114B1A7001D1012300E00223BB
:1081100084F834310A4B93F8D1305A1ED2B25FE161
:1081200044070020080000205807002048070020CE
:10813000700B0020BC0C0020760C0020940B00205B
:1081400070020020E0060020680C0020710B002067
:10815000A84C94F8D050002D72D10DF1670000F0BA
:1081600031FD00286CD000F049FD08B184F867515A
:10817000A04B9DF8670093F867114A1CD2B2C9184A
:10818000092A81F8680183F8672140F05F819A49E4
:1081900093F8682148784FF0000C904283F867C14B
:1081A00007D091F82730002B00F050819A4240F020
:1081B0004D81914B93F82730934203D18D4B01228F
:1081C00083F8652100231A468A4C04F5B471C95C12
:1081D00001335218082BD2B2F6D194F87031934281
:1081E0002CD1864B94F86D1194F86E2194F86F5150
:1081F00094F8696194F86AE194F86BC194F86C01A1
:10820000DD7059711A711E7083F801E083F802C0A5
:10821000987101F0ADFB7A4D94F8D1302860591E69
:1082200078480022C9B202700320012984F8340181
:1082300084F8672140F2D880052B8AE00423D5E03A
:108240006C4C94F8D03083B16C4804F097FA60B16C
:1082500001F08EFB6A4994F8D130086069495A1ED2
:1082600000200870D2B20321B8E0624C94F8D050DC
:10827000002D73D10DF1670000F0CAFC00286DD00D
:1082800000F0E4FC08B184F867515A4B9DF8670090
:1082900093F867114A1CD2B2C918092A81F86801FB
:1082A00083F8672140F0D280534993F868214878D9
:1082B0004FF0000C904283F867C107D091F8273047
:1082C000002B00F0C3809A4240F0C0804A4B93F8E4
:1082D0002730934203D1474B012283F865210023C5
:1082E0001A46444C04F5B471C95C01335218082B8A
:1082F000D2B2F6D194F8703193422DD13F4B94F81D
:108300006D1194F86E2194F86F5194F8696194F8A6
:108310006AE194F86BC194F86C01DD7059711A71BF
:108320001E7083F801E083F802C0987101F020FB11
:10833000334D94F8D1302860591E32480022C9B21A
:1083400002700520012984F8340184F867214BD993
:10835000834249D0013272E0062347E0254B93F86F
:10836000D040002C52D1284B1B78002B4ED017A8A0
:1083700001F05EFD002849D02346224617A9C95CBA
:1083800001335218082BD2B2F8D19DF86410194C61
:1083900091422BD1194B9DF861109DF862209DF8F8
:1083A0005D609DF85EE09DF85FC09DF860009DF8FF
:1083B000635059711A711E70DD7083F801E083F803
:1083C00002C0987101F0D4FA0D4994F8D1300860D8
:1083D0000C495A1E00200870D2B2072184F83411CB
:1083E000012A01D9052B29D1002228E084F8343153
:1083F0002CE000BF7002002008000020E0060020F2
:10840000700C0020750C0020700B0020A14C94F81B
:10841000D130013BDBB2012B18D8A368B3F5006F54
:1084200010D2FCF7EFF868B1A3689B4918460133F6
:10843000A36000F00DFB092384F834310122974B2F
:108440001A7003E0934B002283F8D120914C94F8EA
:10845000D130042B05D1904E327812F0800F00F00D
:10846000EF808C4B93F834313BB1042B05D0082BB3
:1084700003D0062B01D0FEF789FB864C94F83431EB
:10848000092B40F0B28001F073FAD4F8DC30844A52
:10849000C31A002B1268B8BF5B4293420AD9814BC2
:1084A0001A78012A01D101321A7001F061FA794B70
:1084B000C3F8DC0001F05CFA764BD3F8E020784B8F
:1084C000821A002A5B68B8BF52429A420AD9754B99
:1084D0005A78012A01D101325A7001F049FA6D4BE4
:1084E000C3F8E00001F044FA6A4BD3F8E4206C4B87
:1084F000821A002A9B68B8BF52429A420AD9694B35
:108500009A78012A01D101329A7001F031FA614B57
:10851000C3F8E4005F4A537C002B66D0937C002BA9
:1085200063D19C46604BD2F8EC001B68D2F8E8108F
:1085300007935E4B04901B68D2F8108106935C4B46
:10854000D2F814711B68D2F81841059392F82C31B7
:10855000D2F81C610293107C9368D2F82051D2F8B3
:1085600024B1D2F82821039101926246DFF83491B8
:10857000194619F802A0BAF1020F18D14D4951F865
:108580002210B1F1FF3F0ED00546D0B20290039801
:10859000DDF810B00190059E069FDDF81C804FF0BD
:1085A000010C002004E0002109F8021019462346BE
:1085B00001322F2A02D01C460B46D7E7354A91607C
:1085C000C2F818310199029B82F812C0C2F81081DA
:1085D000C2F81471C2F81C611074C2F82051C2F8BC
:1085E00024B1C2F8281182F82C312A4B93F8342197
:1085F000092A06D193F8D120022A02D1033283F846
:10860000D120244BD3F8381100295CD093F83421C1
:10861000092A58D193F8D120012A54D1986800230F
:1086200008E054F823400133A04203D1052382F827
:10863000D13048E0174A8B4202F59E74F1D342E0F4
:1086400094F83431002B3ED0042B3CD0082B3AD088
:10865000062B38D0F3787168D4F83001164D43EA10
:108660000123B0F5006F6A706B6027D2314600F0CD
:108670001FF93146D4F8300100F042F930B1D4F896
:1086800030310133C4F83031652300E007232B700B
:1086900019E000BF70020020E00600205207002011
:1086A000380C0020880C00204007002060070020C4
:1086B000E8060020840200205807002007232B70C2
:1086C000002384F8D1301BB0BDE8F08F70B50446AC
:1086D00000200E46154603210246FCF70BFB002046
:1086E000C4F307210246FCF705FB0020E1B2024675
:1086F000FCF700FB002407E0944214BF0022012293
:10870000FCF7F8FA3055013400206A1EAC420146ED
:10871000F2D370BD10B50446002003210246FCF7D9
:10872000E9FA0020C4F307210246FCF7E3FA00202F
:10873000E1B20246FCF7DEFA002001460122FCF716
:10874000D9FA10BD2DE9F04104460F461646002027
:1087500006210122FCF7CEFA002005210246FCF793
:10876000C9FA002001220146FCF7C4FA10F0020FFA
:10877000F2D0002002210246FCF7BCFA0020C4F32C
:1087800007210246FCF7B6FA0020E1B20246FCF7E8
:10879000B1FA002543E0013414F03F08795D01D1BE
:1087A000012204E0721E954214BF00220122002023
:1087B000FCF7A0FAB8F1000F30D1731E9D422DD204
:1087C000002005210246FCF795FA0020012201460F
:1087D000FCF790FA10F00100F2D106210122FCF71B
:1087E00089FA002005210246FCF784FA00200122C4
:1087F0000146FCF77FFA10F0020FF2D000200221B0
:108800000246FCF777FA0020C4F307210246FCF782
:1088100071FA0020E1B20246FCF76CFA0135B5426C
:10882000B9D3002005210246FCF764FA002001229A
:108830000146FCF75FFA10F0010FF2D1BDE8F081BC
:1088400038B5012204460D4600200621FCF752FAF5
:10885000002005210246FCF74DFA002001220146C6
:10886000FCF748FA10F0020FF2D000200221024675
:10887000FCF740FA0020C4F307210246FCF73AFA5D
:108880000020E1B20246FCF735FA29460020012219
:10889000FCF730FA002005210246FCF72BFA0020F5
:1088A00001220146FCF726FA10F0010FF2D138BD83
:1088B00038B50725454305F500650C462846097877
:1088C0000135FFF7BDFF284661780135FFF7B8FF96
:1088D0002846A1780135FFF7B3FF2846E178013536
:1088E000FFF7AEFF284621790135FFF7A9FF28469B
:1088F0006179FFF7A5FF681CA179FFF7A1FF38BDDB
:108900002DE9F3470725454300200C460246032185
:10891000FCF7F0F905F500650020C5F307210246D4
:10892000FCF7E8F90020E9B20246FCF7E3F9002081
:1089300001460246FCF7DEF9824600200146024667
:10894000FCF7D8F98046002001460246FCF7D2F930
:108950000746002001460246FCF7CCF9814600207C
:1089600001460246FCF7C6F90646002001460246CB
:10897000FCF7C0F90546002001220146FCF7BAF9D0
:10898000237853451DD1637843451AD1A378BB4260
:1089900017D1E37821798DF804608DF805508DF8B2
:1089A0000600627943EA012343EA0243A079019A6F
:1089B00043EA006049EA0229814514BF00200120F2
:1089C00000E00020BDE8FC8738B54FF400640020CB
:1089D00006210122FCF78EF9002005210246FCF752
:1089E00089F9002001220146FCF784F910F0020FFA
:1089F000F2D0002002210246FCF77CF90020C4F3EB
:108A000007210246FCF776F90020E1B20246FCF7A6
:108A100071F9002500203F2D14BF002201220146DC
:108A20000135FCF767F9402DF4D1002005210246FD
:108A3000FCF760F9002001220146FCF75BF910F019
:108A4000010FF2D14034B4F5804FC0D138BD00BF22
:108A500038B50725454300200C4602460321FCF7A4
:108A600049F905F500650020C5F307210246FCF72A
:108A700041F90020E9B20246FCF73CF9002001462A
:108A80000246FCF737F92070002001460246FCF749
:108A900031F96070002001460246FCF72BF9A07006
:108AA000002001460246FCF725F9E070002001464F
:108AB0000246FCF71FF92071002001460246FCF730
:108AC00019F96071002001460122FCF713F9A07129
:108AD00038BD00BF37B5002005210246FCF70AF972
:108AE000002001220146FCF705F910F07104F2D1D3
:108AF00000F03EFF054605E0FFF70CFE422814BFDC
:108B00000024012400F034FF431B002BB8BF5B425C
:108B1000B3F5FA6F40F2FF7002DA002CECD000E0FF
:108B20001CB1234B1B78002B36D040F2FF70002184
:108B3000FFF786FEFFF748FF00201E494022FFF79F
:108B400001FE4FF480701C49B422FFF7FBFD40206A
:108B50001A492022FFF7F6FD002301934FF4C36466
:108B600001AD2046042204342946FFF7EBFDB4F59D
:108B7000FF6FF5D100230193A4F530742046042241
:108B800004342946FFF7DEFDB4F5C36FF6D140F299
:108B9000FF704221FFF754FE002040220549FFF7F5
:108BA00095FD402006492022FFF790FD3EBD00BF05
:108BB000AC0B002008000020F02B0108202C01083D
:108BC000100C0020094B19685A68914201D100200D
:108BD0000BE01A68D118097A013201701A601A681C
:108BE000202A01D100221A6001207047E4030020EE
:108BF000014B9862704700BFE4030020034B1A78D2
:108C0000104612B100221A7001207047D00C0020CB
:108C10000A4BD96A1A6B914201D100200CE0DA6A42
:108C2000D11891F8341001320170DA62DA6A202A20
:108C300001D10022DA620120704700BFE403002066
:108C4000014B5865704700BFE4030020034B1A78BE
:108C5000104612B100221A7001207047D10C00207A
:108C600008B5FBF711FC034B0022DA621A63FBF72D
:108C700009FC08BDE403002008B5FBF705FC034B25
:108C800000221A605A60FBF7FDFB08BDE4030020D8
:108C900038B50B4B84469C6DDA6D0134202C08BF2F
:108CA000002494420AD09D6D0648ED1885F860C0F6
:108CB00040F2277101229C6506F072FC38BD00BFAE
:108CC000E40300200044004038B50D4B8446D3F83F
:108CD0008040D3F884200134202C08BF0024944223
:108CE0000CD0D3F880500748ED1885F888C040F2C2
:108CF00027710122C3F8804006F052FC38BD00BF46
:108D0000E40300200048004038B50546002401E097
:108D1000FFF7DAFF2B5D01341846002BF8D138BD80
:108D20002B4910B50B8813F0200F1DD0294BDB68A1
:108D300013F0020F01D08B8816E0274B1A6BD86A0C
:108D40000132202A08BF0022824206D01C6B88888C
:108D5000E118C0B281F834001A63204B0A221A606D
:108D60001D4B5A6D1E4B1A601948038813F0800F73
:108D70001BD01B4B1A68C2B9174B9C6DD96D8C4226
:108D80000FD0144902240C61D96DCC1894F860C03E
:108D90000131A0F804C0D965D96D202905D1DA6563
:108DA00003E040F2277106F0FBFB0948038813F04B
:108DB000400F0BD040F2266106F0EAFC064BDA6D5C
:108DC0009B6D9A4202D1034B02225A6110BD00BF33
:108DD0000044004000080140E4030020C00C0020D3
:108DE000C80C0020274910B50B8813F0200F15D0B0
:108DF000254B5A6818680132202A08BF0022824297
:108E000005D05C688888E118C0B208725A601F4BB0
:108E10000A221A601C4B9A6A1D4B1A601948038873
:108E200013F0800F1ED01A4B1A68DAB9164BD3F81C
:108E30008040D3F884108C4210D0D3F88410CC1822
:108E400094F888C00131A0F804C0C3F88410D3F8A6
:108E50008410202906D1C3F8842003E040F2277152
:108E600006F09EFB0748038813F0400F08D040F23D
:108E7000266106F08DFC044BD3F88420D3F88030B3
:108E800010BD00BF00480040E4030020CC0C0020CF
:108E9000C40C002030B5054687B0564806F0C8FC23
:108EA0004FF40030012105F011FB0420012105F0F1
:108EB000FFFA0420002105F017FB0820002104F030
:108EC0007FFF06AC4FF0040324F8083D03234A4813
:108ED00021468DF8123015338DF8133004F0E0FE82
:108EE000482345488DF8133021464FF00803ADF86C
:108EF000103004F0D5FE684606F01CFB0B2D25D87B
:108F0000DFE805F02406090C0F1215181B1E20229D
:108F10004FF461531CE04FF4964319E04FF4E143E2
:108F200016E04FF4164313E04FF4614310E04FF4A2
:108F300096330DE04FF4E1330AE04FF4613307E07C
:108F40002E4B05E02E4B03E02E4B01E04FF4165361
:108F50000093009B06A95B0841F8183D2548694627
:108F600006F01EFC26230024012505A88DF81430E8
:108F700007238DF815308DF816408DF8175004F042
:108F8000FFFF1C4840F2FF3106F0DEFB282122469D
:108F9000184806F005FB2A46164840F2277106F0ED
:108FA000FFFA2A46134840F2266106F0F9FA2A46EB
:108FB000104840F2255106F0F3FA22460D4840F2DF
:108FC000244106F0EDFA22460A4840F6460106F032
:108FD000E7FA2246074840F66A1106F0E1FA6021F6
:108FE0002246044806F0DCFA2946024806F0CAFA8E
:108FF00007B030BD004400400008014090D003009D
:1090000020A1070040420F0030B5054687B0524806
:1090100006F00EFC4FF48020012105F057FA4F486E
:10902000002104F0CDFE06AC4FF4806324F8083D27
:1090300003234B4821468DF8123015338DF8133039
:1090400004F02EFE482346488DF8133021464FF495
:109050000063ADF8103004F023FE684606F06AFAAB
:109060000B2D25D8DFE805F02406090C0F12151882
:109070001B1E20224FF461531CE04FF4964319E06D
:109080004FF4E14316E04FF4164313E04FF461430D
:1090900010E04FF496330DE04FF4E1330AE04FF463
:1090A000613307E02F4B05E02F4B03E02F4B01E02E
:1090B0004FF416530093009B06A95B0841F8183D36
:1090C0002548694606F06CFB27230024012505A8E6
:1090D0008DF8143007238DF815308DF816408DF873
:1090E000175004F04DFF1C4840F2FF3106F02CFBF6
:1090F00028212246184806F053FA2A46164840F21C
:10910000277106F04DFA2A46134840F2266106F010
:1091100047FA2A46104840F2255106F041FA224605
:109120000D4840F2244106F03BFA22460A4840F638
:10913000460106F035FA2246074840F66A1106F065
:109140002FFA60212246044806F02AFA29460248EE
:1091500006F018FA07B030BD0048004010001400B7
:10916000000C014090D0030020A1070040420F00F6
:1091700030B50C4B0C4C844622681B689A4201D1D6
:1091800000200EE02368094A5D1C02EB03130FCB9D
:109190008CE80F0025602368082B01D10023236091
:1091A000012030BD600D0020D40C0020E00C002018
:1091B000704700BFF0B5437887B00646426833B1C8
:1091C00004238DF80C3000230292019303E00192F6
:1091D00002938DF80C30B37803B102238DF80D3073
:1091E000327800238DF80E20F21801A8117AC218E7
:1091F0000133082BD172F7D103F094FF042818D162
:109200000D4D0E4B2C681B680134082C08BF002440
:109210009C4201D100200DE096E80F002F68084E17
:1092200006EB071C8CE80F00012001462C6003F0C0
:109230006BFF012007B0F0BDD80C0020DC0C002033
:10924000640D00207FB52B4B2B4A196812689142A0
:1092500004D10120002103F057FF48E01968274A94
:1092600002EB0111487850B11B6802EB03125368FE
:1092700004228DF80C2000220192029307E01B6863
:10928000029002EB031253688DF80C000193194B06
:109290001A681A4B03EB02139B781BB102238DF85B
:1092A0000D3001E08DF80D30124B00221968134B80
:1092B0000901CB5C8DF80E300E4B0DF1180C1868BF
:1092C0000CEB020102EB001C0C4801326044007AF6
:1092D000082A01F8090CEFD11A6801321A601A68DD
:1092E000082A01D100221A6001A803F01BFF07B071
:1092F00000BD00BFDC0C0020D80C0020640D002055
:1093000073B50220002103F0FFFE1020002103F0BE
:10931000FBFE01AC0021012003F0F6FE002507262C
:10932000142320468DF804308DF805608DF8065022
:109330008DF8075004F024FE152320468DF80430E4
:109340008DF805608DF806508DF8075004F018FE72
:10935000204613238DF804308DF805608DF80650F3
:109360008DF8075004F00CFE04F0D8F829464FF0B1
:10937000007005F0ABF87CBD2DE9F04101388AB0F2
:109380000C46154607285BD8DFE800F04C4034282F
:109390001C5A10040C238DF81C3003238DF81D304B
:1093A00000238DF81B304FF0020354E00C238DF89E
:1093B0001C3003238DF81D3000238DF81B304FF037
:1093C00004023AE00C238DF81C3003238DF81D3085
:1093D00000238DF81B304FF010022EE00C238DF887
:1093E0001C3003238DF81D3000238DF81B304FF007
:1093F000140330E00C238DF81C3003238DF81D304E
:1094000000238DF81B304FF0280216E00C238DF856
:109410001C3003238DF81D3000238DF81B304FF0D6
:10942000640318E00C238DF81C3003238DF81D30E5
:1094300000238DF81B304FF0C802ADF81E200CE061
:109440000C238DF81C3003238DF81D3000238DF87C
:109450001B304FF00803ADF81E3004F05FF8012117
:109460004FF0007005F032F80120014605F020F8B9
:109470000820012105F01CF80820002105F034F82F
:1094800001214FF4EA1004F09BFC0AAE4FF4007285
:1094900026F8042D032331468A488DF826301533EB
:1094A0008DF8273004F0FCFB0423314685488DF805
:1094B00027304FF4807300260127ADF8243004F0E4
:1094C000EFFB05A88DF81A608DF814608DF8157003
:1094D0008DF816608DF817608DF818708DF819707A
:1094E00003F010FDB4F5006F01A815DA4FF0FF325C
:1094F0006301ADF80830ADF810608DF812708DF88A
:1095000004608DF805608DF80670ADF80A60ADF85E
:109510000C20ADF80E2013E04FF0FF338DF80670ED
:10952000ADF810608DF812608DF804608DF805605C
:10953000ADF80860ADF80A60ADF80C30ADF80E304B
:1095400003F052FDDDB1B5F5006F18DA00220123FA
:109550006901ADF80A208DF805204FF0FF3201A80F
:10956000ADF808108DF812308DF804308DF8063003
:10957000ADF80C20ADF80E20ADF8103016E0002349
:109580000122ADF80A308DF812308DF80530ADF8B3
:1095900008304FF0FF3301A8ADF810208DF80420FB
:1095A0008DF80620ADF80C30ADF80E3003F01CFD40
:1095B000E30043F004030DF1040800270126022212
:1095C0006413ADF80A3040464FF0FF338DF80420A5
:1095D000ADF808408DF805708DF80660ADF80C30D8
:1095E000ADF80E30ADF810708DF8126003F0FCFC91
:1095F000BD421ADDEB0043F004036D130322ADF806
:109600000A304FF0FF3340468DF804208DF8057086
:10961000ADF808508DF812608DF80660ADF80C308A
:10962000ADF80E30ADF8106017E003238DF804306C
:109630004FF004024FF0FF334046ADF80870ADF82C
:1096400010608DF812708DF805708DF80660ADF819
:109650000A20ADF80C30ADF80E3008AF03F0C4FCB2
:10966000012407260025142338468DF820308DF874
:1096700021608DF822508DF8234004F081FC1523E1
:1096800038468DF820308DF821608DF822508DF805
:10969000234004F075FC132338468DF820308DF8F4
:1096A00021608DF822508DF8234004F069FC0220DF
:1096B000214603F029FD2146102003F025FD0AB0C4
:1096C000BDE8F081000C014030B52A4D2A4B2C68D2
:1096D0001B680134082C08BF00249C4287B044D08A
:1096E000012001A903F0FAFD9DF80C20234B042A68
:1096F00009D12A68012103EB021251702A6803EB99
:109700000213029A08E02A68002103EB021251704A
:109710002A6803EB0213019A5A609DF80D30154A2E
:10972000022B164B04D1126803EB0213012203E053
:10973000126803EB021300229A700E4B9DF80E1074
:109740001A680E4B1201D15400230A4A06A9C81800
:1097500011680A4D03EB011110F8090C0133491986
:10976000082B0872F1D1146002E0012003F09AFD89
:1097700007B030BD600D0020D40C0020E00C0020AC
:1097800030B52A4D2A4B2C681B680134082C08BFC1
:1097900000249C4287B044D0002001A903F09EFD24
:1097A0009DF80C20234B042A09D12A68012103EBE0
:1097B000021251702A6803EB0213029A08E02A6829
:1097C000002103EB021251702A6803EB0213019A85
:1097D0005A609DF80D30154A022B164B04D11268C1
:1097E00003EB0213012203E0126803EB02130022D1
:1097F0009A700E4B9DF80E101A680E4B1201D15440
:1098000000230A4A06A9C81811680A4D03EB011182
:1098100010F8090C01334919082B0872F1D11460B2
:1098200002E0002003F03EFD07B030BD600D0020D7
:10983000D40C0020E00C0020F0B5404B1A78AAB1FF
:1098400059683F4A0131596011683E4B013111603E
:109850001A6812B11A68013A1A603B4B1A6812B1C1
:109860001A68013A1A600022344B00E001221A7093
:10987000364B1A683AB11A68013A1A601B6813B974
:10988000334B01221A70334B1A683AB11A68013A05
:109890001A601B6813B9304B01221A702F4B304AE3
:1098A0009B8C30499BB2136010680B68984218DD9E
:1098B000146808682C4B201AB0F5004F2B4806DAC4
:1098C000D3E90045166809680268701A29E0D3E9EF
:1098D00000450E68116806F5803C0268C1EB0C007B
:1098E00011E010680B68984223DA0C6810681E4B70
:1098F000201AB0F5004F1D480ADAD3E900450E687A
:1099000011680268701A5043261A65EBE0770CE084
:10991000D3E900451268096802F5803C0268C1EB92
:109920000C005043261845EBE07730463946C3E932
:1099300000010B4B1A680B4B1A60F0BD8C04002021
:1099400054070020C40C0020C80C0020CC0C0020C0
:10995000D00C0020C00C0020D10C002000040040DE
:10996000B80C0020900B0020B00B0020B80B00209A
:10997000014B5868704700BF8C04002008B50420D4
:1099800004F0C6FF48F6A04004F0D2FF012004F026
:10999000D5FF04480321002204F0C0FB012004F09D
:1099A000E3FF08BD9AC30200F8B5092806D8DFE82E
:1099B00000F0070A0505050505050E1600205CE008
:1099C0003B4B188801E03A4B588880B255E0384B41
:1099D000988840F2F72380B2584300134DE0344B8F
:1099E000D88880B208F04EFB07F030FF0022314BE0
:1099F00007F080FF22A3D3E9002306460F4607F0B5
:109A000079FF21A3D3E9002307F0C2FD1EA3D3E908
:109A1000002304460D463046394607F06BFF00220E
:109A2000254B07F067FF02460B462046294608F003
:109A30008BF808F021FA07F009FF00221F4B08F00D
:109A400083F807F0ABF912A3D3E9002307F052FF24
:109A500011A3D3E9002307F09BFD02460B4610A19A
:109A6000D1E9000108F070F80FA3D3E9002307F053
:109A70008DFD08F001FA08F023FDF8BDAFF300807A
:109A80006666666666660AC06666666666660A40FA
:109A9000C3F5285C8FA272400000000000FEAA40BF
:109AA0009A999999FD6F2F41C3F5285C8F127140E7
:109AB000940400200000303F0000E03F00002440FC
:109AC000F0B593B0002403254FF03303404811A9AB
:109AD000ADF844308DF846508DF8474004F0E0F87A
:109AE0000120014604F0D6FC01214FF4007004F07F
:109AF000DFFC384803F01EFD374B04270193374B3A
:109B00003448029380230693DB18079303F54073D0
:109B10000893A3F578730DEB0701099303F5FF5341
:109B20000A930394049705940B9403F073FD29485A
:109B3000012103F09FFD01264FF4602328480CA962
:109B40000E930C948DF834608DF835600F948DF879
:109B5000407003F00BF822480E2132462B4603F0EA
:109B600087F81F480F2102222B4603F081F81C487A
:109B70000A212A462B4603F07BF82B463A46184822
:109B80000B2103F075F8224615484FF4FC6103F0F1
:109B900031F81348314603F023F81148314603F0F9
:109BA00015F80F4803F030F80D4803F033F800289B
:109BB000FAD10B4803F032F8094803F035F80028D1
:109BC000FAD10748012103F033F813B0F0BD00BF0C
:109BD00000100140080002404C2401409404002081
:109BE00000240140AFF30080014B03221A6070474C
:109BF0009C040020044A054B927A0AB1052200E039
:109C000001221A60704700BFF00D00209C04002064
:109C1000704700BF014B00225A6070479C0400202F
:109C200008B5074B1A6892B242F008021A601A6827
:109C300092B242F004021A60FFF7D6FF08BD00BFDF
:109C4000405C004010B5064C4FF6FB73226802EAF8
:109C500003032360FFF7CEFF4FF40643236010BDDC
:109C6000405C0040072818BF1F4B10B51E4C18BFA2
:109C700018702378052B33D8DFE803F003060A0EAB
:109C80001621FFF7DFFF2BE0FFF7DCFF042328E0BE
:109C900002236370013324E06378013BDBB263701D
:109CA0006378FBB9042218E0104B1A6892B242F0B4
:109CB00010021A6005232370DB18637012E06378CA
:109CC000013BDBB26370637863B9084A4FF6EF7308
:109CD000116801EA030313600622034B1A7001E0C6
:109CE0000623237010BD00BF540E0020405C0040CE
:109CF000034B9B7A13B1034B05221A60704700BFD8
:109D0000F00D00209C040020014B04221A607047D3
:109D10009C040020034B1A7A202A01D100221A72D7
:109D2000704700BF9C040020704700BF212808B581
:109D300008D1124B1B681B7803F07F03212B1AD12B
:109D40000F4B0EE0202816D10C4B0E4A1B681B78D7
:109D500010720D4A03F07F03212B0CBF1346002322
:109D60004BB1064A4FF00001126800205182936106
:109D70009847002000E0022008BD00BF500E0020E0
:109D8000C19D00089C040020DD9D0008074B1B6856
:109D90001B7803F07F03212B05D1022801D0222854
:109DA00001D1002000E00220704700BF500E0020CB
:109DB00019B9012801D8084600E00220704700BF09
:109DC00028B9044B4FF008021B681A8200E00248D1
:109DD000704700BF500E00204800002028B9044BF7
:109DE0004FF008021B681A8200E00248704700BF6B
:109DF000500E0020480000200B4B10B5DA6882B1ED
:109E00001B68052B01D000220BE0002303E007496B
:109E1000595CC15401330449CC68A342F7D30023F1
:109E2000CB60104610BD00BF9C040020580E0020DF
:109E3000084BDB68082B01D800200AE00023064A03
:109E40009A5CC2540133092BF9D1024B0022DA602B
:109E5000012070479C040020580E002010B5074CCC
:109E60000B468AB2C021636006F0BEFA0120A188C9
:109E700006F0C8FC012006F093FB10BD9C040020F6
:109E800007B5142200238DF8042001A801228DF8C3
:109E900006308DF807208DF8053004F071F80EBDFE
:109EA00007B5142200238DF8042001A801228DF8A3
:109EB00006308DF807208DF8053004F061F80EBDEE
:109EC00008B5064B1B68DB78042B01D9002004E0A1
:109ED000034901EBC30105F02FFE08BD500E002021
:109EE0005000002008B5024905F026FE08BD00BF5D
:109EF0007000002008B5024905F01EFE08BD00BF35
:109F000078000020334B10B51B686FF03F0200242F
:109F10005A72DC729C72204606F0BAFA20464FF460
:109F2000007106F0D3FA1021204606F0E5FA402130
:109F3000204606F03BFC8021204606F027FC204608
:109F400006F064FB244B204693F8641006F07CFC7A
:109F5000204606F033FB0120214606F0B7FA012027
:109F6000C02106F013FC0120202106F0C5FA0120D3
:109F7000214606F0D9FA02204FF4C06106F0A6FA95
:109F800002204FF4807106F001FC0220214606F009
:109F9000CBFA0220202106F0AFFA0320214606F07A
:109FA00095FA03204FF4887106F000FC032040214D
:109FB00006F04AFC03204FF4405106F0B5FA214662
:109FC000032006F099FA204605F0C4FD034B012258
:109FD0001A6010BD500E0020480000209C04002094
:109FE00008B5174B174A196889B2118016491288AB
:109FF000098801EA020212F4806F05D04FF6FF32A1
:10A000001A60124BDB6B98470E4B1A880E4B1B885D
:10A0100003EA020212F4007F08D009490C4A4FF605
:10A02000FF500860117C0131C9B21174054A1288D1
:10A03000134013F4004F01D006F012F908BD00BF21
:10A04000445C0040E60D0020980E002048000020EF
:10A050009C04002010B5032006F026FC064C0346A5
:10A0600002464FF488710548E36006F0D5F90320F5
:10A0700006F0A4FA10BD00BF9C040020580E00207A
:10A0800008B520B10448012103F070FE03E0024846
:10A09000012103F06DFE08BD0008014038B5064DF2
:10A0A00001232B60054B002420461C60FFF7E8FFCE
:10A0B00003232B60204638BD405C0040445C0040D8
:10A0C00008B5FFF7EBFF08BD08B50120FFF7D8FF83
:10A0D000064B0121196006494FF4E0520A800549F8
:10A0E0000020186008601A6008BD00BF405C004096
:10A0F000980E0020445C0040084B10B51B680024FB
:10A100009C72FFF7E1FF064A4FF406431460043ADD
:10A110001360044A1460044A138010BD500E0020DE
:10A12000445C00409C040020980E0020002008B5EC
:10A1300004F034F94FF40000012104F0C7F908BD20
:10A1400007B5FFF7F3FFFFF7ABFE06F02BF804208F
:10A15000012104F0ADF903238DF806300D338DF89D
:10A16000073004484FF0010301A9ADF8043003F0B3
:10A1700097FD0EBD00080140704700BF704700BF4B
:10A18000704700BF704700BF704700BF704700BFF7
:10A19000704700BF704700BF08B5FAF78BFA052873
:10A1A00005D9FAF787FA40F2F933984201D901222A
:10A1B00000E00022094B5A60094B1B786BB1074B3A
:10A1C00008495A68084B0A601AB91A6842F008022E
:10A1D00002E01A6822F008021A6008BD5807002041
:10A1E0005207002040070020E806002010B5FFF7C6
:10A1F000BFFB074C2368C31AB3F5FA7F07D9054B99
:10A20000DA6882F00802DA60FFF7B2FB206010BD66
:10A210009C0E002000100140024B03EBC003D879D4
:10A22000704700BFB0040020024B03EBC003587915
:10A23000704700BFB0040020024B03EBC0039879C5
:10A24000704700BFB0040020024B0B2202FB00331A
:10A25000187A7047B0040020024B0B2202FB003337
:10A26000587A7047B0040020024B0B2202FB0033E7
:10A27000D87A7047B0040020024B0B2202FB003357
:10A28000987A7047B0040020024B0B2202FB003387
:10A29000187B7047B0040020024B0B2202FB0033F6
:10A2A000587B7047B0040020024B0B2202FB0033A6
:10A2B000987B7047B0040020024B0B2202FB003356
:10A2C000187C7047B0040020024B0B2202FB0033C5
:10A2D000587C7047B0040020024B0B2202FB003375
:10A2E000987C7047B0040020024B052202FB00332B
:10A2F000187D7047B0040020024B052202FB00339A
:10A30000587D7047B0040020024B052202FB003349
:10A31000987D7047B0040020024B052202FB0033F9
:10A32000D87D7047B0040020024B052202FB0033A9
:10A33000187E7047B0040020024B032202FB00335A
:10A34000187F7047B0040020034B032202FB003348
:10A3500093F91D00704700BFB0040020024B032298
:10A3600002FB0033987F7047B0040020024B03EBE0
:10A37000C00393F820007047B0040020024B03EBA9
:10A38000C00393F821007047B0040020024B03EB98
:10A39000C00393F822007047B0040020024B03EB87
:10A3A000C00393F823007047B0040020024B03EB76
:10A3B000C00393F824007047B0040020024B03EB65
:10A3C000C00393F825007047B0040020024B03EB54
:10A3D000C00393F826007047B0040020024B03EB43
:10A3E000C00393F827007047B004002006281AD84D
:10A3F000DFE800F004070A0D101316000A4B9B6AF1
:10A4000010E0094BDB6A0DE0074B1B6B0AE0064BC3
:10A410005B6B07E0044B9B6B04E0034BDB6B01E0E1
:10A42000014BDB7B0B607047B004002070B5C0F3BC
:10A430000741054600220120FAF75CFC0A4C06029F
:10A44000C5F3072100220120A662FAF753FC064358
:10A4500001203602E9B20246A662FAF74BFC064337
:10A460003609A66270BD00BFB00400202D4B032248
:10A4700002FB003310B51C3393F901203F2A01DDA4
:10A480003F225A70274B032202FB00331C3393F9FF
:10A49000012012F13F0FBCBF6FF03E025A70214BFA
:10A4A000032202FB00331C339A781F2A01D91F2292
:10A4B0009A701C4B032202FB00324FF440211964B6
:10A4C000127F012A04BF4FF450221A64154B03EB8C
:10A4D000C00292F827203AB9033202FB0032527FC1
:10A4E000196C02F07F020BE0032101FB003191F8AF
:10A4F0001DC002F003020CF07C0C196C4CEA020245
:10A50000084C41EA02221A64032303FB0040236C37
:10A51000827F42EA030318462364FFF787FF236C18
:10A52000A36310BDB004002008B5044B032202FB56
:10A5300000339977FFF79AFF08BD00BFB0040020F1
:10A5400008B5044B032202FB00335977FFF78EFF57
:10A5500008BD00BFB004002008B5044B032202FB75
:10A5600000331977FFF782FF08BD00BFB004002059
:10A57000264B052210B502FB00331A7D012A01D9B2
:10A5800001221A75214B052202FB003314335A783D
:10A59000032A01D903225A701C4B052202FB003307
:10A5A00014339A780F2A01D90F229A70174B05227B
:10A5B00002FB00331433DA78032A01D90322DA705C
:10A5C000124B052202FB003314331A790F2A01D9EA
:10A5D0000F221A710D4C052303FB004000F11402F9
:10A5E0001379017D43F42023507843EAC1339178F5
:10A5F00043EA4033D27843EA012343EA4213184640
:10A600002364FFF713FF236C636310BDB0040020C5
:10A6100008B5044B052202FB00331976FFF7A8FFAB
:10A6200008BD00BFB004002008B5044B052202FBA2
:10A630000033D975FFF79CFF08BD00BFB0040020B0
:10A6400008B5044B052202FB00339975FFF790FF14
:10A6500008BD00BFB004002008B5044B052202FB72
:10A6600000335975FFF784FF08BD00BFB004002018
:10A6700008B5044B052202FB00331975FFF778FF7C
:10A6800008BD00BFB0040020514B0B2210B502FBE7
:10A6900000331A7A032A01D903221A724C4B0B2277
:10A6A00002FB003308339A78032A01D903229A70F7
:10A6B000474B0B2202FB003308331A790F2A01D9CA
:10A6C0000F221A71424B0B2202FB003308335A79D6
:10A6D000072A01D907225A713D4B0B2202FB003396
:10A6E00008339A790F2A01D90F229A71384B0B221D
:10A6F00002FB003310335A780F2A01D90F225A7007
:10A70000334B0B2202FB003310339A780F2A01D906
:10A710000F229A702E4B0B2202FB0032117AC903D2
:10A7200041F400241C64527A12B141F404211964EA
:10A73000274B0B2101FB0031C97A19B1196C41F487
:10A7400000511964224B8AB90B3202FB00320832E5
:10A7500092F804C091784FEACC1C1C6C4CEAC12CD6
:10A7600051794CEA040242EA01121DE00B2202FB7D
:10A770000032127C1AB11A6C42F480521A64144BE3
:10A780000B2101FB0031103191F801E01A6C89783E
:10A7900042EACE1201F0070C42EA0C1211F0080F47
:10A7A0001A6402D042F400621A64094B0B2202FBC5
:10A7B00000300830C27922B981791A6C41EA02026C
:10A7C0001A64034C206CFFF731FE236C236310BD29
:10A7D000B004002008B5064B0B2202FB00330833FF
:10A7E000DA791AB10022DA71FFF74EFF08BD00BF17
:10A7F000B004002008B5064B0B2202FB00330833DF
:10A80000DA791AB90132DA71FFF73EFF08BD00BFED
:10A81000B004002008B5044B0B2202FB00339974EE
:10A82000FFF732FF08BD00BFB004002008B5044B9D
:10A830000B2202FB00335974FFF726FF08BD00BF4F
:10A84000B004002008B5044B0B2202FB003319743E
:10A85000FFF71AFF08BD00BFB004002008B5044B85
:10A860000B2202FB00339973FFF70EFF08BD00BFF8
:10A87000B004002008B5044B0B2202FB00335973CF
:10A88000FFF702FF08BD00BFB004002008B5044B6D
:10A890000B2202FB00331973FFF7F6FE08BD00BF61
:10A8A000B004002008B5044B0B2202FB0033997260
:10A8B000FFF7EAFE08BD00BFB004002008B5044B56
:10A8C0000B2202FB0033D972FFF7DEFE08BD00BF8A
:10A8D000B004002008B5044B0B2202FB0033597270
:10A8E000FFF7D2FE08BD00BFB004002008B5044B3E
:10A8F0000B2202FB00331972FFF7C6FE08BD00BF32
:10A90000B004002010B5254B4FF460221A6403EB0D
:10A91000C00292F8272012B14FF470221A641F4B24
:10A9200003EBC00292F8211092F820C01C6C0903BE
:10A9300041EA8C312143196492F82220012A04BF94
:10A9400041F480611964154B03EBC00191F823C0F9
:10A950001A6C42EA0C221A6491F82410012904BFEF
:10A9600042F080021A640D4B03EBC00292F82520DE
:10A97000012A03D11A6C42F040021A64074C04EB1E
:10A98000C00090F82620236C43EA02131846236483
:10A99000FFF74CFD236CE36310BD00BFB004002043
:10A9A00008B5044B03EBC00383F82610FFF7AAFF9A
:10A9B00008BD00BFB004002070B50F4B064603EB86
:10A9C000C00393F82650032D02D00321FFF7E8FFC0
:10A9D0003046FFF797FF084B9C6A14F4002F1CBF0A
:10A9E0006FEA04346FEA1434032D03D0304629464D
:10A9F000FFF7D6FF204670BDB004002008B5044B19
:10AA000003EBC00383F82510FFF77CFF08BD00BFF0
:10AA1000B004002008B5044B03EBC00383F82410F6
:10AA2000FFF770FF08BD00BFB004002008B5044B5D
:10AA300003EBC00383F82310FFF764FF08BD00BFDA
:10AA4000B004002008B5044B03EBC00383F82210C8
:10AA5000FFF758FF08BD00BFB004002008B5044B45
:10AA600003EBC00383F82110FFF74CFF08BD00BFC4
:10AA7000B004002008B5044B03EBC00383F820109A
:10AA8000FFF740FF08BD00BFB0040020064B10B523
:10AA900003EBC003044683F82710FFF733FF20467B
:10AAA000FFF7E4FC10BD00BFB004002010B5144B4C
:10AAB00000221A6403EBC002527912B14FF4007203
:10AAC0001A640F4B03EBC00292791AB11A6C42F46C
:10AAD00080721A640A4B03EBC003DA790F2A01D99A
:10AAE0000F22DA71064C04EBC000C279236C42EAF3
:10AAF000030318462364FFF799FC236CE36210BD3F
:10AB0000B004002070B5084D9DF810E09DF8146069
:10AB100005EBC00426716270A37084F803E005F8A9
:10AB20003010FFF7C3FF70BDB004002008B5034B21
:10AB300003EBC0039971FFF7B9FF08BDB004002013
:10AB400008B5054B03EBC003597109B10422DA7152
:10AB5000FFF7ACFF08BD00BFB004002008B5054BEF
:10AB6000042903EBC003D97101D000225A71FFF709
:10AB70009DFF08BDB00400202DE9F047344D044688
:10AB8000401990F844000E4617469846DDF820908C
:10AB9000DDF824A004281FD8DFE800F003090F1512
:10ABA0001B002046FFF770FD6519012316E02046C3
:10ABB000FFF7A8FE6519022310E02046FFF7D8FC36
:10ABC000651903230AE02046FFF750FC65190423AA
:10ABD00004E02046FFF76AFF6519002385F844303A
:10ABE0001B4B03EBC40494F82620012A0DD002D39A
:10ABF000022A23D111E016B19B6A9B0C3370EFB18E
:10AC0000134B9B6A9B0A3B7018E0B8F1000F15D0FC
:10AC10009B6A9B0AC8F8003010E0B8F1000F04D01E
:10AC20009B6ADB0B5B01C8F80030B9F1000F05D05F
:10AC3000074B9B6AC3F3842389F80030BAF1000FF5
:10AC400003D0034B9B6A8AF80030BDE8F08700BF51
:10AC5000B0040020214B10B5032200244FF0050C56
:10AC600002214FF0010E83F825E0197383F80EC01E
:10AC70009A745C7483F81CE083F81DC083F81EC0CE
:10AC800083F8202083F8212083F8224083F8234092
:10AC900083F8244083F8261083F827401C755C75E0
:10ACA0009C75DC751C765C719C71DC7119725C7230
:10ACB000DC729C725A73DC731C742046FFF758FCDC
:10ACC0002046FFF7D3FB2046FFF71CFE2046FFF788
:10ACD000EDFE2046FFF7D8FC10BD00BFB0040020F9
:10ACE00008B5044A0023917A034A18461370F9F70D
:10ACF000CBFE08BD100C0020780C00202DE9FF4190
:10AD00007F4B1A7822B901321A706FF000425A60F4
:10AD10007B4B1C7A5CB9E0B2F9F7A2FC784B03F1EB
:10AD20000C0210550134082CF5D101221A72272487
:10AD30000025E8B2F9F794FC724A535D834219D0BA
:10AD4000714B291D53F821305055022B05D0032B90
:10AD50000AD0012B0ED168B106E058B96B4A115DDB
:10AD6000012907D1135505E0684B1A5D012A01D16D
:10AD700001321A5501350134082DDAD1644EF369D8
:10AD800093B1644C25787DB9FEF7F2FD624AF36910
:10AD90001268821A002AB8BF52429A4204D9284641
:10ADA00001F08AFA01232370594E336A93B15B4C48
:10ADB00025787DB9FEF7DCFD594A336A1268821A9C
:10ADC000002AB8BF52429A4204D9284601F074FAC8
:10ADD000012323704A4D534C2A7D930004EBC30199
:10ADE0000E7B002E00F028814F48504F504E00211E
:10ADF000C318BF18B61810460A4600970196FFF709
:10AE0000BBFE2B7D04EB4314227B013A042A00F2A3
:10AE10000281DFE812F005004E00D3004E00D3009F
:10AE2000444A374D926812F4805F1BD15D192A7E27
:10AE3000022A04D1404AD25C002A00F0EC80394A50
:10AE40002F4C02EB43121846517AF9F71DFE207D74
:10AE5000FFF7C0FC237D384A0021E418D1540223B7
:10AE60002376D8E05D192A7E012A04D1324AD25CC9
:10AE7000002A00F0D0802B4C184604EB4313997A3B
:10AE8000F9F702FE1E4B187D04EB4014A37A13B9A8
:10AE9000FFF7B0FC04E0284B1B5C0BB1FFF79AFCFA
:10AEA000174A2549137D0020D218C8540123137670
:10AEB000B1E01F4A124DD256002A3FDB5D192A7EAF
:10AEC000022A02D11C4AD25C8AB1164A0C4C02EB0F
:10AED00043121846517AF9F7D7FD207DFFF77AFC27
:10AEE000237D154A0021E418D15402232376044C13
:10AEF000257DFEF73DFD04EB8504606056E000BF54
:10AF0000F804002004050020380C0020880C0020E4
:10AF100008000020750C0020700C0020710B002030
:10AF2000680C0020100C0020A80B00207C0B0020D7
:10AF3000080C002000100140740C00205B191B7EDF
:10AF4000012B11D0FEF714FD2B7D894A05EB8305FB
:10AF500002EB43139B8B0A2253436A68821A002A2E
:10AF6000B8BF52429A4204DC824B834A1B7DD35CB9
:10AF7000E3B1804D7E4C287D04EB4013997AF9F7BC
:10AF800083FD287D04EB4014A37A13B9FFF732FC4C
:10AF900004E0794B1B5C0BB1FFF71CFC754A76494A
:10AFA000137D0020D218C85401231376714B1A7DEB
:10AFB0006F4B03EB42131B7B042B20E06D4A9A1866
:10AFC000127E022A02D16C4AD25C8AB1684A694C6C
:10AFD00002EB43121846517AF9F756FD207DFFF730
:10AFE000F9FB237D644A0021E418D154022323761F
:10AFF000604B1A7D5E4B03EB42131B7B052B0AD182
:10B000005E4B9A6812F4805F0BBF4FF400524FF40E
:10B0100000521A615A61FEF7ABFC564CE369C31A41
:10B02000002BB8BF5B420A2B40F36783F9F7B4FBF0
:10B03000FEF79EFCE06160E3F9F7AEFBFEF798FCDB
:10B04000EB69C31A002BB8BF5B420A2B40F3558350
:10B05000297D3046490141F00A0101F0EA0100F082
:10B06000EDFF0446287D01F04BF92B7D0C20584361
:10B0700043494218157A0DB1455800E05568414AD8
:10B08000D25C032A00F2E480DFE802F002801C4B6D
:10B09000002C00F0DD80364A364D02EB4311C97FAB
:10B0A000384E29B11846F9F7EFFC2B7D032207E053
:10B0B00002EB43121846517AF9F7E6FC2B7D022287
:10B0C000F254C5E04CB95B0143F0080101F0E8011E
:10B0D000204600F0B3FF002862D0264E244B307D7E
:10B0E00003EB4013D97F002900F0AB80002D84EAE8
:10B0F000E472B8BF6D42A2EBE472AA4202D0002C07
:10B1000040F09980204B53F830108A4280F09980AB
:10B1100003EBC0031979F9F7B7FC164B01211B7D2E
:10B120008DE0002D84EAE471B8BF6D42A1EBE471BB
:10B13000A94202D0002C40F08480134A0D4D52F8F1
:10B140003300104E814208D202EBC3021846117937
:10B15000F9F79AFC2B7D012208E0054A184602EB1C
:10B160004313597AF9F790FC2B7D0222F25468E0E0
:10B17000100C0020F8040020740C00200010014086
:10B18000BC0B0020780C0020800B002044BB5B012E
:10B1900043F0080101F0E801204600F04FFFF8B944
:10B1A000FEF7E6FB1F4D204A2B7D4FF00A0E02EB07
:10B1B0004311B1F81CC099004E1976680EFB0CFCC7
:10B1C000861B002EB8BF7642664541DD02EBC10208
:10B1D0001846917AF9F758FC2B7D144AD45437E07D
:10B1E000104E114A337D02EB4312D17F49B3002D3B
:10B1F00084EAE472B8BF6D42A2EBE472AA4200D0C6
:10B20000C4B90B4951F833108A421AD3064A18467A
:10B2100002EB4313597AF9F737FC024B02211B7DED
:10B220000DE000BFF8040020100C0020780C002076
:10B23000800B00201846F9F727FC337D0321A34A31
:10B24000D154A34D2E7DFEF793FB05EB8605686078
:10B250009F4DA04F2B7DA04E1846F618FF189F4B10
:10B26000002103EB80030A46019600979C4EFFF7EE
:10B2700083FC287D06EB40139B6943B3F9F7F8F88C
:10B2800028B3287D84EAE47206EB40139B69A2EBA5
:10B29000E4729A421BD901F00FF82A7D914906EB1E
:10B2A00042139B7F0120885443B1B27F9A4205D15B
:10B2B000013801F001F8002000F03AFA844B8A4A84
:10B2C0001B7D0F33D15C012901D10131D154804D57
:10B2D0002B7D022B25D8002000F08CFD95F8203026
:10B2E00010F0010F03F0F80385F820301CBF43F085
:10B2F000010385F8203010F0040F8DF80C0006D003
:10B30000734B93F8202042F0020283F8202010F0C3
:10B31000100F06D06E4B93F8202042F0040283F801
:10B320002020724A137853B1694991F820100B42DA
:10B3300005D16F496F480978037001B911706D4BE1
:10B340001B784BB1624A92F8202003EA02029A422B
:10B3500002D1694B01221A705D4B93F8202012F044
:10B36000010F0AD093F8213013F0010F05D15E4B85
:10B37000DA78012A01D10132DA70554B93F8202096
:10B3800012F0020F0AD093F8213013F0020F05D10A
:10B39000554B1A79012A01D101321A714C4B93F89D
:10B3A000202012F0040F0AD093F8213013F0040F7C
:10B3B00005D14D4B5A79012A01D101325A71444DC0
:10B3C00003222B7D04A8B3FBF2F2821812F9042C9D
:10B3D00095F82010002A85F821104ADA5B0143F025
:10B3E0001601002001F0F60102AA00F03FFE9DF8D0
:10B3F0000A3013F0400F08D02A7D3B4952001B321F
:10B40000885C012801D10130885413F0800F0AD0E4
:10B410002F49354A097D0E3112F81100012802D159
:10B42000013002F8110013F0100F09D0284A2E49FC
:10B43000127D52001B32885C012801D101308854F2
:10B4400013F0200F0AD0224A274B127D0E3213F838
:10B450001210012902D1013103F812101C4B0020F7
:10B46000197D02AA490141F0160101F0F60100F030
:10B4700099FF174F1A4E3B7D06EB43125269002A83
:10B4800000F081801D4AD55C002D7CD1002C7AD043
:10B490005B0143F0020101F0E201284600F094FD57
:10B4A0008046387DF9F770FA397DC0EB080806EB65
:10B4B00041135B69B8F1000F83EAE372B8BFC8F1CA
:10B4C0000008A2EBE37290455DDD19E0780C0020E6
:10B4D000F80400207C0B0020080C0020A80B0020A2
:10B4E000100C0020040C0020880C0020A40B00206D
:10B4F000780B0020940B0020BC0C00208C0B00204B
:10B50000002B0EDD084600F0D7FE3B7D06EB431313
:10B510009B7F3BB3B27F9A4224D1284600F0CCFEF9
:10B520001DE02846022200F029FD397D2846490108
:10B5300041F0080101F0E80100F0A0FE3B7D06EBC0
:10B5400043139B7F73B1B27F9A420BD129462846A1
:10B55000022200F013FD2846082100F08FFE284645
:10B5600000F0E6F8664B674A1B7D1533D15C012974
:10B5700001D10131D154624B634A1B7D0121184630
:10B58000D15400F0D5F8614F3B68002B47D05C4E9A
:10B590005D4A337DD55C002D41D1002C40D05B014C
:10B5A00043F0020101F0E201284600F00DFD804663
:10B5B000307DF8F79DFF3B68C0EB0808B8F1000F3D
:10B5C00083EAE372B8BFC8F10008A2EBE3729045CA
:10B5D00031DD002B317D03DD084600F06DFE0CE00F
:10B5E0002846022200F0CAFC317D2846490141F07C
:10B5F000080101F0E80100F041FE414B414A1B7D8A
:10B600001533D15C012901D10131D1543C4B3E4A63
:10B610001B7D01211846D15400F08AF80BE054B983
:10B62000374B0020197D490141F0080101F0E80184
:10B6300000F004FD20B1324D354B2E7D9B5D43B3B0
:10B640002F4B344A1B7D02EB4312D28912B9304A88
:10B65000D35C1BB3FEF78CF9294D2E492B7D4FF09F
:10B660000A0C9A0001EBC201C9895219526A0CFBFB
:10B6700001F1821A002AB8BF52428A420EDD264EDC
:10B68000F25C5AB91846FFF7B5F82B7D0122F25447
:10B6900004E0FEF76DF905EB86056862184E1F4D54
:10B6A000307D002C55F83030B8BF64429C420AD23D
:10B6B000FEF73AFE337D05EBC3056A7982420DD170
:10B6C0001846002108E0FEF72FFE337D05EBC30589
:10B6D0006979884202D01846FEF79AFF084C207D0F
:10B6E00000F034F8237D0133DBB223750BB1002366
:10B6F0002375FEF73DF9024BD861BDE8FF8100BF1D
:10B70000F8040020880C00208C0B00209C0B0020EB
:10B71000800C0020100C0020840C0020800B0020E6
:10B72000024B1A5C0AB901321A54704720050020F6
:10B73000024B1A5C0AB10F221A54704720050020F0
:10B74000014B185C704700BF200500202DE9F3472E
:10B750004601F5B2044645F07C01002001AA00F044
:10B7600085FCB74A610002EB4413187A06EB020726
:10B7700010F0400F9DF8063012D04FF001084FF046
:10B78000020C08FA01F80CFA01FCB1587E680CEAC8
:10B79000030208EA0307C1F10009C6F1000A0FE03D
:10B7A0004FF0010C4FF002080CFA01FC08FA01F10D
:10B7B00056F80290D7F804A00CEA030201EA030746
:10B7C00010F0800F00F03F0606D09E4B9B6883F47C
:10B7D0000048C8F3C03803E09A4B9B68C3F3C038F5
:10B7E000731E072B00F2D182DFE813F00800080077
:10B7F000080008006E016E016E016E01924B1B5D28
:10B80000013B0E2B00F2C182DFE813F00F003D0078
:10B81000530062007A0082008E00A000D100140163
:10B820002401BF0243014E01A60201AA45F0140102
:10B830000020854F00F01AFC9DF8053045F0060504
:10B8400007EB8408C8F804302946002000F0F6FB16
:10B850000222C8F808002146002000F08FFB023EBB
:10B860000020294640F2FF7200F0F4FCF6B20020FE
:10B870000322214600F05CFB012E01D8022300E0E8
:10B8800004233B5581E2704E002006EB84035A6886
:10B89000214602F00402824214BF0522012200F078
:10B8A00047FB45F008014A46002000F0D3FC032383
:10B8B00024E0002A00F0698245F00201002000F037
:10B8C00083FB614B04221A55604B43F824005CE271
:10B8D0005D4E002006EB84035A68214602F0040204
:10B8E000824214BF0622022200F022FB45F008012A
:10B8F000C9F10002002000F0ADFC0523335544E2FD
:10B90000002F00F04282204600F0D6FC06222FE2F3
:10B9100000202146032200F00BFB45F008015246AF
:10B92000002000F097FC68E1002F40F02E8245F0E7
:10B9300008053A463846294600F08CFCCAF1000258
:10B940003846294600F086FC082211E2002F00F05C
:10B950001C8245F00201002000F036FB0646002064
:10B96000024645F0080100F075FC384B002053F802
:10B9700024702146BF1B43F82470032200F0D8FA3C
:10B980008AEAEA7245F00601A2EBEA72002000F0B2
:10B9900061FC610101F0E0013246002000F0C6FBCD
:10B9A00000200246214600F0E9FA0922E0E10020E9
:10B9B00000F020FA630050FA03F313F0010F00F0D7
:10B9C000E48145F002073946002000F0FDFA204BE3
:10B9D00045F0080543F8240000200246294600F0FF
:10B9E00039FC00200222214600F0C8FA002002465D
:10B9F000394600F09BFB00206101024601F0E001A6
:10BA0000033E00F093FBF6B200212046F8F792FFC8
:10BA1000012E0D4E0CD800202146022200F0AEFA75
:10BA20002946CAF10002002000F014FC0A2365E751
:10BA30000E2363E7002F00F0A8810B2298E100BFDE
:10BA4000100C00200008014020050020740B00208D
:10BA5000340C0020002F40F0988145F00201384658
:10BA600000F0B2FA45F0080106463A46384600F0C2
:10BA7000F1FB6101022296FBF2F201F0E00138468F
:10BA800000F054FB3A463846214600F077FA0D2282
:10BA90006EE1002000F0AEF9630050FA03F313F0FA
:10BAA000010F00F0728162E1A84E45F0060106EB3D
:10BAB00084050020AA6800F0CDFB2A7900202146E9
:10BAC00000F036FA002319E7A04B1B5D013B0E2B5B
:10BAD00000F25B81DFE813F00F00340052006200D7
:10BAE00081005901930059015901CC00DC00AD00DF
:10BAF00008014F01400145F0140101AA0020934FB5
:10BB000000F0B4FA9DF805C007EB84030020022280
:10BB1000C3F804C0214600F031FA002045F00601C8
:10BB200040F2FF7200F096FB00200322214600F055
:10BB3000FFF9062E02D0082E7FF4A2AE022217E1F2
:10BB4000062E0CD1814B002003EB84035A6821465A
:10BB500002F00402824214BF0522012204E0082EF2
:10BB600004D100202146032200F0E2F94A4645F0C4
:10BB70000801002000F06EFB0322F9E0731FDBB226
:10BB8000012B05D822B1062E704E30D10423B5E624
:10BB9000B8F1000F00F0F9800C22E9E0052E0CD17D
:10BBA0006A4B002003EB84035A68214602F004022A
:10BBB000824214BF0622022204E0072E04D1002094
:10BBC0002146032200F0B4F9C9F1000245F0080152
:10BBD000002000F03FFB0522CAE0731FDBB2012BFF
:10BBE00007D837B1052E594E01D1022386E60F231F
:10BBF00084E6B8F1000F00F0C8800722B8E0B8F181
:10BC0000000F40F0C280073EF6B2012E0DD94F4B17
:10BC1000404603EB84035A68214602F00402002ADE
:10BC200014BF0522012200F083F945F008015246B5
:10BC300019E0B8F1000F40F0A880073EF6B2012EDF
:10BC40000DD9424B404603EB84035A68214602F06B
:10BC50000402002A14BF0622022200F069F945F00E
:10BC60000801CAF10002002000F0F4FA0A227FE085
:10BC7000B8F1000F00F0898045F00201002000F0CB
:10BC8000A3F9324B0B2103EB84021955D0607CE001
:10BC9000B8F1000F79D145F00201404600F094F967
:10BCA0002B4BA700294E03EBC7038AEAEA728146B1
:10BCB00045F00601A2EBEA72404683F80D80BF19F9
:10BCC00000F034FAFB6861019944022399FBF3F216
:10BCD00001F0E001404600F029FA40462146424684
:10BCE00000F04CF90D2309E6002000F083F8630012
:10BCF00050FA03F313F0010F47D0144B0E2245F016
:10BD000002061A553146002000F05EF9114B45F04D
:10BD1000080143F824000020024600F09BFA214667
:10BD20000020022200F02AF900203146024600F0ED
:10BD3000FDF900206101024601F0E00100F0F6F992
:10BD400020460021F8F7F6FD1FE000BF2005002087
:10BD5000100C0020340C002000202146022200F0AC
:10BD60000DF9002045F00801024600F073FA0E229A
:10BD7000074B1A5509E0064D002005EB84031A799C
:10BD8000214600F0D5F800232B55BDE8FC8700BF05
:10BD90002005002000000000154B10B503EB001239
:10BDA000926891420EDD8A1AC2F18074A2424FEA73
:10BDB000001C03DC63445C6812190EE063445A689B
:10BDC000141B0FE00FDA521AC2F18074A2424FEA3C
:10BDD000001C04DC63445C68A21A5A6003E06344FC
:10BDE0005A68A4185C60024B03EB0010816010BD20
:10BDF000A00E0020012108B502200A46F8F77AFFBC
:10BE000008BD00BFF8B51378144613F0600F06465E
:10BE10000D4627D1414A127B22BB13F0010F21D1DD
:10BE20005F2B1FD83E4A1278E2B913F09F0301D06E
:10BE3000082B17D13B4F387860B9384BD97F19B1EF
:10BE4000F8F722FE032304E00846597AF8F71CFEAF
:10BE500002233B70344F3B7823B10020FEF7BAFC3D
:10BE600000233B70002221780220F8F743FF28705E
:10BE7000002261780220F8F73DFF68700022A17867
:10BE80000220F8F737FFA87001220220E178F8F7C6
:10BE900031FFE870237813F0010F3ED15F2B3CD8BF
:10BEA00003F01E02082A04D0142A2CD0062A34D10A
:10BEB0001BE0242171435B090C2000FB0313A578D0
:10BEC00094F803C0194A4CEA05259D50A37813F055
:10BED000080F22D02678760900FB0616B3586FEAC1
:10BEE00003536FEA1353B35017E0242256435B0900
:10BEF0000C22A17802FB0363E27842EA01220B499B
:10BF00005B185A6009E0242256435B090C2202FBAD
:10BF100003630649E2785B181A72F8BD100C002022
:10BF2000800C0020780C0020840C0020BC0B00202A
:10BF30002DE9F3414901CEB201AC46F01503174695
:10BF4000694622468DF804308046FFF75BFF9DF876
:10BF500001C09DF8033046F014064046694622466B
:10BF60006D468DF804608DF805C08DF806708DF86B
:10BF70000730FFF747FFBDE8FC8100BF2DE9F34123
:10BF80004901CEB201AC46F0150317466946224678
:10BF90008DF804308046FFF735FF9DF801C09DF80D
:10BFA000023046F014064046694622466D468DF83A
:10BFB00004608DF805C08DF806308DF80770FFF726
:10BFC00021FFBDE8FC8100BF37B541F001030C46FD
:10BFD0006A4601A98DF800300546FFF713FF9DF86A
:10BFE00006009DF8052000029DF8073040EA024057
:10BFF000184310F4000F18BF40F07F405F2C1AD890
:10C00000C4F3411314F01E0402D0022C13D106E035
:10C01000032202FB0535084A2D01A8580BE0032234
:10C0200002FB053520F07F41E8B2FFF7B5FE024B79
:10C0300003EB051568683EBDA00E002007B541F072
:10C0400001036A4601A98DF80030FFF7DBFE9DF879
:10C0500006009DF8073043EA002010F4006F1CBF73
:10C060006FEA00506FEA10500EBD00BF13B541F0EB
:10C070000103144601A96A468DF80030FFF7C2FE9D
:10C080009DF805109DF806309DF807202170A270DC
:10C0900063709DF804001CBD07B5410141F0160115
:10C0A00001F0F601002001AAFFF7E0FF9DF805303E
:10C0B000D80913F0200F18BF40F002000EBD00BFDA
:10C0C00007B5410141F0160101F0F601002001AA77
:10C0D000FFF7CCFF9DF80530C3F3801013F0100F6D
:10C0E00018BF40F002000EBD37B50C4641EA4011C2
:10C0F00001AA0546C9B20020FFF7B8FFB4235D438B
:10C100006408032305F5807503FB04549DF80410AF
:10C110002046FCF795FB601C9DF80510FCF790FB92
:10C12000A01C9DF80610FCF78BFB3EBD5F292DE996
:10C13000F3410D460646144662D8C1F3411811F08A
:10C140001E0102D002295BD11EE0032202FB0088FF
:10C15000344A4FEA081083185B688450E01A0028BC
:10C16000B8BF4042B0F5000F0ADB9C42CCBF2E4C5A
:10C170002E4C2C4A1C1902EB0812012313733FE0CA
:10C1800002EB081211733BE0032707FB0087254BE6
:10C190003801C1587A00C4EB010C0132BCF1000F28
:10C1A000B8BFCCF1000C00EB030EBCF5000F24F07F
:10C1B0007F40CEF8044043F832001DDBA142CCBFE3
:10C1C000194B1A4B4FEA4818E3184FEA234E4FEA2F
:10C1D000232C3046694601AA8DF807308DF804807B
:10C1E0008DF805E08DF806C0FFF70CFE0D4B03EB54
:10C1F000071701233B7303E003EBC20300221A710C
:10C200004FEA244C23123046694601AA8DF80450A7
:10C210008DF805C08DF806308DF80740FFF7F2FD68
:10C22000BDE8FC81A00E0020FFFF7F00010080FF21
:10C2300038B50D4668210446FFF7C6FE15B140F03B
:10C24000010201E020F0010220466821FFF76EFFA5
:10C2500038BD00BF07B513464FEA222C8DF80410F5
:10C260004FF0000E694601AA8DF805E08DF806C072
:10C270008DF80730FFF7C6FD0EBD00BF07B50B46B2
:10C2800011F01E01024601D0022905D110461946BF
:10C290000022FFF74BFF0DE04FF0000C694601AAAA
:10C2A0008DF804308DF807C08DF805C08DF806C0F4
:10C2B000FFF7A8FD0EBD00BF10B5C4B22146640152
:10C2C00000200222E4B2FFF759FE002044F00801EA
:10C2D000FFF7D4FF44F00A010020FFF7CFFF10BDA5
:10C2E00007B59DF810C08DF804108DF8052069463B
:10C2F00001AA8DF806308DF807C0FFF783FD0EBD4B
:10C3000030B5430185B0044643F00303002003A980
:10C3100002AA8DF80830FFF775FD9DF80E109DF804
:10C320000D209DF80F30090241EA024119432046D1
:10C33000FFF732FD174B03EB041108310A7932B3D2
:10C34000154A0C2000FB0422107A00BB2201D518EC
:10C35000D2586B68C3EB020CBCF1000FB8BFCCF134
:10C36000000CBCF5000F05DB9A42CCBF0B4A0C4A0F
:10C370009A1800E008716101C2F30723D4B201F0FA
:10C38000E0010020C2F307420094FFF7A9FF05B0C7
:10C3900030BD00BFA00E0020BC0B0020FFFF7F00BF
:10C3A000010080FF07B5937892F800E092F801C091
:10C3B0008DF8041001AA69468DF805E08DF806C0D5
:10C3C0008DF80730FFF71EFD0EBD00BF37B54401E5
:10C3D00044F01604E4B20D4601AA21460020FFF7FE
:10C3E00045FE9DF8053015F0010F1ABF6FEA436353
:10C3F0006FEA536303F07F038DF805309DF8053035
:10C4000015F0020F14BF43F0200323F020038DF832
:10C41000053000231846214601AA8DF80630FFF7A3
:10C42000C1FF3EBD37B5440144F01604E4B20D46E9
:10C4300001AA21460020FFF719FE9DF8053015F0EE
:10C44000010F14BF43F0400323F040038DF8053083
:10C450009DF8053015F0020F14BF43F0100323F0D0
:10C4600010038DF8053000231846214601AA8DF8E7
:10C470000630FFF797FF3EBD73B5B42545434B0823
:10C48000032205F5807502FB0355044628460E4637
:10C49000FCF740F98DF80400681CFCF73BF98DF8B7
:10C4A0000500A81CFCF736F946EA44148DF806008E
:10C4B000E1B2002001AAFFF775FF7CBD2DE9F74F1F
:10C4C0004001C7B24C05002047F0180101AAFFF750
:10C4D000CDFD9DF80560640D06F00F053609B542E7
:10C4E0000EDB204605F090F9AD1B80460120A840E8
:10C4F000894605F099F90022334B05F0FBF90FE06E
:10C50000204605F081F9751B80460120A840894628
:10C5100005F08AF902460B4600202B4905F014FB72
:10C5200002460B464046494605F00EFB05F0A4FCCA
:10C5300005F08CF922A3D3E9002305F0DBF905F01F
:10C540009BFC05F083F90022204B05F0D3F94FF056
:10C55000FF36B046002582468B460120A84005F0F4
:10C5600063F902460B465046594605F0C3F905F0FB
:10C570005BFCA0F180027F2A98BF2E46034605F19E
:10C58000010588BF43460E2D01D09846E5E70025FA
:10C5900047F0120101AA28468DF805308DF8066093
:10C5A0008DF80450FFF7FEFE284647F00C012246A6
:10C5B000FFF750FE2846BDE8FE8F00BFAFF30080B6
:10C5C00004560E2DB29DEF3F000060400000204059
:10C5D00013B5154B587E10F0010003D000206821E0
:10C5E000212201E0682120220024FFF79FFD204640
:10C5F0007E21202223460094FFF772FEE1B2002044
:10C600000134FFF739FF1D2CF8D10C210020FFF772
:10C61000DBFC01460020FFF751FF0020162143F20A
:10C62000FF12FFF717FE1CBD08000020AFF30080CB
:10C63000084B1868034605E02C2A02D100221A7024
:10C6400003E001331A78002AF6D1024A013313605D
:10C65000704700BF3005002010B50E4B02461B7816
:10C66000ABB10D4B1C7994B19C68601CE4180D2A89
:10C670002273986002D03F2800D851B9064C014679
:10C6800004F10C00FDF7EAFB0023A36001E0FCF7D6
:10C690001BFB10BD700B00203005002030B50121C0
:10C6A000044687B02020FFF7D7FF002C04DA2D20A6
:10C6B0000121FFF7D1FF644200230A2194FBF1F22C
:10C6C00001FB124101AD3031E954591C141E01DD4A
:10C6D0000B46F2E7ED181C460121013C15F8010953
:10C6E000FFF7BAFFB4F1FF3FF6D107B030BD00BF8E
:10C6F00038B50C4D0446A87801214030C0B2FFF790
:10C70000ABFF687801214030C0B2FFF7A5FF207869
:10C71000FFF7C4FF6068FFF7C1FF0D200121FFF79D
:10C720009BFF38BD0800002070B5124B06461B78F1
:10C73000EBB1FCF747FA104C054618B10023237102
:10C74000012016E0E36C226D934208D21A1992F888
:10C750005420013301203270E364207109E004F1B8
:10C760005400FDF749FBE5642065284601E0FCF72D
:10C7700029FA70BD700B0020300500202DE9F3412F
:10C7800004460DF10700FFF7CFFF002800F0CB8033
:10C790008B4B8C4A93F8941019BB51789DF8070085
:10C7A000403188420DD1D3F89810002940F0BB8069
:10C7B0001179012231F0010183F8942040F0B38017
:10C7C000AFE00D2801D01B2802D100227C4B05E0F0
:10C7D000D3F898207E2A00F2A6800132C3F8982070
:10C7E000A1E0117931F0010103D19DF80700FFF7B5
:10C7F00033FF9DF807301F2B0BD9714AD2F89810E0
:10C800007E297FD8481C891881F89C30C2F898008E
:10C8100078E0082B08D16A4BD3F89820002A71D011
:10C82000013AC3F898206DE00D2B6BD1644BD3F81F
:10C830009830002B66D0634B1A79112A15D158789D
:10C8400001214030C0B2FFF707FF002503E0585D2B
:10C85000FFF702FF01355A4B0121D3F898209C3392
:10C860009542F4D30D20FFF7F7FE554A00231568D3
:10C87000D2F8987019461A4633E001290FD002D336
:10C8800002292DD122E04E4E06F19C00805C20282A
:10C8900026D09E1986F81C010133012120E048486A
:10C8A00000F19C0C1CF802C0BCF1200F0AD1012B36
:10C8B00004D91818002180F81C110133424D0221BF
:10C8C000ED180DE0181880F81CC108E03C4E06F188
:10C8D0009C00805C202803D09E1986F81C0101333F
:10C8E0000132BA42C9D3364A0021981880F81C1187
:10C8F0000120C2F89810156082F8A001C2F89C319E
:10C9000082F894109DF807301B2B0CD12D4A2C4B2C
:10C9100012790021012A83F89410C3F8981002D1EB
:10C920000D20FFF799FE264B93F8A001002878D040
:10C930000022164683F8A0211546DFF8A8800727B5
:10C9400007FB058720483946013504F03BF930B92B
:10C95000BE797B7916F0010F237049D007E018F8F3
:10C9600006300736002B5ED0FF2DE6D15BE0FFF7E7
:10C970005FFE23780546042B0CD1144904F022F9FC
:10C980000346D8B12846124904F01CF970B1284674
:10C9900010490FE00D2B28D10F4904F013F903467D
:10C9A00060B128460D4904F00DF908B9012305E0EE
:10C9B0000B49284604F006F9B0B90223637017E06A
:10C9C00030050020080000204C060020012F01083F
:10C9D000052F0108092F01080F2F0108152F010845
:10C9E0001A2F0108F82C0108284604F0E5F86070B9
:10C9F00016F0020F04D0FFF71BFE04F0DDF8A07064
:10CA000016F0040F0CD0FFF713FE04F0D5F8010E5A
:10CA1000C0F30722C0F30743A17122716371E07074
:10CA20000120BDE8FC8100232370F9E7704700BFB7
:10CA3000FEE700BFFEE700BFFEE700BFFEE700BF66
:10CA4000704700BF704700BF704700BF704700BF0E
:10CA5000704700BF704700BF704700BF704700BFFE
:10CA6000704700BF704700BF704700BF704700BFEE
:10CA7000704700BF704700BF704700BF704700BFDE
:10CA8000704700BF704700BF704700BF704700BFCE
:10CA9000704700BF704700BF08B5024B1B6898473E
:10CAA00008BD00BF980B002008B5024B1B689847D3
:10CAB00008BD00BF7C0C002008B5024B1B689847DE
:10CAC00008BD00BF0C0C002008B5024B1B6898473E
:10CAD00008BD00BF300C0020704700BF704700BF8A
:10CAE000704700BF704700BF704700BF704700BF6E
:10CAF000704700BF704700BF704700BF704700BF5E
:10CB0000704700BF704700BF704700BF704700BF4D
:10CB1000704700BF704700BF704700BF704700BF3D
:10CB2000704700BF704700BF704700BF704700BF2D
:10CB3000704700BF704700BF704700BF704700BF1D
:10CB4000704700BF704700BF704700BF704700BF0D
:10CB5000704700BF704700BF704700BF704700BFFD
:10CB6000704700BF704700BF704700BF436830B5D3
:10CB700023F470230C680A7923F48073234343EA77
:10CB80000223436082688D68CC680A4B45EA040C36
:10CB900002EA03034A794CEA030343EA420383604F
:10CBA0000B7CC26A013B22F47002DBB242EA0353FF
:10CBB000C36230BDFDF7F1FF002301220274C360A0
:10CBC0000360037143718360704700BF19B18368CC
:10CBD00043F0010302E0836823F0010383607047A0
:10CBE00019B1836843F4807302E0836823F480738F
:10CBF00083607047C9B212B14368194302E04368C9
:10CC000023EA010141607047836843F008038360B1
:10CC1000704700BF8068C0F3C0007047836843F06E
:10CC200004038360704700BF8068C0F380007047D2
:10CC300019B1836843F4A00302E0836823F4A003DE
:10CC4000836070478068C0F3805070474368013943
:10CC500023F4604343EA41334360704719B14368AA
:10CC600043F4006302E0436823F4006343607047C9
:10CC7000092930B511D94FF0030C0CFB01FC072535
:10CC8000ACF11E0C05FA0CF503FA0CFCC46824EA9E
:10CC9000050343EA0C03C3600EE04FF0030C0CFBEA
:10CCA00001FC072505FA0CF503FA0CFC046924EADB
:10CCB000050343EA0C030361062A0DD80523013A54
:10CCC0005A434FF01F0C0CFA02FC9140436B23EACD
:10CCD0000C020A4342631CE00C2A0DD805235A4378
:10CCE0004FF01F0C233A0CFA02FC9140036B23EA2D
:10CCF0000C020A4302630CE005235A434FF01F0C59
:10CD0000413A0CFA02FC9140C36A23EA0C020A433E
:10CD1000C26230BD19B1836843F4801302E08368B6
:10CD200023F4801383607047C06C80B2704700BFEB
:10CD3000014B1868704700BF4C24014019B143688B
:10CD400043F4806302E0436823F4806343607047E8
:10CD500019B1436843F4805302E0436823F48053DD
:10CD600043607047836823F4E04341EA0303836030
:10CD7000704700BF19B1836843F4004302E0836841
:10CD800023F400438360704719B1836843F40213AE
:10CD900002E0836823F40213836070478068C0F365
:10CDA00040507047092930B511D94FF0030C0CFBE6
:10CDB00001FC0725ACF11E0C05FA0CF503FA0CFC7E
:10CDC000C46824EA050343EA0C03C3600EE04FF095
:10CDD000030C0CFB01FC072505FA0CF503FA0CFC0F
:10CDE000046924EA050343EA0C030361836BC3F37C
:10CDF000015CCCEB020202324FF0050CD2B20CFB0C
:10CE000002F20CF11A0C0CFA02FC914023EA0C031A
:10CE10000B43836330BD00BF836B013923F44013A0
:10CE200043EA0153836370470A50704728304058E3
:10CE300080B27047436823F4400323F4007341EA4F
:10CE400003034360704700BF41628262704700BFC6
:10CE5000436823F01F0341EA03034360704700BFA8
:10CE600020B1054B9A6842F4000203E0024B9A6835
:10CE700022F400029A6070470024014003681942BE
:10CE80000CBF002001207047C9430160704700BFFC
:10CE90004368006810EA112004D0C9B219420CBFDF
:10CEA00000200120704700BF6FEA11210160704728
:10CEB00008B5134B98420FD003F5A053984213D0F6
:10CEC000A3F5C053984219D14FF40070012101F02D
:10CED0000BFB4FF400700EE04FF48060012101F075
:10CEE00003FB4FF4806006E04FF40040012101F0A5
:10CEF000FBFA4FF40040002101F0F6FA08BD00BF34
:10CF000000280140374B01221A605A6812F00102D2
:10CF100001D1104664E00278012A0BBF1A681A6832
:10CF200042F0800222F080021A604378012B04D183
:10CF30002C4B1A6842F0400203E02A4B1A6822F098
:10CF400040021A608378012B04D1264B1A6842F004
:10CF5000200203E0234B1A6822F020021A60C378F3
:10CF6000012B04D11F4B1A6842F0100203E01D4B45
:10CF70001A6822F010021A600379012B04D1194BB0
:10CF80001A6842F0080203E0164B1A6822F0080201
:10CF90001A604379012B04D1124B1A6842F0040243
:10CFA00003E0104B1A6822F004021A608279C379F8
:10CFB00090F808C0920742EA03624189437A42EA44
:10CFC0000C4242EA03520139064B0A43DA611A68FD
:10CFD00022F001021A60586880F0010000F00100A0
:10CFE000704700BF0064004090F800C0012202FAC0
:10CFF0000CF23B4B2DE9F045D3F8004292B244F0DD
:10D000000104C3F80042D3F81C42D14301EA0404EE
:10D01000C3F81C428478A4B90CF1480CD3F80C7204
:10D02000B0F80AA0C688B0F8088085884FEACC041A
:10D0300004F1804446EA0A4645EA084501EA070742
:10D0400015E0012C1AD10CF1480CD3F80C72B0F891
:10D0500004A0C688B0F8088045894FEACC0404F1E2
:10D06000804446EA0A4645EA084542EA070704F5CD
:10D07000C844C3F80C7243F83C60656043782BB930
:10D08000174BD3F8044201EA040404E0144BD3F82C
:10D09000044242EA0404C3F80442838923B9104BD2
:10D0A000D3F81442214006E0012B06D10C4BD3F8F3
:10D0B000141242EA0101C3F81412837B012B05D13B
:10D0C000074BD3F81C120A43C3F81C22044BD3F8B5
:10D0D000002222F00102C3F80022BDE8F08500BF63
:10D0E0000064004003220272013A002342724FF0B2
:10D0F0000102C3714281037043708370C370037176
:10D1000043718371704700BF19B1054B5A691043D1
:10D1100003E0034B5A6922EA00005861704700BFE0
:10D1200000640040364B70B59968024611F0806F7C
:10D1300001D000200CE0996811F0006F01D00120AF
:10D1400006E09B6813F0805F01D1042056E00220C6
:10D150002B4B00F118010901CC5804F00104CC500C
:10D16000157A92F809C035B9146864051460CD5871
:10D170004CEA050C07E0546845EA0C0CE4005460E6
:10D18000CE584CEA060C4CEA0404CC50947A00F1D8
:10D19000180C4FEA0C1C04F00F040CF1804394723D
:10D1A00003F5C8435D68010125F00F055D605D680A
:10D1B00001F180412C435C60537B947BD57A1B0446
:10D1C00043EA0463147B2B4343EA042301F5C8417B
:10D1D000C1F88831557C937CD47B2D0445EA0365E6
:10D1E000137C45EA040242EA0322054BC1F88C2174
:10D1F0005CF8032042F001024CF8032070BD00BF30
:10D2000000640040012810D002D302282CD11AE07B
:10D21000164A91689368926801F0010103F00203D5
:10D2200043EA8103C2F380621AE0104A936891686E
:10D2300003F48073926801F400719B0943EA11239F
:10D24000C2F3C0620CE0094A9368916803F480332A
:10D25000926801F400319B0B43EA1143C2F3007260
:10D260001343034AD05C70470023FAE70064004090
:10D27000D82D0108012808D002D302280FD109E0D7
:10D28000074B9A6842F0800208E0054B9A6842F426
:10D29000004203E0024B9A6842F400029A60704731
:10D2A0000064004018B9044B2022DA6002E0024B0F
:10D2B00020221A61704700BF0064004010B9064B7D
:10D2C000D86805E0012801D0002003E0024B18696E
:10D2D00000F00300704700BF00640040254B00F1E0
:10D2E0001B02120110B5D45804F004040C721CB9CE
:10D2F000D3585B0D0B6002E0D358DB084B6000F1A4
:10D300001B021C4B1201D35802F1804203F00203AE
:10D310004B7202F5C8425468030104F00F0C81F807
:10D320000AC0526803F18043120ACA7403F5C84365
:10D33000D3F8B821CA72D3F8B821120A0A73D3F805
:10D34000B821120C4A73D3F8B821120E8A73D3F89D
:10D35000BC21CA73D3F8BC21120A0A74D3F8BC21C9
:10D36000120C4A74D3F8BC311B0E8B74FFF79AFF72
:10D3700010BD00BF00640040044B1A6842F0020276
:10D380001A601868C0F34000704700BF0064004096
:10D39000054B1A6822F002021A60186880F0020039
:10D3A000C0F34000704700BF00640040034B9B691E
:10D3B00018420CBF00200120704700BF00640040ED
:10D3C000024B9A6922EA00029A61704700640040A9
:10D3D000202831D00CD8062820D004D8042825D005
:10D3E000052844D118E007281DD008283FD11FE0A8
:10D3F000B0F5007F2BD005D840281FD0B0F5807F36
:10D4000035D11FE0B0F5803F2CD0B0F5003F2BD0D8
:10D41000B0F5806F2BD11FE0012201E04FF4807244
:10D42000134B9A6023E04FF48032F9E7082200E0C2
:10D4300010220F4BDA601AE0082200E010220C4B99
:10D440001A6114E00A4B9A6922F0010208E0084BC5
:10D450009A6922F0020203E0054B9A6922F0040265
:10D460009A6104E0082200E01022014B5A607047E4
:10D470000064004001420CBF00200120704700BF43
:10D48000202808B532D00CD8062821D004D804288A
:10D4900026D0052818D119E007281ED0082813D156
:10D4A00020E0B0F5007F29D005D8402820D0B0F585
:10D4B000807F09D120E0B0F5803F27D0B0F5003F54
:10D4C00022D0B0F5806F1BD0002024E0012101E0C4
:10D4D0004FF48071104B98681BE04FF48031F9E7EE
:10D4E000082100E010210C4BD86812E0082100E070
:10D4F0001021094B18690CE0012102E0022100E033
:10D500000421054B986904E0102100E00821024B3A
:10D510005868FFF7AFFF08BD00640040012108B55F
:10D520004FF0007000F0EEFF4FF00070002100F0AF
:10D53000E9FF08BD0268002322F0010202600360D7
:10D5400043608360C3602D4B984233D011D83C3B7D
:10D55000984229D006D8283B984221D014339842CB
:10D560004BD11FE0264B984220D01433984244D12F
:10D570001EE0244B98422CD008D8A3F5677398423C
:10D580001DD003F56273984237D11DE01E4B9842BF
:10D5900029D0143398422BD0283B98422DD11DE03E
:10D5A0001A4B12E0194B15E0184B18E0174B1BE013
:10D5B000164B1EE0154B5A6842F470021CE0134BE8
:10D5C0005A6842F0706217E0114B5A6842F00F023D
:10D5D00012E00F4B5A6842F0F0020DE00C4B5A6813
:10D5E00042F4706208E00A4B5A6842F4704203E069
:10D5F000074B5A6842F470225A6070476C00024030
:10D60000440002401C040240440402400000024066
:10D61000000402408A6870B50C6A0B6944EA020291
:10D620004C691A438B692243CC6905684E6A42EA09
:10D63000030323438C6A334325F4FE4C23432CF02D
:10D64000F00C43EA0C030360CB6843600B68836013
:10D650004B68C36070BD00BF0023836203604360FA
:10D660008360C360036143618361C361036243629A
:10D67000704700BF19B1036843F0010302E003687B
:10D6800023F001030360704712B10368194302E0FD
:10D69000036823EA01010160704700BF406880B25F
:10D6A000704700BF10F0805F14BF044B044B1B6831
:10D6B00003420CBF00200120704700BF000402405D
:10D6C0000000024010F0805F14BF024B024B586014
:10D6D000704700BF000402400000024010F0805F6D
:10D6E00014BF044B044B1B6803420CBF00200120F5
:10D6F000704700BF000402400000024010F0805F4D
:10D7000014BF024B024B5860704700BF0004024038
:10D7100000000240044B00221A605A609A60DA60EE
:10D72000024A5A61704700BF00040140FFFF070032
:10D73000837930B5016802794BB3184BCC431D682F
:10D7400090F805C004EA05051D605D682C405C602A
:10D75000D45844EA0101D15002689868D14301EAE3
:10D7600000009860D8680140BCF1100FD96007D163
:10D77000996811439960D96841EA0202DA600BE0C6
:10D780005CF8031041EA02024CF8032004E0034B6A
:10D79000D05820EA0101D15030BD00BF0004014043
:10D7A00000230C228371427103600371704700BF34
:10D7B000024B1A6940EA02021A61704700040140F4
:10D7C000034B5B6918420CBF00200120704700BF6B
:10D7D00000040140014B5861704700BF0004014044
:10D7E000054B1A685B69034001D1184603E01042FB
:10D7F0000CBF00200120704700040140014B58611C
:10D80000704700BF00040140044B1A6802F0380260
:10D810001A601A6840EA02021A607047002002404B
:10D82000044B1A6822F008021A601A6840EA0202E1
:10D830001A60704700200240044B1A6822F0100260
:10D840001A601A6840EA02021A607047002002401B
:10D85000034B044A5A6002F188325A60704700BF95
:10D860000020024023016745024B1A6942F0800202
:10D870001A61704700200240014BD8698008704748
:10D8800000200240014B186A704700BF0020024090
:10D89000024BD869C0F34000704700BF002002402F
:10D8A000024B1868C0F34010704700BF00200240D0
:10D8B00019B1054B1A69104303E0034B1A6922EAB8
:10D8C00000001861704700BF00200240012804D109
:10D8D000054BD86900F0010005E0034BDB681842F6
:10D8E0000CBF00200120704700200240014BD8608F
:10D8F000704700BF00200240094BDA6812F0010FA8
:10D9000001D001200BE0DA6812F0040F01D00220F0
:10D9100005E0DB6813F0100F14BF032004207047EC
:10D920000020024013B504460AE000230193FF33B0
:10D9300001E0019B013B0193019B002BF9D1013CCC
:10D94000FFF7DAFF012802D1002CEED100E004B984
:10D9500005201CBDF8B5124C124B0546A36003F11F
:10D9600088330F20A3600E461746FFF7DBFF04281D
:10D9700014D1236945F0F80543F0100323612E43C9
:10D98000094B37430B305F80FFF7CCFF012805D0F0
:10D99000226941F6EF7302EA03032361F8BD00BF79
:10D9A000002002402301674500F8FF1F38B50546F7
:10D9B00040F6FF70FFF7B6FF04283CD11E4C1F4B0A
:10D9C00040F6FF70A36003F18833A360236943F03E
:10D9D00020032361236943F040032361FFF7A2FF83
:10D9E000042820D1226941F6DF7302EA0303236190
:10D9F000236943F0100323611DB1114B4FF0000266
:10DA000002E00F4B4FF0A5021A8040F6FF70FFF7BF
:10DA100089FF01280FD0084A41F6EF73116901EA26
:10DA20000303136107E0012805D0226941F6DF7383
:10DA300002EA0303236138BD002002402301674549
:10DA400000F8FF1F10B504460F20FFF76BFF0428F6
:10DA50003DD11F4A1F4BE443936003F18833936029
:10DA60001169E3B241F01001FF2B116106D01A4A8F
:10DA70000B301381FFF756FF04281FD1C4F307238F
:10DA8000FF2B06D0144A0F205381FFF74BFF0428C9
:10DA900014D1C4F30743FF2B06D00F4A0F20938104
:10DAA000FFF740FF042809D1240EFF2C01D10420E8
:10DAB00006E0094B0F20DC81FFF734FF012806D078
:10DAC000034A41F6EF73116901EA0303136110BDC4
:10DAD000002002402301674500F8FF1F70B504468F
:10DAE0000F200E46FFF71EFF042815D10B4D0C4BDF
:10DAF0000B30AB6003F18833AB602B6943F010034C
:10DB00002B612680FFF70EFF012805D02A6941F618
:10DB1000EF7302EA03032B6170BD00BF00200240D7
:10DB20002301674570B504460F200E46FFF7FAFE45
:10DB3000042810D1084D0B302B6943F001032B61F1
:10DB40002680FFF7EFFE012805D02A6941F6FE7313
:10DB500002EA03032B6170BD0020024070B5044649
:10DB60000F200E46FFF7DEFE042818D10C4DB3B28D
:10DB70002A690B3042F001022A612380FFF7D2FEAE
:10DB8000042804D1360C66800B30FFF7CBFE012849
:10DB900005D02A6941F6FE7302EA03032B6170BDCA
:10DBA0000020024010B540F6FF70FFF7BBFE0428CE
:10DBB0002CD1174C174B40F6FF70A36003F188334C
:10DBC000A360236943F020032361236943F04003EA
:10DBD0002361FFF7A7FE042810D1226941F6DF7305
:10DBE00002EA0303236123694FF0A50243F0100307
:10DBF0002361094B0B301A80FFF794FE012805D0F2
:10DC0000226941F6EF7302EA0303236110BD00BFEE
:10DC1000002002402301674500F8FF1F10B540F6C1
:10DC2000FF70FFF77FFE042814D10B4C40F6FF7005
:10DC3000236943F004032361236943F04003236114
:10DC4000FFF770FE012805D0226941F6FB7302EA56
:10DC50000303236110BD00BF0020024038B5054614
:10DC600040F6FF70FFF75EFE042815D10B4C40F61E
:10DC7000FF70236943F0020323616561236943F068
:10DC800040032361FFF74EFE012805D0226941F6CB
:10DC9000FD7302EA0303236138BD00BF0020024088
:10DCA000CB78F0B513F0100F18BF8A78098803F00D
:10DCB0000F0C18BF4CEA020C11F0FF0F1AD00468C9
:10DCC00000220126964006EA0105B5420ED19600D3
:10DCD0000F27B7400CFA06F624EA07043443282B32
:10DCE00001D1456102E0482B08BF05610132082AD5
:10DCF000E7D10460FF291CD94468002202F108051D
:10DD00000126AE4006EA0105B5420ED196000F2766
:10DD1000B7400CFA06F624EA07043443282B01D155
:10DD2000456102E0482B08BF05610132082AE5D1B0
:10DD30004460F0BD0423C370022383704FF0FF33AF
:10DD400003807047836819420CBF00200120704790
:10DD5000806880B2704700BFC36819420CBF0020C2
:10DD600001207047C06880B2704700BF01617047F2
:10DD7000416170470AB1016100E04161704700BF35
:10DD8000C160704741F4803383618161836183693D
:10DD900083697047064A10B514684FF6807341EAEC
:10DDA000001104EA030341EA0303136010BD00BF3E
:10DDB00000000140014B1860704700BF1C0020426A
:10DDC0000304154A00F4401C1B0CBCF5401F30B581
:10DDD000546806D1556824F0706425F0706555606C
:10DDE00011E010F4801F06D0C0F303424FF0030C83
:10DDF0000CFA02F203E0420D120113FA02F224EAD5
:10DE0000020444F0706419B1400D000183401C43CA
:10DE1000014B5C6030BD00BF0000014001F0030316
:10DE20009B000F229A4010FA03F310B58908074CA3
:10DE3000023154F8210020EA020244F8212054F86B
:10DE40002120134344F8213010BD00BF00000140E1
:10DE50000120014608B500F047FB0120002100F039
:10DE600043FB08BD08B5264B98422BD00CD8A3F530
:10DE7000006398421AD003F5806398421CD0A3F542
:10DE8000006398423AD10BE01E4B984226D003F52E
:10DE90008063984228D0A3F5006398422ED117E002
:10DEA0000420012100F020FB042024E008200121AF
:10DEB00000F01AFB08201EE01020012100F014FBE6
:10DEC000102018E02020012100F00EFB202012E09D
:10DED0004020012100F008FB40200CE080200121BF
:10DEE00000F002FB802006E04FF48070012100F07A
:10DEF000FBFA4FF48070002100F0F6FA08BD00BF75
:10DF000000140140001C01400B4B4FF0FF316FF03B
:10DF10007042C3F88010C3F88420C3F88011C3F89E
:10DF20008421002303F1C001034A013300200F2B99
:10DF300042F82100F6D1704700E100E0094B4FF0B4
:10DF400020605860084800224FF0FF319A60D86086
:10DF50001A615A619A61DA611A625A629962D962E7
:10DF60001963704700ED00E00000FA0540F0BE6064
:10DF7000024B40F42020D860704700BF00ED00E065
:10DF800030B5C27803787AB31C4A4178D2684FF032
:10DF90000F0CD243C2F302222CFA02FCC2F104029B
:10DFA0009140807803F003020CEA000C4CEA010C6B
:10DFB000D2004FEA0C1CFF2090400CFA02FC012416
:10DFC00003F01F02944099080D4AC03152F82150C5
:10DFD0000CEA000C25EA00004CEA00005B0942F85C
:10DFE000210042F8234008E003F01F020121914084
:10DFF0005B09034A203342F8231030BD00ED00E0F6
:10E0000000E100E00023C370037043708370704729
:10E01000024B5868C0F30930704700BF00ED00E0C4
:10E02000012200F01F0312FA03F34009044A4030B2
:10E0300052F820001840984214BF00200120704779
:10E0400000E100E0014B1860704700BF00EF00E006
:10E0500000F01F0301229A404009024B603043F850
:10E060002020704700E100E0024B58688005800DD9
:10E07000704700BF00ED00E0012200F01F0312FA1C
:10E0800003F34009044A803052F8200018409842B7
:10E0900014BF00200120704700E100E0014B186828
:10E0A000704700BF00ED00E021F0604121F07F01EA
:10E0B000014B01439960704700ED00E0014A024BBB
:10E0C000DA6070470400FA0500ED00E0014A024BF7
:10E0D000DA6070470100FA0500ED00E019B1054B68
:10E0E0001A69104303E0034B1A6922EA0000186121
:10E0F000704700BF00ED00E000F01F00012313FA9D
:10E1000000F019B1044B5A6A104303E0024B5A6AFB
:10E1100022EA00005862704700ED00E0144B70B531
:10E12000DC684FF0FF0CE443C4F302242CFA04F53E
:10E13000C4F1040411FA04F4C0F30126F6000CFA49
:10E1400006FC02EA050545EA0404240114FA06F671
:10E15000C0F38110063053F8202022EA0C0243F865
:10E16000202053F82020164343F8206070BD00BFE4
:10E1700000ED00E0C0F3832001238340044A506A8D
:10E1800003EA0000984214BF00200120704700BF3E
:10E1900000ED00E000F01F0001228240024B5968B0
:10E1A0000A435A60704700BF00ED00E000F01F0214
:10E1B0000123013A13FA02F2024B59680A435A60EA
:10E1C000704700BF00ED00E0C0F3833001238340BF
:10E1D000044A506A03EA0000984214BF002001205C
:10E1E000704700BF00ED00E0C0F3814313B90A4B54
:10E1F000D86A10E0012B0CD1074AC0F30153906A92
:10E20000DA00D040022B14BF00F00F0000F0FF0036
:10E2100001E0014B186B704700ED00E010F4800F37
:10E220000BBF024B014B586B986B704700ED00E041
:10E2300008B5F5F79DFF08BD08B50001F5F795FF96
:10E2400008BD00BF08B5F5F78EFF08BD08B5F5F7A6
:10E2500088FF08BD08B5F5F782FF08BD08B5F5F7DA
:10E260007CFF08BD0D4B0E4A196841F00101196091
:10E27000596801EA02025A601A6822F0847222F494
:10E2800080321A601A6822F480221A605A6822F4D6
:10E29000FE025A6000229A60704700BF00100240E0
:10E2A0000000FFF80C4BB0F5803F1A6822F4803272
:10E2B0001A601A6822F480221A6003D0B0F5802F09
:10E2C00008D103E01A6842F4803202E01A6842F48E
:10E2D000A0221A60704700BF00100240034B1A686A
:10E2E00022F0F80242EAC0021A60704700100240B1
:10E2F000014B1860704700BF00004242044B5A684F
:10E3000022F47C1240EA02020A435A60704700BFBE
:10E3100000100240014B1860704700BF600042428D
:10E32000034B5A6822F0030240EA02025A60704727
:10E3300000100240024B586800F00C00704700BF0C
:10E3400000100240034B5A6822F0F00240EA020239
:10E350005A60704700100240034B5A6822F4E06292
:10E3600040EA02025A60704700100240034B5A68AC
:10E3700022F4605242EAC0025A6070470010024024
:10E3800019B1054B1A78104303E0034B1A7822EABF
:10E3900000001870704700BF09100240014B186060
:10E3A000704700BFD8004242034B5A6822F44042F3
:10E3B00040EA02025A60704700100240064B0022F9
:10E3C00001281A701A7002D0042804D101E01870D4
:10E3D00001E005221A70704720100240014B1860BE
:10E3E000704700BF80044242024B1A6A40EA0202B0
:10E3F0001A62704700100240014B1860704700BF5E
:10E400003C0442421F4B10B55A6802F00C02042A29
:10E4100013D0082A11D15A685968C2F383420232D4
:10E4200011F4803F03D05B6813F4003F01D0164B1A
:10E4300000E0164B5A43026001E0144B0360114A9E
:10E44000134B51680468C1F30311595C34FA01F1AC
:10E4500041605468C4F3022C13F80C4031FA04F400
:10E4600084605468C4F3C22C13F80CC021FA0CF178
:10E47000C1605268C2F381329B181B7CB1FBF3F17F
:10E48000016110BD0010024000093D0000127A0039
:10E49000E02D010819B1054B5A69104303E0034B05
:10E4A0005A6922EA00005861704700BF001002401C
:10E4B00019B1054B9A69104303E0034B9A6922EAAC
:10E4C00000009861704700BF0010024019B1054B71
:10E4D000DA69104303E0034BDA6922EA0000D861ED
:10E4E000704700BF0010024019B1054BDA681043B5
:10E4F00003E0034BDA6822EA0000D860704700BFEF
:10E500000010024019B1054B1A69104303E0034B98
:10E510001A6922EA00001861704700BF001002402B
:10E52000014B1860704700BF40044242014B186025
:10E53000704700BF4C004242014B1870704700BF4B
:10E54000071002404309012B02D1084B1B6805E06C
:10E55000022B0BBF054B054B1B6A5B6A00F01F00CB
:10E5600033FA00F000F00100704700BF00100240D5
:10E5700008B53120FFF7E6FF094B18705A680132E1
:10E580005A601A7822B95A6840F2FF139A42F0D1C1
:10E590003120FFF7D7FF003818BF012008BD00BFAA
:10E5A000D4060020024B5A6A42F080725A627047C9
:10E5B00000100240034B9B6818420CBF0020012052
:10E5C000704700BF00100240014B1870704700BF39
:10E5D0000A1002400B884A88B1F804C01A43CB885D
:10E5E00042EA0C02B1F808C01A434B8930B542EA3E
:10E5F0000C028D89B0F800C0CC891A432A4322430B
:10E600000CF4415313439BB20380838B23F40063C8
:10E610001B041B0C83830B8A038230BD00234FF045
:10E620000702C3810282038043808380C380038109
:10E6300043818381704700BF00234381038043806F
:10E640008380C3804FF002030381704721B10388A8
:10E650009BB243F0400304E0038823F040031B0413
:10E660001B0C0380704700BF21B1838B9BB243F426
:10E67000806304E0838B23F480631B041B0C83837F
:10E68000704700BF0909012313FA01F189B21AB1D9
:10E6900083889BB2194303E083889BB223EA01017C
:10E6A000818070471AB183889BB2194303E0838845
:10E6B0009BB223EA01018180704700BF81817047CE
:10E6C000808980B2704700BF4FF6FF63994205D042
:10E6D00003889BB243F48073038002E003881940EF
:10E6E0000180704721B183889BB243F0040304E0AA
:10E6F000838823F004031B041B0C8380704700BF36
:10E70000038823F400631B041B0C038003889BB263
:10E7100041EA03030380704703889BB243F48053AC
:10E720000380704721B103889BB243F4005304E097
:10E73000038823F400531B041B0C0380704700BFA5
:10E74000012914BF008B808A80B27047008A80B292
:10E75000704700BFB1F5804F04D103889BB243F4EA
:10E76000804304E0038823F480431B041B0C0380D4
:10E77000704700BF038919420CBF00200120704779
:10E78000202906D1038903889BB243F0400303800C
:10E7900008E0402901D0082901D1038902E0C943DA
:10E7A00089B20181704700BF012301F00F0213FA03
:10E7B00002F2B0F804C000891FFA8CFC80B210404D
:10E7C00006D009098B401CEA030F0CBF0020012072
:10E7D000704700BF552906D1038903889BB243F0D7
:10E7E000400303800DE0562901D0532901D103894C
:10E7F00007E001F00F01012313FA01F1C94389B2C7
:10E8000001817047838BF0B523F47A6323F01F03F3
:10E810001B041B0C83834FF0020303840B89868B3C
:10E82000022B87B004460D46B6B201D1002225E086
:10E8300001A88F88FFF7E6FDEB88002F0CBF0127AA
:10E840000227B3F5007F2989019A06D1A3F5FB734E
:10E8500053430902B3FBF1F305E00A2349015A438C
:10E860004F43B2FBF7F305330A229BB2B3FBF2F33B
:10E8700003F001021202C3F34F0392B2991E89B250
:10E88000FE2928BF002228BF0223E98842EA0303A9
:10E890000B439BB223842B886A8846EA0303A9882A
:10E8A00043F4006313436A890B4313439BB2A3836E
:10E8B00007B0F0BD08B5154B98421BD003F5744363
:10E8C000984204D0A3F5784398421DD10AE0012173
:10E8D0004FF48050FFF708FE4FF480500021FFF7FF
:10E8E00003FE11E04FF480400121FFF70BFE4FF4CF
:10E8F000804006E04FF400400121FFF703FE4FF493
:10E9000000400021FFF7FEFD08BD00BF003C0040B5
:10E91000042804D1054B1A6842F0040203E0034BBB
:10E920001A6822F004021A60704700BF10E000E08D
:10E93000014B5860704700BF10E000E0012804D18F
:10E94000084B1A6842F0010206E010F1020F05D1EF
:10E95000044B1A6822F001021A6002E0014B002207
:10E960009A60704710E000E020B1054B1A6842F051
:10E97000020203E0024B1A6822F002021A6070479A
:10E9800010E000E0014B9868704700BF10E000E025
:10E99000C308022B0BBF044B034B1B68DB6833FA25
:10E9A00000F000F00100704710E000E0038803F081
:10E9B0008F0303800388B1F806C04A889BB243EAFC
:10E9C0000C0313439BB203808B8883850B880385DC
:10E9D000064B984203D003F50063984201D10B7AAD
:10E9E00003864FF001038382704700BF002C014073
:10E9F000038C2DE9F04123F001031B041B0C03845D
:10EA0000038C0A894C8823F002031C4E14431B0418
:10EA10008288B1F806C0058B1B0CA4B2B04244EA50
:10EA2000030392B20C88ADB2A0F834C003D006F54F
:10EA30000066B04218D18E894F89B1F80E804FF62A
:10EA4000F77C03EA0C0C4CEA070748EA06064FF687
:10EA5000FB73898847F6FF4C02EA0C0C07EA0303B4
:10EA6000B2B20B4342EA0C024FF68F7105EA010184
:10EA70002143828001830384BDE8F081002C0140A2
:10EA8000038C2DE9F04123F010031B041B0C0384BD
:10EA9000028CB1F808C022F0200212048488120C03
:10EAA0004B8842EA0C1242EA0313A2B21B4C068BBB
:10EAB000B1F806C0A0420D88B6B29BB2A0F838C02B
:10EAC00003D004F50064A0421BD1B1F80A804FF6D0
:10EAD0007F748F8903EA040447F2FF3C02EA0C0CBE
:10EAE00044EA0814CA894FF6BF73898804EA03030D
:10EAF0004CEA870C43EA01134CEA82023C469BB283
:10EB000092B248F6FF7106EA010141EA052189B295
:10EB1000828001830384BDE8F08100BF002C0140A6
:10EB2000038C2DE9F04123F480731B041B0C038438
:10EB3000028CB1F808C022F4007212048488120C0E
:10EB40004B8842EA0C2242EA0323A2B21A4C868B7B
:10EB5000B1F806C0A0420D88B6B29BB2A0F83CC086
:10EB600003D004F50064A0421BD1B1F80A804FF233
:10EB7000FF748F8903EA040444F6FF7C02EA0C0C5C
:10EB800044EA0824CA894FF6FF33898804EA03035C
:10EB90004CEA071C43EA01234CEA02123C469BB2B2
:10EBA00092B24FF68F7106EA010129438280818378
:10EBB0000384BDE8F08100BF002C0140038CF0B558
:10EBC00023F480531B041B0C0384B1F806C0078C8C
:10EBD0000C8882880D89868B4B88A0F840C0DFF8AE
:10EBE00048C0BFB2604592B2B6B203D00CF5006C1B
:10EBF000604505D192048989920C42EA811292B251
:10EC00004DF6FF7C07EA0C0C48F6FF7106EA01019D
:10EC10004CEA053C41EA04214CEA033389B29BB239
:10EC2000828081830384F0BD002C0140B1F802C0D2
:10EC30000B888A884CEA0303B1F806C013430A899B
:10EC400043EA0C03B1F80AC013438A8943EA0C0370
:10EC500013439BB2A0F84430704700BF00234FF02D
:10EC6000FF320372438082800380C380704700BFFD
:10EC70000023C381038043808380C3800381438159
:10EC80008381704700234FF001020381038043809A
:10EC90008280C380704700BF00238381038043804C
:10ECA0008380C38003814381704700BF21B1038803
:10ECB0009BB243F0010304E0038823F001039B05AA
:10ECC0009B0D0380704700BF39B1B0F844306FEA44
:10ECD00043436FEA53439BB203E0B0F844305B0414
:10ECE0005B0CA0F8443070471AB183899BB219437A
:10ECF00003E083899BB223EA01018181704700BF51
:10ED0000818270470A43A0F8482070471AB183896E
:10ED10009BB2194303E083899BB223EA01018181FD
:10ED2000704700BF038923F007031B041B0C0381FA
:10ED3000704700BFB0F808C05FFA8CFC41EA0C0CC9
:10ED400042EA0C0C4CEA032C1FFA8CFCA0F808C019
:10ED5000704700BF10B50446FFF7ECFF23899BB254
:10ED600043F48043238110BD10B50446FFF7E2FF52
:10ED7000238923F077031B041B0C43F077032381C3
:10ED800010BD00BF01858282704700BF038823F059
:10ED900070039B059B0D41EA03030380704700BF8E
:10EDA000038923F070031B041B0C41EA0303038156
:10EDB000704700BF10B50446FFF7F2FF23899BB2EE
:10EDC00043F00703238110BD30B50489B0F818C0A3
:10EDD000058C2CF4407CADB22CF0030C24F007041D
:10EDE0004FEA0C4C25F0220542EA050524044FEABF
:10EDF0001C4C45EA0315240C4CF4807C21434CF058
:10EE0000010CADB20181A0F818C0058430BD00BF6F
:10EE1000038B23F070031B041B0C41EA03030383E1
:10EE2000704700BF038B23F4E0431B041B0C43EA31
:10EE300001239BB203837047838B23F070031B0471
:10EE40001B0C41EA03038383704700BF838B23F4C9
:10EE5000E0431B041B0C43EA01239BB283837047EE
:10EE600021B103889BB243F0800304E0038823F0C0
:10EE700080039B059B0D0380704700BF21B18388F1
:10EE80009BB243F0040304E0838823F004031B04D3
:10EE90001B0C8380704700BF21B183889BB243F075
:10EEA000080304E0838823F008031B041B0C838001
:10EEB000704700BF21B183889BB243F0010304E097
:10EEC000838823F001031B041B0C8380704700BF61
:10EED000038B23F008031B041B0C41EA0303038389
:10EEE000704700BF038B23F400631B041B0C43EA31
:10EEF00001239BB203837047838B23F008031B0419
:10EF00001B0C41EA03038383704700BF838B23F408
:10EF100000631B041B0C43EA01239BB283837047ED
:10EF2000038B23F004031B041B0C41EA030303833C
:10EF3000704700BF038B23F480631B041B0C43EA60
:10EF400001239BB203837047838B23F004031B04CC
:10EF50001B0C41EA03038383704700BF838B23F4B8
:10EF600080631B041B0C43EA01239BB2838370471D
:10EF7000038B23F080031B041B0C41EA0303038370
:10EF8000704700BF038B5B045B0C43EA01239BB219
:10EF900003837047838B23F080031B041B0C41EA1F
:10EFA00003038383704700BF838B5B045B0C43EADE
:10EFB00001239BB283837047038C23F002031B045D
:10EFC0001B0C41EA03030384704700BF038C23F04A
:10EFD00008031B041B0C41EA03030384704700BFB2
:10EFE000038C23F020031B041B0C43EA01139BB288
:10EFF00003847047038C23F080031B041B0C43EA3B
:10F0000001139BB203847047038C23F400731B0429
:10F010001B0C43EA01239BB203847047038C23F447
:10F0200000631B041B0C43EA01239BB2038470475B
:10F03000038C23F400531B041B0C43EA01339BB2E3
:10F040000384704701238B408A40018C89B221EAF6
:10F0500003030384018C0A4392B20284704700BF09
:10F0600004238B408A40018C89B221EA0303038484
:10F07000018C0A4392B20284704700BF01238B4087
:10F08000B0F820C010B51FFA8CFC2CEA03030384EF
:10F0900009B1082909D11830490844584FF68F732F
:10F0A00004EA0303435043580CE004391830C1F319
:10F0B0004E01445848F6FF7304EA0303435012021A
:10F0C000435892B243EA0202425010BD21B1038874
:10F0D0009BB243F0020304E0038823F002039B0584
:10F0E0009B0D0380704700BF21B103889BB243F0A2
:10F0F000040304E0038823F004039B059B0D0380B5
:10F10000704700BF21B183889BB243F0800304E0C5
:10F11000838823F080031B041B0C8380704700BF8F
:10F12000038823F008039B059B0D038003889BB293
:10F1300041EA030303807047838823F070031B04B4
:10F140001B0C838083889BB241EA03038380704752
:10F15000038923F007031B041B0C038103899BB263
:10F1600041EA030303817047038923F080031B04F2
:10F170001B0C038103899BB241EA0303038170479F
:10F180008184704781857047818670470187704709
:10F1900081877047A0F84010704700BF038B23F0B1
:10F1A0000C031B041B0C0383038B9BB241EA030378
:10F1B00003837047038B23F440631B041B0C0383FE
:10F1C000038B9BB243EA01239BB20383704700BFCA
:10F1D000838B23F00C031B041B0C8383838B9BB258
:10F1E00041EA030383837047838B23F440631B044A
:10F1F0001B0C8383838B9BB243EA01239BB28383E3
:10F20000704700BF0388DBB2038003889BB241EAEA
:10F2100003030380704700BF808E80B2704700BF39
:10F22000008F80B2704700BF808F80B2704700BFF0
:10F23000B0F8400080B27047808C80B2704700BF49
:10F24000008D80B2704700BF038A19420CBF0020B6
:10F2500001207047C94389B201827047038A8289BD
:10F2600011EA030092B203D011420CBF002001202A
:10F27000704700BFC94389B201827047B0F820C00F
:10F2800010B52CF0010C4FEA0C4C4FEA1C4CA0F8C6
:10F2900020C0048BB0F820C0A4B21FFA8CFC24F06C
:10F2A000F30442EA04042CF0020C44EA03144CF088
:10F2B000010C4CEA010CA4B20483A0F820C010BDDC
:10F2C000B0F820C010B52CF0100C4FEA0C4C4FEAEF
:10F2D0001C4CA0F820C0B0F818C0048C2CF4407C62
:10F2E000A4B24FEA0C5C4FEA1C5C24F020044CEA08
:10F2F000022C44F010044CEA033C44EA01141FFAC7
:10F300008CFCA4B2A0F818C0048410BD38B50D461A
:10F31000602D1146044603D10122FFF7D1FF02E020
:10F320000122FFF7ABFF29462046FFF739FD23896D
:10F330009BB243F00703238138BD00BFF8B50C46EC
:10F34000A2884988B4F800C0054600290CBF0227EE
:10F350000027012A0CBF022601262389BCF1000FD9
:10F3600010D1FFF78BFF2846E188FFF717FF2846EB
:10F37000394632462389FFF7A3FF2846E188FFF785
:10F3800019FF0FE0FFF79CFF2846E188FFF712FF07
:10F390002846394632462389FFF770FF2846E18820
:10F3A000FFF7FCFEF8BD00BF38B50B880C460546DC
:10F3B0004BB94988A2882389FFF760FF2846E18876
:10F3C000FFF7ECFE53E0042B09D14988A28823897A
:10F3D000FFF776FF2846E188FFF7ECFE47E0082BB1
:10F3E000B1F802C0B1F804E0098920D1028C22F4FE
:10F3F00080721204120C0284838B028C9BB292B234
:10F4000023F0F30322F4007243EA011142EA0C2CC8
:10F4100089B21FFA8CFC41EA0E0E4CF4807CA0F8F5
:10F420001CE0A0F820C0E188FFF7D2FE1FE0028CAC
:10F4300022F480521204120C0284838B028C23F477
:10F44000407392B21B051B0D22F4005243EA0E23B7
:10F4500042EA0C3C43EA01331FFA8CFC9BB24CF4A9
:10F46000805C8383A0F820C0E188FFF7BDFE38BD33
:10F4700008B52D4B984237D00BD8A3F500639842BE
:10F4800026D003F58063984228D0B0F1804F4AD14E
:10F4900018E0264B984233D004D8A3F580639842F5
:10F4A00041D127E0224B984204D003F500639842F3
:10F4B00039D12EE04FF400600121FFF715F84FF429
:10F4C00000602DE001200146FFF71CF801201CE040
:10F4D00002200121FFF716F8022016E00420012186
:10F4E000FFF710F8042010E008200121FFF70AF8C8
:10F4F00008200AE010200121FFF704F8102004E0A2
:10F5000020200121FEF7FEFF20200021FEF7FAFF58
:10F5100009E04FF400500121FEF7E6FF4FF40050E0
:10F520000021FEF7E1FF08BD000C00400014004080
:10F53000002C0140002383814FF416528380C38046
:10F5400003814FF00C030260438170470A8810B5B5
:10F550004C88B1F804C0038AC98844EA020242EA2E
:10F560000C0223F470630A431B041B0C92B242EAA0
:10F570000303038210BD00BF0023C38003804380C8
:10F580008380704721B183899BB243F4005304E028
:10F59000838923F400531B041B0C8381704700BF35
:10F5A00001F01F034FF0010CC1F3421161450CFA49
:10F5B00003F301D10C3004E0022901D1103000E046
:10F5C00014301AB1026842EA030302E0026822EA38
:10F5D00003030360704700BF1AB1838A9BB21943CB
:10F5E00003E0838A9BB223EA01018182704700BF56
:10F5F000038A23F00F031B041B0C0382038A9BB2B4
:10F6000041EA030303827047838923F400631B04E8
:10F610001B0C838183899BB241EA0303838170477A
:10F6200021B183899BB243F0020304E0838923F074
:10F6300002031B041B0C8381704700BF038A23F065
:10F6400020031B041B0C0382038A9BB241EA0303C1
:10F650000382704721B1038A9BB243F4804304E0E4
:10F66000038A23F480431B041B0C0382704700BFF2
:10F67000C905C90D818070478088C005C00D7047DD
:10F6800083899BB243F0010383817047038BDBB214
:10F690000383038B9BB243EA01230383704700BFBC
:10F6A000038B03F47F430383038B9BB241EA030381
:10F6B0000383704721B1838A9BB243F0200304E0A7
:10F6C000838A23F020031B041B0C8382704700BF36
:10F6D00021B1838A9BB243F0100304E0838A23F0B4
:10F6E00010031B041B0C8382704700BF21B1838A67
:10F6F0009BB243F0080304E0838A23F008031B0451
:10F700001B0C8382704700BF838A23F004031B0411
:10F710001B0C8382838A9BB241EA03038382704776
:10F7200021B1838A9BB243F0020304E0838A23F071
:10F7300002031B041B0C8382704700BF038819421D
:10F740000CBF002001207047C94389B20180704777
:10F750004FF0010CC1F3421201F01F0362450CFA95
:10F7600003F301D1828903E0022A0CBF028A828A54
:10F7700092B21340028892B20BB9184607E0090A08
:10F78000012313FA01F111420CBF00200120704740
:10F79000090A01238B40DB439BB20380704700BF03
:10F7A000038ACA8823F440531B041B0C13430382AF
:10F7B00083898A8830B5044608890D4623F4B053FE
:10F7C000498940EA020223F00C030A431B041B0C84
:10F7D00092B242EA0303A381A38AAA8923F4407365
:10F7E0001B041B0C134387B0A38201A8FEF70AFE7B
:10F7F0000E4B2A689C420CBF049B039B1921594362
:10F8000092006423B1FBF2F1B1FBF3F21201100993
:10F8100003FB101109013231B1FBF3F303F00F03C5
:10F8200043EA020292B2228107B030BD00380140A3
:10F8300008B5214B98422BD008D8A3F50063984215
:10F8400016D003F58063984234D119E01B4B9842DF
:10F8500026D003F5684398422CD101214FF4804013
:10F86000FEF742FE4FF480400021FEF73DFE21E00E
:10F870004FF400300121FEF745FE4FF4003016E052
:10F880004FF480200121FEF73DFE4FF480200EE072
:10F890004FF400200121FEF735FE4FF4002006E072
:10F8A0004FF480100121FEF72DFE4FF4801000214F
:10F8B000FEF728FE08BD00BF004C0040005000408D
:10F8C000684620F007018D4601B5002303E00B498F
:10F8D0005958995004330A4A0A4998188842F6D36D
:10F8E000094B02E0002243F8042B084A9342F9D363
:10F8F000F4F772FCBDE8014085467047382F0108D7
:10F90000000000203002002030020020B80E00204D
:10F9100010B5074C20B922684FF00103138205E0AF
:10F92000044B1B681B68984720680A3010BD00BF55
:10F93000500E00200C0E002010B50A4B0A4A1B681E
:10F940005178DA7891420AD3997841B99C8834B9D0
:10F950009A72064B1B685B689847204600E00220BD
:10F9600010BD00BF500E0020040100200C0E00202E
:10F9700010B5074C20B922684FF00103138205E04F
:10F98000044B1B689B68984720680C3010BD00BF73
:10F99000500E00200C0E002038B50E4C0E4B226885
:10F9A0001B68D1789B695079984723689A7A7AB115
:10F9B00070B91A7962B99D7855B9084B1B68DB6834
:10F9C0009847236828465979DA78D9721A7300E083
:10F9D000022038BD500E0020E80D00200C0E002043
:10F9E00008B50246244B20B91B684FF0020119826A
:10F9F00040E0224A4FF000011B681180197811F095
:10FA00007F0113D15B7A13F0200F03D0117841F0FE
:10FA10000201117013F0400F184B15BF1A781A78B5
:10FA200022F0010242F001021A701EE0012921D0E9
:10FA3000022901D000221DE0597911F0800F01F058
:10FA40000F0306D00E4951F8233003F03003102B7A
:10FA500006E00B4951F8233003F44053B3F5805FBF
:10FA600003D1137843F001031370064B1B681B6925
:10FA70009847024A104608BD500E0020B00E0020E4
:10FA8000005C00400C0E002010B51E4B19684A792E
:10FA900012F0800F22F0800305D01B4850F823009D
:10FAA00000F0300004E0184850F8230000F4405003
:10FAB000164C94F800C0634522D24C8804BBF8B1C0
:10FAC000897AE9B112F0800F09D00F4948F6BF7268
:10FAD00051F8230000EA020282F0100208E00A490D
:10FAE0004BF68F7251F8230000EA020282F4805232
:10FAF00041F82320064B1B689B699847002000E0D3
:10FB0000022010BD500E0020005C004004010020C7
:10FB10000C0E002008B5064B1B685A7A42F02002F2
:10FB20005A72044B1B68DB699847002008BD00BF70
:10FB3000500E00200C0E0020054B1A68538A18B98D
:10FB40008988CB1A138201E008681818704700BF33
:10FB5000500E002030B50E4B1C78002310E05FFAE9
:10FB600083FC4FEA8C0202F1804202F5B84215682C
:10FB700048F68F7105EA010141EA0C011160013379
:10FB8000A342ECD3034B40F08000186030BD00BFAF
:10FB9000040100204C5C0040704700BF08B50C4BCE
:10FBA000002093F82C1000F04FFE0A4B1B68187AC7
:10FBB000082807D1084B4FF480521A80074B4FF0AA
:10FBC00010021A80092814BF0020012008BD00BFC0
:10FBD00080000020500E0020B20E0020B40E002045
:10FBE00070B52D4B1C68237A032B01D0052B46D111
:10FBF000A369228AABB1A2B1A58A954228BF154656
:10FC000028469847228A638A521BEB1806462282AE
:10FC10006382002000F0E8FD2A460146304600F0ED
:10FC2000FBFB238A5BB11D4B4FF4405200201A802E
:10FC3000014600F0E7FD1A4B4FF030021A80A28A0D
:10FC4000238A9A4203D8144B03221B6803E0124A0A
:10FC50001BB1136805221A720DE012680621117299
:10FC6000104A1168104A89B28A18520013600C4B6E
:10FC70004FF030021A80084B1B681B7A06E0072BF6
:10FC800003D10A4B1B68DB6898470823024A1268B5
:10FC90001372FFF783FF70BD500E0020B20E0020DC
:10FCA000B40E0020505C004002300020E80D00201F
:10FCB000F8B5244B1C68238A267ABBB9042E15D1CB
:10FCC000214822490278012A0BD1214C214A24687B
:10FCD0000370A0B28218520013604FF030020A8005
:10FCE0002BE04FF010030B80072626E0A68AA269BE
:10FCF0009E4234BF35461D462846B34294BF042673
:10FD0000022690470746002000F060FD2A46014683
:10FD1000384600F069FB2946002000F073FD638A35
:10FD2000228AEB186382094B551B4FF03002258263
:10FD30001A80094B4FF440521A80024B1B681E7206
:10FD4000F8BD00BF500E0020DC060020B40E0020DD
:10FD5000505C004002300020B20E002008B5144B69
:10FD60001B681A7A022A01D0042A05D1FFF7A0FFE6
:10FD70000F4B1B681B7A14E0062A11D15A78052A0A
:10FD80000AD11A7812F07F0F06D1D878FFF7E2FE79
:10FD9000084B1B681B6A9847074B1B689B68984772
:10FDA0000823034A12681372FFF7F8FE08BD00BF6C
:10FDB000500E00200C0E0020E80D002038B5324B0C
:10FDC0001B68187810F07F0004D15A7A22F02002C4
:10FDD0005A7258E0022855D15A88002A52D11A790D
:10FDE000002A4FD15A7912F0800F22F0800405D0FA
:10FDF000264951F8241001F0300104E0234951F85C
:10FE0000241001F440512248007884423AD200295B
:10FE100038D09B7A002B35D012F0800F0FD01B4BBF
:10FE200053F8243003F03003102B25D1E4B22046E0
:10FE300000F082FC2046302100F05EFB1CE0134DF8
:10FE400055F8243003F44053B3F5805F14D134B92E
:10FE5000104B204693F82C1000F0F6FC02E02046F0
:10FE600000F056FC55F824204BF68F7302EA03038A
:10FE700083F4405345F82430074B1B685B6998476F
:10FE8000002000E0022038BD500E0020005C004041
:10FE900004010020800000200C0E0020F7B58D4BDF
:10FEA0008D4E1A6835688D4B92B2D3182A7A5B0052
:10FEB000092A1B681BD09BB203F1005303F5405382
:10FEC0005B001C4614F8012B03F10A072A705B78CB
:10FED0006B70B4F8030000F063FE6880B4F80700AC
:10FEE000346800F05DFEA08033687F88DF807A4C44
:10FEF00001212368DA8819725D78002A62D11A78A4
:10FF000012F07F022ED1092D02D1FFF715FD3BE043
:10FF1000052D0DD193F90320002A4EDB9A78002A93
:10FF20004BD19A88002A48D19B7A002B37D044E0E5
:10FF3000032D0BD1DA78012A27D19A882ABB5B7A64
:10FF400013F0200F21D0FFF7E5FD1DE0012D1CD19E
:10FF5000DA78012A19D19A88BAB95B7A13F0200F9E
:10FF600013D00AE0012A04D10B2D0ED1FFF714FDA6
:10FF70000AE0022A09D1012D02D1FFF71FFF03E099
:10FF8000032D02D1FFF780FD48B1554B28461B6871
:10FF90005B699847032801D109230FE068B94D4AEE
:10FFA000504B12684FF0300192B2D3185B00002220
:10FFB0001A604D4B1980062300E00823464A126858
:10FFC0001372E3E0062D18D11A7812F07F0F40F07B
:10FFD00097809B78012B03D1414B1B68DB696EE056
:10FFE000022B03D13E4B1B681B6A68E0032B40F0D9
:10FFF00087803B4B1B685B6A61E0002D3CD15988D0
:020000040801F1
:1000000000297DD15A6822F47F42B2F5003F77D1B2
:100010001A7812F07F0203D19B88002B70D129E05F
:10002000012A0BD158792E4B1B689B6998470028F1
:1000300066D123689B7A002B62D01BE0022A5FD135
:100040005B7913F0800F03F00F0205D0274951F8B8
:10005000221001F0300104E0244951F8221001F48B
:1000600040512348007882424AD213F0700F47D1A2
:10007000002945D01F4B23E0082D05D11B7813F034
:100080007F0F3DD11C4B1BE00A2D39D11A7802F0AD
:100090007F02012A34D19A7A002A31D05988002966
:1000A0002ED15A6822F47F42B2F5803F28D1587988
:1000B0000B4B1B689B69984710BB104B00E0FBB1D2
:1000C000054A4FF000011268002093615182984761
:1000D000002020E0505C0040500E00200430002042
:1000E000E80D002002300020B40E0020005C00402B
:1000F00004010020E1F9000811F9000871F9000875
:10010000244C254B22681B6850781B6998470328AC
:1001100001D1236806E01F4B4FF6FF711B681A8A56
:100120008A4201D1092203E0022800D012B9082234
:100130001A722BE093F90010002921DAD988019175
:100140000198824202D9019A1A8211E08A420FD2A2
:100150001149096891F82C108A4201D2002105E06A
:1001600092FBF1F001FB102212B901210B4A117030
:10017000094A126892F82C209A82FFF799FD05E04F
:1001800003221A72064B4FF440521A80FFF706FD05
:10019000FEBD00BF500E0020E80D0020DC06002050
:1001A000B20E0020074A022108B50748117207491C
:1001B000074B086007490A60074A13601B689847A5
:1001C00008BD00BFF00D0020080100200C0E00202B
:1001D00080000020500E0020E80D002008B529E026
:1001E00047F6FF700860198801F00F018B0003F1DA
:1001F0008043117003F5B843196889B211F4004FB8
:1002000009D0186840F68F7100EA01011960127870
:100210000E4B013A0BE011F0800F0BD0186848F636
:100220000F7100EA010119601278094B013A53F885
:10023000223098470749084B0868084A80B218805E
:10024000188800B20028CBDB08BD00BFE800002002
:10025000CC000020445C0040E60D0020EC0D0020A6
:10026000F8B59AE047F6FF761E601688564F06F0FE
:100270000F06B30003F1804303F5B8433E70002E30
:1002800064D127682668236807F4405C03EA00000D
:1002900080F400502060236806F0300003EA01017A
:1002A00081F0200121601388484A13F0100F10805C
:1002B000A5F800C004D023689BB213F0800F08D0CB
:1002C000226848F60F7302EA03032360FFF746FD36
:1002D00016E013F4006F08D0226840F68F7302EA2C
:1002E00003032360FFF7DAFD0AE013F4004F54D054
:1002F000226840F68F7302EA03032360FFF770FC65
:1003000021682A884BF68F7301EA030312F4805F99
:1003100018BF83F4805312F4005F2D4A18BF83F492
:1003200000531360294B11681A8848F6BF7301EA1D
:10033000030312F0100F18BF83F0100312F0200F08
:10034000234A18BF83F0200313603BE01C68A4B26B
:1003500014F4004F0BD0196840F68F7201EA0202C4
:100360001A603A781B4B013A53F82230984714F040
:10037000800F12D0144948F60F720B789B0003F1DE
:10038000804303F5B843186800EA02021A600A784D
:10039000114B013A53F822309847104B104A1D6810
:1003A0000B4C1FFA85FCA2F800C0B2F800C04BF657
:1003B0008F700FFA8CFCBCF1000F48F6BF71094D2D
:1003C000FFF650AFF8BD00BFEC0D0020B40E0020CA
:1003D000005C0040E8000020CC000020445C0040AD
:1003E000E60D0020B20E002001F10051013201F5AE
:1003F000405110B549005208002308E010F803C02E
:100400006478013A4CEA042C21F813C00233C41872
:10041000002AF3D110BD00BF01F10051013201F5F6
:10042000405110B549005208002304E031F8134050
:10043000013AC4520233002AF8D110BD014B1860B2
:10044000704700BF405C0040014B186880B27047A5
:10045000405C0040014B1860704700BF445C0040A6
:10046000014B186880B27047445C0040014B18682B
:1004700080B27047485C0040014B1860704700BF75
:100480004C5C0040014B186880B270474C5C0040E7
:100490004FF6F873024A00EA03031360704700BF87
:1004A000505C0040014B186880B27047505C0040BF
:1004B000014B43F820107047005C0040024B53F89A
:1004C000200080B2704700BF005C0040054B10B5B3
:1004D00053F8204048F68F1204EA02020A4343F818
:1004E000202010BD005C0040024B53F8200000F4B7
:1004F000C0607047005C00400A4B10B553F82020E4
:1005000048F6BF7402EA040411F0100F18BF84F01B
:10051000100411F0200F18BF84F0200443F820408D
:1005200010BD00BF005C00400A4B10B553F82020FE
:100530004BF68F7402EA040411F4805F18BF84F450
:10054000805411F4005F18BF84F4005443F8204035
:1005500010BD00BF005C004038B50D460446FFF7F3
:10056000ADFF012D02D120F4805003E0022D04D113
:1005700020F01000014B43F8240038BD005C00401F
:10058000024B53F8200000F030007047005C004040
:10059000024B53F8200000F440507047005C0040CC
:1005A000054B48F6BF7253F8201001EA020282F0B0
:1005B000300243F820207047005C0040054B4BF6AA
:1005C0008F7253F8201001EA020282F4405243F87D
:1005D00020207047005C0040054B48F68F6253F8BE
:1005E000201001EA020242F4807243F82020704792
:1005F000005C0040044B48F68F6253F8201001EA7B
:10060000020243F820207047005C0040044B48F68B
:100610008F6253F8201001EA020243F8202070474D
:10062000005C0040054B48F68F6253F8201001EA49
:10063000020242F4807243F820207047005C0040C0
:10064000054B48F68F6253F8201001EA020242F48B
:10065000807243F820207047005C0040044B48F64D
:100660008F6253F8201001EA020243F820207047FD
:10067000005C0040044B53F8200000F030001028CC
:1006800014BF002001207047005C0040054B53F868
:10069000200000F44050B0F5805F14BF002001201E
:1006A000704700BF005C0040044B40F68F7253F867
:1006B000201001EA020243F820207047005C00404D
:1006C000044B48F60F7253F8201001EA020243F877
:1006D00020207047005C0040054B48F68F7253F8AD
:1006E000201001EA020242F4804243F820207047C1
:1006F000005C0040054B48F68F7253F8201001EA69
:10070000020242F0400243F820207047005C0040A3
:10071000084B53F8202012F4804F09D053F82010D2
:1007200048F68F7201EA020242F4804243F8202028
:10073000704700BF005C0040084B53F8202012F0C7
:10074000400F09D053F8201048F68F7201EA0202D8
:1007500042F0400243F82020704700BF005C004098
:10076000054B10B553F8204048F68F7204EA020298
:100770000A4343F8202010BD005C0040024B53F8B0
:10078000200000F00F007047005C0040064B490855
:100790001B6849009BB203EBC00303F1005303F550
:1007A00040535B0019607047505C0040054A064B9F
:1007B0001268490892B202EBC002D3185B004900EC
:1007C00019607047505C004004300020054B1B68E6
:1007D0009BB203EBC00303F1005303F540535B00EE
:1007E00018887047505C0040044A054B126892B26A
:1007F00002EBC002D3185B0018887047505C0040C1
:1008000004300020044A054B126892B202EBC00289
:10081000D3185B0019607047505C00400230002024
:100820003E2909D94B0911F01F0F01D1013B9BB2A1
:100830009B0243F4004305E04B0811F0010F18BF81
:1008400001339B02036070470D4A0E4B126892B24F
:10085000D31803EBC0035B003E2909D94A0911F004
:100860001F0F01D1013A92B2920242F4004205E018
:100870004A0811F0010F18BF013292021A60704746
:10088000505C004006300020054A064B126892B2C8
:1008900002EBC002D3185B0018688005800D70471A
:1008A000505C004002300020054A064B126892B2AC
:1008B00002EBC002D3185B0018688005800D7047FA
:1008C000505C0040063000200C4B30B51D681C68A1
:1008D000C0001FFA85FC8444A4B2094B00190CF136
:1008E000005CC3180CF5405C490852084FEA4C0004
:1008F00049005B00520001601A6030BD505C00404E
:1009000004300020064B49081B6849009BB203EBEA
:10091000C00303F1005303F540535B0019607047B7
:10092000505C0040054A064B1268490892B202EB3F
:10093000C002D3185B00490019607047505C00404A
:1009400004300020054B1B689BB203EBC00303F18E
:10095000005303F540535B0018887047505C00401B
:10096000044A054B126892B202EBC002D3185B0036
:1009700018887047505C004004300020012910B5F1
:1009800024D1254B25491B68C0009BB25918091872
:100990004B003E2A09D9510912F01F0F01D101392C
:1009A00089B2890241F4004105E0510812F0010FBB
:1009B00018BF0131890219601749194B096889B2BA
:1009C000CB18181840003E2A1ED913E0022922D164
:1009D000114BC0001C681B68A4B21FFA83FC0F49AE
:1009E0000F4B844400194118634449005B000A60BE
:1009F0001A6010E0530912F01F0F01D1013B9BB2A6
:100A00009B0243F4004305E0530812F0010F18BFA6
:100A100001339B02036010BD505C00400230002097
:100A20000630002001291BD11349144B096889B2F3
:100A3000CB1803EBC00040003E2A09D9530912F03D
:100A40001F0F01D1013B9BB29B0243F4004305E021
:100A5000530812F0010F18BF01339B0203600AE034
:100A6000022908D10449054B096889B201EBC0008D
:100A7000C3185B001A607047505C004002300020D1
:100A800001291BD11349144B096889B2CB1803EB18
:100A9000C00040003E2A09D9530912F01F0F01D1AE
:100AA000013B9BB29B0243F4004305E0530812F064
:100AB000010F18BF01339B0203600AE0022908D12D
:100AC0000449054B096889B201EBC000C3185B00FB
:100AD0001A607047505C004006300020054A064B03
:100AE000126892B202EBC002D3185B00186880054E
:100AF000800D7047505C004002300020054A064BD4
:100B0000126892B202EBC002D3185B00186880052D
:100B1000800D7047505C0040063000200D4BC00037
:100B200019680D4A89B241188A185200128812F4C5
:100B30007C4F01D001200CE01A68084B92B280185B
:100B4000C3185B0018888005800D002814BF0220A0
:100B500000207047505C004006300020023000202A
:100B6000012909D10B4A48F68F7352F8201001EA87
:100B7000030343F040030AE002290AD1054A48F67C
:100B80008F7352F8201001EA030343F4804342F8C4
:100B900020307047005C004041EA0020704700BFF1
:100BA000030AC0B243EA0020704700BF08B5002224
:100BB0000A2300F045F808BD08B500210A2200F01C
:100BC000DFF808BDF0B40378002B2DD040F23412CA
:100BD000C2F20002156802E010F8013FEBB15A19A9
:100BE00003F12004527812F001070A7808BF1C466E
:100BF00001F10101561C9446AE5D16F0010F18BFBD
:100C000002F1200C6445E7D007B1203316F0010F44
:100C100018BF2032981AF0BC70470A786F78561CBB
:100C200007F00107AE5DEFE740F234100A78C2F238
:100C30000000561C05686F78AE5D07F00107E3E71A
:100C40002DE9F04F40F23415C2F2000583B00C4696
:100C50001F46D5F800800E460190009216F8015B01
:100C600008EB050393F801B01BF0080BF6D12D2D0E
:100C700065D02B2D08BF16F8015BD7F1010338BFF3
:100C80000023102F14BF1A4643F0010232B1302D59
:100C900066D01BB1302D0CBF08270A27BBF1000F0F
:100CA000394614BF4FF000496FF00049484600F044
:100CB00059FC48468A46394600F026FB00218C46FE
:100CC00008EB0502A5F13003527812F0040F08D1A9
:100CD00012F0030F20D012F0010F14BF3723572357
:100CE000EB1A9F4218DD844594BF0022012252EA8C
:100CF000D1714FF0FF310CD1844514BF0022012285
:100D00005345D4BF002202F0010212B907FB0C3C8C
:100D1000012116F8015BD3E7B1F1FF3F14D0BBF11D
:100D2000000F09D16046009B1BB101B1741E009AEF
:100D3000146003B0BDE8F08FCCF10000F3E716F8C3
:100D4000015B4FF0010B98E7019ABBF1000F4FF0E8
:100D5000220314BF4FF000406FF000401360E2E741
:100D60003278782A14BF00210121582A14BF0A467C
:100D700041F00102002A8CD07578102702368DE7E9
:100D800010B540F23814C2F200048C4613460146F6
:100D900062462068FFF754FF10BD00BF2DE9F04305
:100DA0008BB006460F4600F07BF840F22C24C2F2CE
:100DB000000494F90030B3F1FF3F8046894638D0F3
:100DC0003046394600F084FA0546002831D13046D5
:100DD00039460022002301F01DF8002829D124788B
:100DE00042F62873C0F6010308950193CDE9026726
:100DF000CDE90467002C21D040F200030022CFF699
:100E0000F0733046CDE9062339460022002300F076
:100E1000D9FF002822D0022300939C4234D0684698
:100E200000F064FA00282FD0089B002B27D1DDE9C1
:100E30000689404649460BB0BDE8F0834FF6FF7384
:100E40004FF06042CCF2EF733046CDE906233946CD
:100E50000022002300F0B6FF0028DCD10123022C81
:100E6000009316D0684600F041FA90B142F62C701B
:100E7000C0F6010000F03CFACDE90601D4E700F02D
:100E80003DFA089B0360D2E700F038FA22230360A2
:100E9000CAE700F033FA21230360E7E7000000000F
:100EA000B1F5801F0B462DE9F04F804687B089468B
:100EB00004460D463EDB4FF6FF720026C7F6EF7282
:100EC000934251DC23F07F4445F6647C24F47004A3
:100ED000C0F2090CA44440F20002A6F57E760CF4A0
:100EE000801C073EC3F6F0728CEA020206EB235622
:100EF00040F20003404642EA0401C3F6F0730022C8
:100F000006EB1C5600F042FBA31C23F07F4323F4A6
:100F10007003022B804689462FDC0022002300F05C
:100F200051FF002800F0CA80002E40F07C81002094
:100F300000211FE021F00043034300F0B5800029A9
:100F4000C0F2468140F200030022C4F250336FF039
:100F5000350600F0CFFC4FF6FF72C7F6EF720B4676
:100F6000804693428946ADDD4046494642464B465F
:100F700000F00EFB07B0BDE8F08F00224FF0804379
:100F800000F006FB4EF68635CFF6F9756519024678
:100F90000B464046494600F0D7FDCDE902013046F8
:100FA00000F042FCCDE90401DDE9020102460B46F6
:100FB00000F0A0FC02460B46CDE9000100F09AFCCF
:100FC000A7A3D3E9002382468B4600F093FCA6A397
:100FD000D3E9002300F0DCFA52465B4600F08AFCBD
:100FE000A3A3D3E9002300F0D3FA52465B4600F0F6
:100FF00081FCA1A3D3E9002300F0CAFADDE90023B4
:1010000000F078FC9EA3D3E90023CDE9000150460F
:10101000594600F06FFC9CA3D3E9002300F0B8FA16
:1010200052465B4600F066FC99A3D3E9002300F02A
:10103000AFFA52465B4600F05DFC0B460246DDE926
:10104000000100F0A5FA4BF65103C0F206031B1B8A
:1010500043EA0505002D82468B4656DD40F200032B
:101060000022C3F6E0734046494600F043FC424686
:101070004B4600F03FFC04460D46002E75D152460B
:101080005B4600F085FADDE9022300F033FC0246FE
:101090000B462046294600F079FA02460B464046A8
:1010A000494600F073FA65E740F200010020002293
:1010B0000023CCF2503100F047FD5BE742464B463F
:1010C0004046494600F016FC73A3D3E900230446CA
:1010D0000D464046494600F00DFC40F20003002258
:1010E000C3F6E07300F054FA02460B462046294648
:1010F00000F000FC04460D46002E72D140464946E1
:1011000022462B4600F042FA34E7002E00F0D4804D
:1011100063A3D3E90023DDE9040100F0EBFB5246B1
:101120005B4606460F464046494600F02FFADDE989
:10113000022300F0DFFB5CA3D3E9002304460D4645
:10114000DDE9040100F0D6FB02460B4620462946A5
:1011500000F01EFA42464B4600F018FA02460B46D3
:101160003046394600F012FA04E74DA3D3E90023D4
:10117000DDE9040100F0BEFB52465B46CDE900010B
:101180002046294600F004FADDE9022300F0B2FB14
:1011900047A3D3E9002306460F46DDE9040100F02A
:1011A000A9FB02460B463046394600F0F1F90246EB
:1011B0000B462046294600F0E9F942464B4600F02E
:1011C000E5F902460B46DDE9000100F0DFF9D1E662
:1011D00002460B4600F0DAF90022002300F0B4FCCE
:1011E000C8E6304600F020FB2DA3D3E900230646D5
:1011F0000F4600F07FFB2CA3D3E9002382468B46E9
:101200003046394600F076FB22462B4600F0C0F906
:1012100042464B4600F0BAF902460B465046594644
:1012200000F0B4F9A6E6304600F0FEFA1CA3D3E9BC
:10123000002306460F4600F05DFB1DA3D3E9002303
:1012400004460D463046394600F054FB02460B4634
:101250002046294600F09CF98CE600BFAFF30080E1
:1012600044523EDF12F1C23FDE03CB966446C73FD5
:10127000599322942449D23F935555555555E53FEE
:101280009FC678D0099AC33FAF788E1DC571CC3FF9
:1012900004FA97999999D93F555555555555D5BF44
:1012A0000000E0FE422EE63F763C7935EF39EABD9C
:1012B000763C7935EF39EA3D02460B4640464946D1
:1012C00000F064F9DDE9022300F014FBE5E600BF5D
:1012D00002464042104321F0004141EAD070C0F183
:1012E000FE4000F57000C00F704700BF002070473F
:1012F00040F200010020C7F6F871704740F2381341
:10130000C2F20003186870474A1E08BF7047C0F059
:101310002481884240F21681114200F01781B0FA10
:1013200080F3B1FA81F2A2EB0303C3F11F0304A21D
:1013300002EB03134FF000029F4600BFAFF30080A3
:10134000B0EBC17F00BF42EB020228BFA0EBC1702F
:10135000B0EB817F00BF42EB020228BFA0EB81709F
:10136000B0EB417F00BF42EB020228BFA0EB41700F
:10137000B0EB017F00BF42EB020228BFA0EB01707F
:10138000B0EBC16F00BF42EB020228BFA0EBC1600F
:10139000B0EB816F00BF42EB020228BFA0EB81607F
:1013A000B0EB416F00BF42EB020228BFA0EB4160EF
:1013B000B0EB016F00BF42EB020228BFA0EB01605F
:1013C000B0EBC15F00BF42EB020228BFA0EBC150EF
:1013D000B0EB815F00BF42EB020228BFA0EB81505F
:1013E000B0EB415F00BF42EB020228BFA0EB4150CF
:1013F000B0EB015F00BF42EB020228BFA0EB01503F
:10140000B0EBC14F00BF42EB020228BFA0EBC140CE
:10141000B0EB814F00BF42EB020228BFA0EB81403E
:10142000B0EB414F00BF42EB020228BFA0EB4140AE
:10143000B0EB014F00BF42EB020228BFA0EB01401E
:10144000B0EBC13F00BF42EB020228BFA0EBC130AE
:10145000B0EB813F00BF42EB020228BFA0EB81301E
:10146000B0EB413F00BF42EB020228BFA0EB41308E
:10147000B0EB013F00BF42EB020228BFA0EB0130FE
:10148000B0EBC12F00BF42EB020228BFA0EBC1208E
:10149000B0EB812F00BF42EB020228BFA0EB8120FE
:1014A000B0EB412F00BF42EB020228BFA0EB41206E
:1014B000B0EB012F00BF42EB020228BFA0EB0120DE
:1014C000B0EBC11F00BF42EB020228BFA0EBC1106E
:1014D000B0EB811F00BF42EB020228BFA0EB8110DE
:1014E000B0EB411F00BF42EB020228BFA0EB41104E
:1014F000B0EB011F00BF42EB020228BFA0EB0110BE
:10150000B0EBC10F00BF42EB020228BFA0EBC1004D
:10151000B0EB810F00BF42EB020228BFA0EB8100BD
:10152000B0EB410F00BF42EB020228BFA0EB41002D
:10153000B0EB010F00BF42EB020228BFA0EB01009D
:10154000104670470CBF012000207047B1FA81F2AD
:10155000C2F11F0220FA02F0704708B14FF0FF30CD
:1015600000F00EB80029F8D02DE90340FFF7CCFEBB
:10157000BDE8064002FB00F3A1EB0301704700BF8A
:10158000704700BF81F0004102E000BF83F00043DC
:1015900030B54FEA41044FEA430594EA050F08BF0E
:1015A00090EA020F1FBF54EA000C55EA020C7FEAD2
:1015B000645C7FEA655C00F0E2804FEA5454D4EB4F
:1015C0005555B8BF6D420CDD2C4480EA020281EA19
:1015D000030382EA000083EA010180EA020281EA51
:1015E0000303362D88BF30BD11F0004F4FEA0131A3
:1015F0004FF4801C4CEA113102D0404261EB4101B2
:1016000013F0004F4FEA03334CEA133302D0524237
:1016100063EB430394EA050F00F0A780A4F10104F3
:10162000D5F1200E0DDB02FA0EFC22FA05F280182D
:1016300041F1000103FA0EF2801843FA05F3594113
:101640000EE0A5F120050EF1200E012A03FA0EFC92
:1016500028BF4CF0020C43FA05F3C01851EBE371BC
:1016600001F0004507D54FF0000EDCF1000C7EEBD9
:1016700000006EEB0101B1F5801F1BD3B1F5001F17
:101680000CD349085FEA30004FEA3C0C04F1010436
:101690004FEA445212F5800F80F09A80BCF1004F5F
:1016A00008BF5FEA500C50F1000041EB045141EAE1
:1016B000050130BD5FEA4C0C404141EB010111F4E2
:1016C000801FA4F10104E9D191F0000F04BF01468D
:1016D0000020B1FA81F308BF2033A3F10B03B3F16B
:1016E00020020CDA0C3208DD02F1140CC2F10C02FB
:1016F00001FA0CF021FA02F10CE002F11402D8BF59
:10170000C2F1200C01FA02F120FA0CFCDCBF41EA24
:101710000C019040E41AA2BF01EB0451294330BDF3
:101720006FEA04041F3C1CDA0C340EDC04F11404D0
:10173000C4F1200220FA04F001FA02F340EA0300A7
:1017400021FA04F345EA030130BDC4F10C04C4F1ED
:10175000200220FA02F001FA04F340EA03002946CD
:1017600030BD21FA04F0294630BD94F0000F83F417
:10177000801306BF81F480110134013D4EE77FEAFA
:10178000645C18BF7FEA655C29D094EA050F08BF46
:1017900090EA020F05D054EA000C04BF1946104627
:1017A00030BD91EA030F1EBF0021002030BD5FEA6B
:1017B000545C05D14000494128BF41F0004130BD93
:1017C00014F580043CBF01F5801130BD01F00045E7
:1017D00045F0FE4141F470014FF0000030BD7FEA5A
:1017E000645C1ABF194610467FEA655C1CBF0B4655
:1017F000024650EA013406BF52EA033591EA030F6C
:1018000041F4002130BD00BF90F0000F04BF002163
:10181000704730B54FF4806404F132044FF0000596
:101820004FF0000150E700BF90F0000F04BF00210F
:10183000704730B54FF4806404F1320410F0004575
:1018400048BF40424FF000013EE700BF42004FEA70
:10185000E2014FEA31014FEA02701FBF12F07F43ED
:1018600093F07F4F81F06051704792F0000F14BFEA
:1018700093F07F4F704730B54FF4607401F000452E
:1018800021F0004120E700BF50EA010208BF704785
:1018900030B54FF000050AE050EA010208BF70477A
:1018A00030B511F0004502D5404261EB41014FF4E3
:1018B000806404F132045FEA915C3FF4DCAE4FF0E7
:1018C00003025FEADC0C18BF03325FEADC0C18BFCE
:1018D000033202EBDC02C2F1200300FA03FC20FA1F
:1018E00002F001FA03FE40EA0E0021FA02F114446C
:1018F000C1E600BF70B54FF0FF0C4CF4E06C1CEA81
:1019000011541DBF1CEA135594EA0C0F95EA0C0FF5
:1019100000F0DEF82C4481EA030621EA4C5123EA68
:101920004C5350EA013518BF52EA033541F4801197
:1019300043F4801338D0A0FB02CE4FF00005E1FB4A
:1019400002E506F00042E0FB03E54FF00006E1FB94
:1019500003569CF0000F18BF4EF0010EA4F1FF04D7
:10196000B6F5007F64F5407404D25FEA4E0E6D4117
:1019700046EB060642EAC62141EA55514FEAC52028
:1019800040EA5E504FEACE2EB4F1FD0C88BFBCF5A4
:10199000E06F1ED8BEF1004F08BF5FEA500E50F155
:1019A000000041EB045170BD06F0004646EA01011B
:1019B00040EA020081EA0301B4EB5C04C2BFD4EB4D
:1019C0000C0541EA045170BD41F480114FF0000E46
:1019D000013C00F3AB8014F1360FDEBF002001F0B4
:1019E000004170BDC4F10004203C35DA0C341BDC2E
:1019F00004F11404C4F1200500FA05F320FA04F000
:101A000001FA05F240EA020001F0004221F0004133
:101A100010EBD37021FA04F642EB06015EEA430EA6
:101A200008BF20EAD37070BDC4F10C04C4F12005D6
:101A300000FA04F320FA05F001FA04F240EA020089
:101A400001F0004110EBD37041F100015EEA430E5A
:101A500008BF20EAD37070BDC4F1200500FA05F27A
:101A60004EEA020E20FA04F301FA05F243EA0203F9
:101A700021FA04F001F0004121FA04F220EA020008
:101A800000EBD3705EEA430E08BF20EAD37070BD4E
:101A900094F0000F0FD101F00046400041EB01012E
:101AA00011F4801F08BF013CF7D041EA060195F010
:101AB000000F18BF704703F00046520043EB0303CA
:101AC00013F4801F08BF013DF7D043EA06037047B7
:101AD00094EA0C0F0CEA135518BF95EA0C0F0CD0C2
:101AE00050EA410618BF52EA4306D1D181EA030108
:101AF00001F000414FF0000070BD50EA410606BF02
:101B00001046194652EA430619D094EA0C0F02D146
:101B100050EA013613D195EA0C0F05D152EA03368B
:101B20001CBF104619460AD181EA030101F00041A9
:101B300041F0FE4141F470014FF0000070BD41F0F2
:101B4000FE4141F4780170BD70B54FF0FF0C4CF4CC
:101B5000E06C1CEA11541DBF1CEA135594EA0C0FEB
:101B600095EA0C0F00F0A7F8A4EB050481EA030E38
:101B700052EA03354FEA013100F088804FEA03331F
:101B80004FF0805545EA131343EA12634FEA0222ED
:101B900045EA111545EA10654FEA00260EF00041AE
:101BA0009D4208BF964244F1FD0404F5407402D200
:101BB0005B084FEA3202B61A65EB03055B084FEA91
:101BC00032024FF480104FF4002CB6EB020E75EB8E
:101BD000030E22BFB61A754640EA0C005B084FEAB6
:101BE0003202B6EB020E75EB030E22BFB61A754633
:101BF00040EA5C005B084FEA3202B6EB020E75EB7E
:101C0000030E22BFB61A754640EA9C005B084FEAF5
:101C10003202B6EB020E75EB030E22BFB61A754602
:101C200040EADC0055EA060E18D04FEA051545EAF1
:101C300016754FEA06164FEAC30343EA52734FEA9A
:101C4000C2025FEA1C1CC0D111F4801F0BD141EA13
:101C500000014FF000004FF0004CB6E711F4801F78
:101C600004BF01430020B4F1FD0C88BFBCF5E06F58
:101C70003FF6AFAEB5EB030C04BFB6EB020C5FEA68
:101C8000500C50F1000041EB045170BD0EF0004EBD
:101C90004EEA113114EB5C04C2BFD4EB0C0541EAEF
:101CA000045170BD41F480114FF0000E013C90E6EC
:101CB00045EA060E8DE60CEA135594EA0C0F08BFB0
:101CC00095EA0C0F3FF43BAF94EA0C0F0AD150EAAF
:101CD00001347FF434AF95EA0C0F7FF425AF104642
:101CE00019462CE795EA0C0F06D152EA03353FF46A
:101CF000FDAE1046194622E750EA410618BF52EAE7
:101D000043067FF4C5AE50EA41047FF40DAF52EABA
:101D100043057FF4EBAE12E74FF0FF3C06E000BF57
:101D20004FF0010C02E000BF4FF0010C4DF804CD64
:101D30004FEA410C7FEA6C5C4FEA430C18BF7FEA24
:101D40006C5C1BD001B050EA410C0CBF52EA430C52
:101D500091EA030F02BF90EA020F0020704710F1D2
:101D6000000F91EA030F58BF994208BF90422CBF61
:101D7000D8176FEAE37040F0010070474FEA410C5A
:101D80007FEA6C5C02D150EA013C07D14FEA430C78
:101D90007FEA6C5CD6D152EA033CD3D05DF8040BE9
:101DA000704700BF8446104662468C46194663461B
:101DB00000E000BF01B5FFF7B7FF002848BF10F1F2
:101DC000000F01BD4DF808EDFFF7F4FF0CBF012037
:101DD00000205DF808FB00BF4DF808EDFFF7EAFFB3
:101DE00034BF012000205DF808FB00BF4DF808ED6E
:101DF000FFF7E0FF94BF012000205DF808FB00BF63
:101E00004DF808EDFFF7CEFF94BF012000205DF8EC
:101E100008FB00BF4DF808EDFFF7C4FF34BF0120F9
:101E200000205DF808FB00BF4FEA410212F50012E6
:101E300015D211D56FF47873B3EB625212D94FEA11
:101E4000C12343F0004343EA505311F0004F23FAFB
:101E500002F018BF404270474FF00000704750EA50
:101E6000013005D111F0004008BF6FF0004070470D
:101E70004FF00000704700BF4FEA4102B2F1E0436B
:101E800024BFB3F5001CDCF1FE5C0DD901F0004C61
:101E90004FEAC0024CEA5070B2F1004F40EB8300B1
:101EA00008BF20F00100704711F0804F21D113F1DD
:101EB0003872BCBF01F00040704741F480114FEA16
:101EC0005252C2F11802C2F1200C10FA0CF320FA9F
:101ED00002F018BF40F001004FEAC1234FEAD323BC
:101EE00003FA0CFC40EA0C0023FA02F34FEA430326
:101EF000CCE77FEA625307D150EA01331EBF4FF0AF
:101F0000FE4040F44000704701F0004040F0FE40C9
:101F100040F40000704700BF80F0004002E000BFC6
:101F200081F0004142001FBF5FEA410392EA030FC4
:101F30007FEA226C7FEA236C6AD04FEA1262D2EB0E
:101F40001363C1BFD218414048404140B8BF5B4213
:101F5000192B88BF704710F0004F40F4000020F0AC
:101F60007F4018BF404211F0004F41F4000121F0C2
:101F70007F4118BF494292EA030F3FD0A2F101020C
:101F800041FA03FC10EB0C00C3F1200301FA03F14A
:101F900000F0004302D5494260EB4000B0F5000F6D
:101FA00013D3B0F1807F06D340084FEA310102F12C
:101FB0000102FE2A51D2B1F1004F40EBC25008BFDE
:101FC00020F0010040EA03007047490040EB0000A8
:101FD00010F4000FA2F10102EDD1B0FA80FCACF1D7
:101FE000080CB2EB0C0200FA0CF0AABF00EBC250D6
:101FF00052421843BCBFD0401843704792F0000FC4
:1020000081F4000106BF80F400000132013BB5E716
:102010004FEA41037FEA226C18BF7FEA236C21D08C
:1020200092EA030F04D092F0000F08BF08467047F1
:1020300090EA010F1CBF0020704712F07F4F04D1BF
:10204000400028BF40F00040704712F100723CBFD2
:1020500000F50000704700F0004343F0FE4040F4FC
:10206000000070477FEA226216BF08467FEA2363BA
:102070000146420206BF5FEA412390EA010F40F4A5
:10208000800070474FF0000304E000BF10F00043F1
:1020900048BF40425FEA000C08BF704743F09643D8
:1020A00001464FF000001CE050EA010208BF7047F3
:1020B0004FF000030AE000BF50EA010208BF70477A
:1020C00011F0004302D5404261EB41015FEA010C8F
:1020D00002BF84460146002043F0B64308BFA3F187
:1020E0008053A3F50003BCFA8CF2083AA3EBC25369
:1020F00010DB01FA02FC634400FA02FCC2F1200288
:10210000BCF1004F20FA02F243EB020008BF20F0BE
:102110000100704702F1200201FA02FCC2F1200224
:1021200050EA4C0021FA02F243EB020008BF20EA19
:10213000DC7070474FF0FF0C1CEAD0521EBF1CEA47
:10214000D15392EA0C0F93EA0C0F6FD01A4480EA35
:10215000010C400218BF5FEA41211ED04FF000631E
:1021600043EA501043EA5111A0FB01310CF000404A
:10217000B1F5000F3EBF490041EAD3715B0040EA70
:10218000010062F17F02FD2A1DD8B3F1004F40EB40
:10219000C25008BF20F00100704790F0000F0CF013
:1021A000004C08BF49024CEA502040EA51207F3AD7
:1021B000C2BFD2F1FF0340EAC250704740F40000B2
:1021C0004FF00003013A5DDC12F1190FDCBF00F0A3
:1021D00000407047C2F10002410021FA02F1C2F151
:1021E000200200FA02FC5FEA310040F1000053EAED
:1021F0004C0308BF20EADC70704792F0000F00F03B
:10220000004C02BF400010F4000F013AF9D040EA40
:102210000C0093F0000F01F0004C02BF490011F4D4
:10222000000F013BF9D041EA0C018FE70CEAD153D2
:1022300092EA0C0F18BF93EA0C0F0AD030F0004C52
:1022400018BF31F0004CD8D180EA010000F0004006
:10225000704790F0000F17BF90F0004F084691F0C4
:10226000000F91F0004F14D092EA0C0F01D14202FE
:102270000FD193EA0C0F03D14B0218BF084608D1C7
:1022800080EA010000F0004040F0FE4040F4000011
:10229000704740F0FE4040F4400070474FF0FF0CA4
:1022A0001CEAD0521EBF1CEAD15392EA0C0F93EAEB
:1022B0000C0F69D0A2EB030280EA010C49024FEA3D
:1022C000402037D04FF0805343EA111143EA1013F6
:1022D0000CF000408B4238BF5B0042F17D024FF4AE
:1022E000000C8B4224BF5B1A40EA0C00B3EB510F89
:1022F00024BFA3EB510340EA5C00B3EB910F24BF72
:10230000A3EB910340EA9C00B3EBD10F24BFA3EBF6
:10231000D10340EADC001B0118BF5FEA1C1CE0D1BE
:10232000FD2A3FF650AF8B4240EBC25008BF20F071
:10233000010070470CF0004C4CEA50207F32C2BFC5
:10234000D2F1FF0340EAC250704740F400004FF062
:102350000003013A37E792F0000F00F0004C02BF93
:10236000400010F4000F013AF9D040EA0C0093F05D
:10237000000F01F0004C02BF490011F4000F013BB7
:10238000F9D041EA0C0195E70CEAD15392EA0C0F1F
:1023900008D142027FF47DAF93EA0C0F7FF470AF57
:1023A000084676E793EA0C0F04D14B023FF44CAF9A
:1023B00008466EE730F0004C18BF31F0004CCAD12F
:1023C00030F000427FF45CAF31F000437FF43CAF6B
:1023D0005FE700BF4FF0FF3C06E000BF4FF0010C8D
:1023E00002E000BF4FF0010C4DF804CD4FEA40026F
:1023F0004FEA41037FEA226C18BF7FEA236C11D0B9
:1024000001B052EA530C18BF90EA010F58BFB2EB6B
:10241000030088BFC81738BF6FEAE17018BF40F0EB
:10242000010070477FEA226C02D15FEA402C05D19F
:102430007FEA236CE4D15FEA412CE1D05DF8040B24
:10244000704700BF844608466146FFE70FB5FFF7B7
:10245000C9FF002848BF10F1000F0FBD4DF808ED6F
:10246000FFF7F4FF0CBF012000205DF808FB00BF60
:102470004DF808EDFFF7EAFF34BF012000205DF8BA
:1024800008FB00BF4DF808EDFFF7E0FF94BF012007
:1024900000205DF808FB00BF4DF808EDFFF7D2FF04
:1024A00094BF012000205DF808FB00BF4DF808ED47
:1024B000FFF7C8FF34BF012000205DF808FB00BF14
:1024C00042000ED2B2F1FE4F0BD34FF09E03B3EB9E
:1024D000126209D44FEA002343F0004323FA02F0CA
:1024E00070474FF00000704712F1610F01D14202B6
:1024F00002D14FF0FF3070474FF00000704700BF2F
:1025000073B96AB9002908BF0028BCBF00204FF08A
:102510000041C4BF6FF000414FF0FF30FFF730B80B
:1025200082B0EC462DE9005000F01CF8DDF804E024
:1025300002B00CBC704700BFF8B514461D460646F5
:102540000F4600F0D3F900FB05F5A0FB042304FBC4
:102550000154E318B61A67EB0307069BC3E900674B
:10256000F8BD00BFF8B514461D4606460F4600F0FC
:102570000FF800FB05F5A0FB042304FB0154E3184E
:10258000B61A67EB0307069BC3E90067F8BD00BFF7
:1025900000292DE9F04F85B0C0F2C9800026002B3C
:1025A000C0F2C0808946144605469B46002B4BD19D
:1025B0008A4258D9B2FA82F353B1C3F1200001FA2A
:1025C00003F925FA00F812FA03F49D4048EA0909D4
:1025D000270C484639461FFA84FBFEF795FE39461C
:1025E00082464846FEF7BEFF4FEA15420BFB0AF350
:1025F00042EA01494B4509D919EB04090AF1FF3AAE
:1026000004D24B4584BF0AF1FF3AA144C3EB090948
:1026100039464846ADB2FEF777FE39468046484611
:10262000FEF7A0FF0BFB08FB45EA0145AB4507D9C8
:102630002D1908F1FF3803D2AB4588BF08F1FF38E8
:1026400048EA0A48002703E08B4257D90027B846DA
:1026500042463B4616B1524263EB430319461046CD
:1026600005B0BDE8F08F22B911460120FEF74CFEFF
:102670000446B4FA84F8B8F1000F5ED1C4EB09083F
:10268000270C1FFA84F90121029139464046FEF7D2
:102690003BFE394682464046FEF764FF4FEA154846
:1026A00009FB0AF348EA014B5B4509D91BEB040B14
:1026B0000AF1FF3A04D25B4584BF0AF1FF3AA34412
:1026C000C3EB0B0B39465846ADB2FEF71DFE39463B
:1026D00080465846FEF746FF09FB08F945EA0145E2
:1026E000A94507D92D1908F1FF3803D2A94588BF9C
:1026F00008F1FF3848EA0A48029FA9E7B3FA83F7CE
:10270000002F67D18B422CBF4FF000094FF0010919
:1027100082428CBF4C4649F00104002C96D04FF009
:10272000010895E7524263EB4303F6433AE7404220
:1027300061EB41014FF0FF3631E704FA08F4C8F1CC
:10274000200735FA07F329FA07FA270C09FA08FBDC
:102750003946504643EA0B020292FEF7D5FD394650
:102760001FFA84F983465046FEF7FCFE029809FBE7
:102770000BF2030C43EA01439A4204D91B190BF1F3
:10278000FF3BC0F0AD809B1A394618460193FEF717
:10279000BBFD0199824608463946FEF7E3FE0298E2
:1027A00009FB0AF31FFA80FC4CEA0142934208D964
:1027B00012190AF1FF3A04D2934284BF0AF1FF3A98
:1027C000121905FA08F54AEA0B4EC3EB0208CDF8D8
:1027D00008E05AE7C7F1200003FA07FAC24035FAC9
:1027E00000F342EA0A0B21FA00F801FA07F9404621
:1027F0004FEA1B4A43EA0901029151461FFA8BF244
:102800000392FEF781FD514681464046FEF7AAFE3F
:102810000398029B00FB09F2180C14FA07F340EA34
:102820000144A24204D914EB0B0409F1FF3951D33E
:10283000A41A514620460193FEF766FD5146804694
:102840002046FEF78FFE039C019B04FB08F2029CCE
:102850001FFA84FC4CEA0140824204D910EB0B00C1
:1028600008F1FF3830D348EA09481FFA83FC1B0CF3
:10287000801A1FFA88FE4FEA184A0CFB0EF90CFB6F
:102880000AF203FB0E2103FB0AF301EB19418A4212
:1028900088BF03F5803303EB114E704510D31FFA48
:1028A00089F905FA07F709EB014014BF002201225C
:1028B00087422CBF002702F00107002F3FF4C8AE6B
:1028C00008F1FF380027C3E6824284BF584408F16C
:1028D000FF38C8E7A24284BF09F1FF395C44A7E78B
:1028E0009A4284BF0BF1FF3B1B194CE72DE9F04FD7
:1028F0000C4683B08046164689461F4615468A46D2
:10290000002B4BD18A425CD9B2FA82F35BB1C3F19E
:10291000200001FA03FA28FA00F216FA03F508FA81
:1029200003F842EA0A0A2E0C50463146AFB2FEF7CF
:10293000EBFC31464FEA184481465046FEF712FE42
:1029400007FB09F344EA014A534509D91AEB050A82
:1029500009F1FF3904D2534584BF09F1FF39AA4474
:10296000C3EB0A0A314650461FFA88F8FEF7CCFC42
:10297000314604465046FEF7F5FD07FB04F748EAEA
:102980000148474506D9013C18EB050802D24745E6
:1029900088BF013C44EA094400265CE08B4258D8D9
:1029A000B3FA83F6002E5BD18B422CBF00220122AA
:1029B00085428CBF154642F00105002D49D0012407
:1029C00049E022B911460120FEF79EFC0546B5FA02
:1029D00085F6002E40F0BB80641B2F0C1FFA85FA91
:1029E000012639462046FEF78FFC39464FEA184B40
:1029F00081462046FEF7B6FD0AFB09F34BEA014B80
:102A00005B4509D91BEB050B09F1FF3904D25B4586
:102A100084BF09F1FF39AB44C3EB0B0B3946584671
:102A20001FFA88F8FEF770FC394604465846FEF750
:102A300099FD0AFB04FA48EA0148C24506D9013C5F
:102A400018EB050802D2C24588BF013C44EA09449C
:102A500001E0002634463146204603B0BDE8F08F41
:102A6000C6F12000B34032FA00F721FA00FB1F4301
:102A700014FA06F228FA00F158464FEA174A1143B1
:102A800000915146BBB20193FEF73EFC5146B54062
:102A900081465846FEF766FD019C009804FB09F349
:102AA0004FEA104C4CEA014B5B4505D91BEB070B79
:102AB00009F1FF39C0F08F80C3EB0B0B514658462C
:102AC000FEF722FC514604465846FEF74BFD01989E
:102AD000009A00FB04F31FFA82FC4CEA0142934285
:102AE00006D9013CD21903D2934201D9D219013C33
:102AF00044EA0944A8B2D21A2D0C1FFA84FC4FEA0A
:102B0000144300FB0CF700FB03FE05FB0CE105FB87
:102B100003F501EB17418E4588BF05F5803505EBC0
:102B20001145AA4210D3BFB208FA06F607EB0142DC
:102B300014BF4FF0000E4FF0010E96422CBF00263E
:102B40000EF00106002E86D0013C002683E7B5403A
:102B5000C6F1200124FA01F928FA01F22F0CB44041
:102B60003946484622430092FEF7CEFB39461FFA0B
:102B700085FA83464846FEF7F5FC009B1A0C0AFBD3
:102B80000BF342EA0144A34203D964190BF1FF3B62
:102B900027D3E41A39462046FEF7B6FB394681466C
:102BA0002046FEF7DFFC00980AFB09F31FFA80FCC1
:102BB0004CEA0144A34208D9641909F1FF3904D24F
:102BC000A34284BF09F1FF39641908FA06F8E41A30
:102BD00049EA0B4605E75B4584BF09F1FF39BB4471
:102BE0006AE7A34284BF0BF1FF3B6419D1E700BF42
:102BF0000000000000000000010003E800000000E9
:102C000000000003E800000000000200FA060003D4
:102C10000000000000370600000000000000000077
:102C2000F4010000640000000180080800000000BA
:102C3000006400000000000000000000C800000068
:102C40001201100102000040D016510601180102C5
:102C50000301000009024300020100C03209040020
:102C600000010202010005240010010524010001F9
:102C7000042402020524060001070582030800FF60
:102C800009040100020A00000007050302400000D9
:102C900007058102400000000403090426035400D4
:102CA000720069006E0061006D00690063004D00F4
:102CB0006F00740069006F006E0020004300740014
:102CC0006C000000320354004D0043004D002D0005
:102CD0003100310036003000200028007600690005
:102CE00072007400750061006C00200043004F000A
:102CF0004D00290020000000524F520000010652F2
:102D00004F4C000002064D5354000003024D565034
:102D100000000407534150000005074741500000E0
:102D20000603535441500007035253415000080317
:102D30005347500000090747475000000A03535407
:102D40004750000B0352534750000C0352465300A8
:102D5000000D0353494F00000E0747494F00000F75
:102D60000353414300001D0753434F00001E074714
:102D7000434F00001F0343434F0000200341434FD4
:102D8000000027035546300000400755463100003B
:102D900041075546320000420755463300004307BD
:102DA0005546340000440755463500004507554652
:102DB00036000046075546370000470752554E007B
:102DC00000810553544F5000800042494E00008B53
:102DD00000000000000000000200000000000001F0
:102DE00000000000010203040102030406070809B1
:102DF000020406080020202020202020202028284F
:102E000028282820202020202020202020202020AA
:102E100020202020208810101010101010101010EA
:102E2000101010101004040404040404040404101A
:102E300010101010101041414141414101010101A8
:102E40000101010101010101010101010101010172
:102E5000101010101010424242424242020202027E
:102E60000202020202020202020202020202020242
:102E700010101010200000000000000000000000F2
:102E80000000000000000000000000000000000042
:102E90000000000000000000000000000000000032
:102EA0000000000000000000000000000000000022
:102EB0000000000000000000000000000000000012
:102EC0000000000000000000000000000000000002
:102ED00000000000000000000000000000000000F2
:102EE00000000000000000000000000000000000E2
:102EF000000000000000000031313630563132341D
:102F0000004142530052454C00434F4F524400533E
:102F1000544152540053544F50005354415455534C
:102F200000000000430000006C6F6700000000001C
:082F300060F6FF7F01000000C4
:102F3800F82E01080001000000010200000800004E
:102F48000100000002000000000000000000000076
:102F58000000000000000000000000000000000069
:102F68000000000000000000000000000000000059
:102F7800000000000000000000C20100000008007E
:102F8800982C0108040000009C2C01082600000071
:102F9800C42C010832000000B00000201A00000014
:102FA800542C010843000000402C010812000000C6
:102FB800F9A00008059F0008159D0008299D000834
:102FC8002D9D00088D9D0008B19D0008F59E000804
:102FD800E59E0008C19E00080000000040000000B7
:102FE8001A0354004D004300310031003600300010
:102FF800000000000000000000000000159C000810
:1030080099FB000899FB000899FB000899FB000848
:1030180099FB000899FB000899FB000899FB000838
:1030280055A0000899FB000899FB000899FB0008C7
:1030380099FB00080401000099FB0008F19C0008B6
:1030480099FB000899FB000899FB000899FB000808
:1030580099FB000899FB0008099D00080100000081
:10306800F52D0108F42D01083C01002000000000A6
:103078000000000000000000000000000000000048
:10308800000000000000000000000000242F0108DC
:103098000000000000000000000000000000000028
:1030A8000000000000000000000000000000000018
:1030B8000000000000000000000000000000000008
:1030C80000000000000000000000000000000000F8
:1030D80000000000000000000000000000000000E8
:1030E80000000000000000000000000000000000D8
:1030F80000000000000000000000000000000000C8
:1031080000000000000000000000000000000000B7
:1031180000000000000000000000000000000000A7
:103128000000000000000000000000000000000097
:103138000000000000000000000000000000000087
:103148000000000000000000000000000000000077
:103158000000000000000000000000000100000066
:04000005080041109E
:00000001FF
